:100000000C9424090C9443090C9443090C94D509CD
:100010000C940B0A0C9443090C9443090C94430967
:100020000C9443090C9443090C9443090C94430920
:100030000C9443090C9443090C9443090C94360D19
:100040000C9443090C9443090C9443090C94430900
:100050000C94B36C0C9464640C9443090C944309A1
:100060000C9443090C9439650C9443090C942D6548
:100070000C9443090C9443090C9443090C944309D0
:100080000C94E6770C9443090C9443090C944309AF
:100090000C9477650C9443090C946B650C9443099C
:1000A0000C9443090C9443090C9443090C944309A0
:1000B0000C9443090C9443090C9443090C94430990
:1000C0000C9443090C9443090C9443090C94430980
:1000D0000C9443090C9443090C9443090C94430970
:1000E0000C9443090C946C6C0C94766C0C94626CBC
:1000F0000C94226C0C94A76C0C94986C0C948C6CE3
:100100000C94806C0C9443090C9443090C9443099F
:100110000C9443090C9443090C9443090C9443092F
:100120001F813E81BD81AC82CC82EC82F482A182AF
:10013000084AD73B3BCE016E84BCBFFDC12F3D6C4E
:1001400074319ABD56833DDA3D00C77F11BED9E4B4
:10015000BB4C3E916BAAAABE000000803F076342E1
:1001600036B79BD8A71A39685618AEBAAB558C1D4E
:100170003CB7CC5763BD6DEDFD753EF6177231BFD0
:10018000000000803F08000000BE922449123EABF0
:10019000AAAA2ABECDCCCC4C3E00000080BEABAAA1
:1001A000AAAA3E00000000BF000000803F0000003F
:1001B0000000084178D3BB4387D1133D190E3CC3DF
:1001C000BD4282AD2B3E68EC8276BED98FE1A93E5E
:1001D0004C80EFFFBE01C4FF7F3F00000000002500
:1001E000730A005854414C5F5452494D3D256400F8
:1001F00025730A0025730A00546573742036202580
:10020000730A005465737420352025730A00546501
:10021000737420342025730A0054657374203320CE
:1002200025730A005465737420322025730A005424
:1002300065737420312025730A006368616E3D2563
:10024000640A0074787077723D25640A0035303096
:100250006B0A003235306B0A003131356B0A0035DC
:10026000366B0A0033386B0A0025730A00765F6C20
:100270006F773D252D332E32660A0025730A0073F1
:10028000656E743D252D75206475703D252D752096
:1002900069676E6F7265643D252D752074746C5F9F
:1002A0007A65726F3D252D750A0025372E3366203D
:1002B00025372E33660025352E32662000457272B2
:1002C0006F72203020566F6C74004E6F74207375FF
:1002D00070706F727465640A004572726F722030BC
:1002E00020566F6C74004572726F72203020566F0A
:1002F0006C7400256C7500416C6C6F7765642073BD
:100300007065656420312F31302F3130302F34301B
:1003100030206B6269742F730025630074746C3D28
:10032000252D64200074746C3D252D6420004E65DD
:10033000772074746C3D252D6420002563004D5397
:100340003536313120503D252D372E326620252D72
:10035000372E32666D0A00424D5030383520256CFC
:10036000642050612020252D372E32666D002563D4
:1003700000545F484541545F4944583D252D352E72
:1003800032662000545F4445573D252D352E326698
:10039000200041483D252D352E32662000545F5304
:1003A000485432583D252D352E3266200052485F84
:1003B00053485432583D252D352E32662000545F67
:1003C00052483D252D342E3166200052483D252DC2
:1003D000342E316620002563002563002563002547
:1003E00063002563007265706F72745F616C6C3DB1
:1003F000007265706F72743D0025630025630025EF
:100400006300256300204F534343414C3D25642046
:100410000020467573653A2065653D2530327820A9
:1004200068663D25303278206C663D253032782074
:100430006C623D25303278004D43553D2530366C99
:10044000780025630074785F6C656E3D252D6C75B2
:100450002C765F6C6F773D252D6C752C736874322C
:10046000783D252D6C750A002563004F4B0A002549
:100470006300256300256300256300256300256371
:100480000025630025630064656275675F616C6CBD
:100490003D0064656275673D0064656275673D0097
:1004A00025730A00646565700A006E6F6E650A0048
:1004B000707772733D00696E74725F7365635F700D
:1004C000313D252D372E33660A00696E74725F70D8
:1004D000313D252D6C640A00696E74725F7365632B
:1004E0005F70303D252D372E33660A00696E7472B9
:1004F0005F70303D252D6C640A00765F6D63753D3D
:10050000252D352E32660A00745F6D63753D252DED
:10051000352E32660A00707077723D25730A0064CA
:10052000656275673D0072636D643D25730A002541
:10053000730A006175746F0A006C6F675F6D6F649A
:10054000653D007573625F7077723D25730A0072B6
:10055000656C61793D25730A0074746C3D252D64CA
:100560000A0052494D455F616464723D252D642E39
:10057000252D640A006E65696768626F725F746139
:10058000626C655F73697A653D25640A00765F6C0D
:100590006F773D252D332E32660A00747870773DD3
:1005A00025640A006368616E3D25640A0069643D44
:1005B000006932635F6275733D006932635F737017
:1005C0006565643D252D6C750A007478743D25734E
:1005D0000A0053797374656D2053756D6D6172797E
:1005E0000A006D61736B3D002C00696E7465727654
:1005F000616C3D252D750023252D642C00745F68EA
:100600006561745F69647800745F64657700616830
:1006100000705F6D73353631310072685F736874D6
:10062000327800745F736874327800706100700013
:1006300061643400616433006164320061643100DC
:10064000613300613200613100765F696E0072686B
:100650000065727200757074696D650070315F6C51
:1006600073740070315F740070310070305F6C73B0
:10067000740070305F7400703000765F6D637500D9
:10068000745F6D63750074310074006964006536D1
:100690003400747874002D002B006175746F006E47
:1006A0006F6E6500706F7765725F736176655F6C02
:1006B000656472790072656C61795F6C656479005C
:1006C000636F6D7061737300616363656C0070725A
:1006D000657300705F707772006165730070315FE1
:1006E0006C6564790070305F6C6564720065766576
:1006F0006E74006C6564006F7700706B74007478C2
:100700005F6C6564790072785F6C656472006F700D
:100710006572006E6F6E65002530327800765F611D
:1007200064343D252D382E3666002000765F6164E6
:10073000333D252D382E3666002000765F61643209
:100740003D252D382E3666002000765F6164313DF0
:10075000252D382E3666002000765F6C6967687438
:100760003D252D382E3666002000765F61323D250E
:100770002D372E3366002000765F61313D252D3701
:100780002E3366002000765F696E3D252D352E32B2
:100790006600204E657665722D75736564207374EE
:1007A00061636B203E2025642062797465730A00C2
:1007B000757074696D653D252D642D646179732DA7
:1007C000253032643A253032643A253032642D685F
:1007D0006F7572730A0074657374205B6F66667C54
:1007E000317C327C337C347C355D202020202020FD
:1007F00020202D2074657374206D6F6465730A0D5D
:10080000007478205B706B74207061796C6F616428
:100810005D2020202020202020202020202D20733B
:10082000656E6420726164696F20706B74206B6503
:1008300079626F6172640A0D00776474205B6F6E79
:100840007C6F66667C746573745D20202020202098
:1008500020202020202D207761746368646F670A50
:100860000D00765F6C6F77205B765F6C6F775D2035
:1008700020202020202020202020202020202D206B
:100880006C6F77657374207265706F727420766F09
:100890006C746167650A0D007570677220202020F6
:1008A0002020202020202020202020202020202048
:1008B000202020202D207265626F6F742076696180
:1008C00020626F6F746C6F616465720A0D007561F0
:1008D0007274205B33386B7C35366B7C3131356B11
:1008E0007C3235306B7C3530306B5D202D2073656C
:1008F00074207465726D2F756172742073706565F4
:10090000640A0D00626F6F742020202020202020B8
:1009100020202020202020202020202020202020D7
:100920002D207265626F6F740A0D007077727320EC
:100930005B646565707C6E6F6E655D202020202095
:10094000202020202020202D206D637520736C65D1
:100950006570206D6F64650A0D00726573742065A3
:100960006570726F6D202020202020202020202004
:100970002020202020202D20726573746F72652046
:10098000656570726F6D0A0D0070707772205B6F15
:100990006E7C6F66665D2020202020202020202095
:1009A00020202020202D2070726F6772616D6D6194
:1009B000626C65207077720A0D00747874205B7326
:1009C0007472696E675D2020202020202020202066
:1009D0002020202020202D20536574207265706F08
:1009E0007274207465787420737472696E670A0D6E
:1009F0000074787077205B31352D305D2020202009
:100A0000202020202020202020202020202D2054A5
:100A100058205077722E20486967686573742030BB
:100A200020283364426D290A0D0074746C205B30F9
:100A30002D31355D20202020202020202020202046
:100A40002020202020202D2074696D652D746F2DAD
:100A50006C69766520666F72207061636B65747374
:100A60000A0D007373202020202020202020202029
:100A70002020202020202020202020202020202D69
:100A80002073797374656D2073756D6D6172790A69
:100A90000D007273202020202020202020202020E4
:100AA00020202020202020202020202020202D2039
:100AB000726164696F2073746174730A0D007269E6
:100AC000205B236E5D205B696E745D2020202020FA
:100AD000202020202020202020202D207265706FD3
:100AE000727420696E74657276616C0A0D007263AF
:100AF0006D64205B6F6E7C6F66665D202020202019
:100B0000202020202020202020202D20616C6C6FB0
:100B10007720636D642066726F6D206E65746F72EE
:100B20006B0A0D007265205B236E5D205B2B7C2DB4
:100B30005D205B6D61736B7C6175746F2C6D61738F
:100B40006B5D202D206D6F7465207265706F7274FF
:100B5000207365742F6D6F646966790A0D006F7775
:100B60002020202020202020202020202020202085
:100B7000202020202020202020202D206F6E652D79
:100B8000776972652073656E736F72730A0D006CFE
:100B90006F67205B6175746F7C6F6E7C6F66665DDE
:100BA00020202020202020202020202D206D6F7448
:100BB00065732064617461206F6E205553420A0D85
:100BC000006E65205B666C7573685D2020202020B8
:100BD000202020202020202020202020202D206EBA
:100BE00065696768626F72207461626C650A0D00E6
:100BF000657272202020202020202020202020200C
:100C00002020202020202020202020202D20657240
:100C1000726F722073746174730A0D006D637520B6
:100C200020202020202020202020202020202020C4
:100C300020202020202020202D206D637520696E2B
:100C4000666F0A0D00693263205B70726F62657CAB
:100C5000737065656420236E5D2020202020202095
:100C6000202D206932632070726F62652062757377
:100C70007C736574206275732073706565640A0DFA
:100C8000006964205B72657365745D2020202020FC
:100C9000202020202020202020202020202D2069FE
:100CA000642068616E646C696E670A0D0068756D1A
:100CB0002020202020202020202020202020202034
:100CC0002020202020202020202D2068756D6964A0
:100CD0006974792073656E736F720A0D0072656CAA
:100CE0006179205B6F6E7C6F66667C737461747370
:100CF0005D20202020202020202D2072656C61792D
:100D0000206E6574776F726B207265706F7274738A
:100D10000A0D006465205B6D61736B5D20202020EF
:100D20002020202020202020202020202020202DB6
:100D30002064656275670A0D006368616E205B312F
:100D4000312D32365D202020202020202020202020
:100D500020202020202D206368616E2031312D322B
:100D6000362028322E3430352D32343830204D683C
:100D70007A290A0D0063616C69205B5B765F696E9E
:100D80007C61317C61325D20766F6C747C7265733E
:100D900065747C6E6F6E655D202D2063616C696289
:100DA000726174650A0D0061646320202020202098
:100DB0002020202020202020202020202020202033
:100DC0002020202D2073686F7720765F696E2C209D
:100DD00061312C20613220766F6C74616765730A13
:100DE0000D007520202020202020202020202020E1
:100DF00020202020202020202020202020202D20E6
:100E0000757074696D650A0D007620202020202001
:100E100020202020202020202020202020202020D2
:100E200020202020202D2076657273696F6E0A0DB8
:100E3000006820202020202020202020202020208A
:100E4000202020202020202020202020202D20684D
:100E5000656C700A0D00256300756E6B6E6F776EA2
:100E600020636D640A00484D4335383833002573DC
:100E700000257300202573002025362E32662000C1
:100E8000253032780074656D705F65787465726EB8
:100E90003D252D362E326600202573002025362E66
:100EA0003266204F6E2D426F6172640025303278B9
:100EB0000074656D705F626F6172643D252D362E22
:100EC0003266000A00503A20256C642050612020D0
:100ED000252D372E3266206D0A002563002563001C
:100EE0004932433A2000452025642E256420636C56
:100EF0006F636B20256C752063707520256C7520E1
:100F00006C706D20256C752069727120256C7520C0
:100F1000676C656420256C7520796C656420256C90
:100F20007520726C656420256C7520747820256CA2
:100F300075206C697374656E20256C752073656E01
:100F4000736F727320256C752073657269616C20F4
:100F5000256C750A00532025642E256420636C6F70
:100F6000636B20256C7520747820256C7520727851
:100F700020256C752072747820256C75207272782B
:100F800020256C75207265786D697420256C75203C
:100F900061636B747820256C75206E6F61636B7470
:100FA0007820256C752061636B727820256C752024
:100FB00074696D65646F757420256C752062616459
:100FC00061636B727820256C7520746F6F6C6F6E27
:100FD0006720256C7520746F6F73686F727420259D
:100FE0006C752062616473796E636820256C75206E
:100FF00062616463726320256C7520636F6E746533
:101000006E74696F6E64726F7020256C75207365E5
:101010006E64696E6764726F7020256C75206C6CED
:10102000747820256C75206C6C727820256C750A9C
:1010300000257325730A004F6E6C696E650A000AFD
:10104000002C20636865636B2072617465202575D0
:1010500020487A0025732025732C206368616E6E0A
:10106000656C20257520706F776572202575000AE4
:101070000025783A004D41432061646472657373C2
:10108000200052616E646F6D2045554936342061F1
:101090006464726573732067656E657261746564FC
:1010A0000A000A2A2A2A2A2A2A2A426F6F74696E9B
:1010B000672025732A2A2A2A2A2A2A0A0045455007
:1010C000524F4D20697320636F72727570742C20BB
:1010D000726577726974696E6720776974682064D5
:1010E000656661756C74732E0A006C6F63616C6861
:1010F0006F73740041544D45474131323872666117
:101100003100020000FFFE0000016E616E00696E9A
:10111000660000407A10F35A00A0724E18090010C1
:10112000A5D4E80000E87648170000E40B5402005C
:1011300000CA9A3B000000E1F50500008096980087
:10114000000040420F000000A086010000001027B0
:1011500000000000E8030000000064000000000040
:101160000A00000000000100000000002C76D88872
:10117000DC674F0823DFC1DFAE59E1B1B796E5E385
:10118000E453C63AE651997696E8E6C28426EB899E
:101190008C9B62ED407C6FFCEFBC9C9F40F2BAA53B
:1011A0006FA5F490055A2AF75C936B6CF9676DC1D3
:1011B0001BFCE0E40D47FEF520E6B500D0ED902ED7
:1011C0000300943577050080841E080000204E0A35
:1011D000000000C80C333333330F986E1283114173
:1011E000EF8D2114893BE65516CFFEE6DB18D1843E
:1011F0004B381BF77C1D901DA4BBE4242032847265
:101200005E228100C9F124ECA1E53D274E414E4903
:101210004E495459494E46CDCCCC3D0AD7233C17B4
:10122000B7D13877CC2B329595E6241FB14F0A0001
:101230000020410000C84200401C4620BCBE4CCAF1
:101240001B0E5AAEC59D740011241FBECFEFD1E412
:10125000DEBFCDBF19E0A0E0B2E0EEECFBE201E0C2
:101260000BBF02C007900D92AE3BB107D9F711E357
:10127000AEEBB9E001C01D92A337B107E1F70E94C0
:10128000C3830C94E5950C9400008115910511F031
:101290000197F1F7089580EB94E09F938F930E945C
:1012A000BE928091580290915902A0915A02B09139
:1012B0005B020F900F9093FF03C08AEA94E002C094
:1012C00084EA94E09F938F930E94BE920F900F90B8
:1012D0000895E091771BEF71F0E0E453F44E8083C2
:1012E0008091771B8F5F8093771B8091AD288860FA
:1012F0008093AD284EE352E061E1CA010E9444545C
:1013000080E090E00895CF93DF93EC018091C509D0
:101310009091C60986FF1DC08E811F928F938D818B
:101320001F928F938C811F928F938B811F928F932B
:101330008A811F928F9385E693E09F938F930E94FB
:10134000AC928DB79EB70C960FB6F8949EBF0FBEA9
:101350008DBFBE018CEF99E00E947655BE0184E0FE
:1013600092E0DF91CF910C94EB548823B9F052981E
:101370005A981DBA80916900806280936900EA9A48
:1013800053985B98EB9A809169008068809369001C
:1013900080916800816080936800089510926900D0
:1013A0005A9AEA985B9AEB9808951F920F920FB69B
:1013B0000F9211248F939F93AF93BF9380916800F6
:1013C00080FF20C08091882890918928A0918A2848
:1013D000B0918B280196A11DB11D80938828909310
:1013E0008928A0938A28B0938B288091C509909171
:1013F000C60987FF07C0749882E090E09093850249
:1014000080938402BF91AF919F918F910F900FBEF7
:101410000F901F9018951F920F920FB60F921124E4
:101420008F939F93AF93BF938091680080FF20C0FC
:1014300080918C2890918D28A0918E28B0918F2832
:101440000196A11DB11D80938C2890938D28A093A7
:101450008E28B0938F288091C5099091C60990FF7E
:1014600007C0739882E090E0909385028093840295
:10147000BF91AF919F918F910F900FBE0F901F90D2
:10148000189580937C0080917B00877F80937B0000
:1014900080917C00806C80937C0085E080937A0052
:1014A00080917A00806880937A0080917B0087FF2A
:1014B000FCCF80917B0085FFFCCF80917A00806417
:1014C00080937A0080917A0086FDFCCF109279009B
:1014D0001092780084E090E060E070E020917A0063
:1014E000206420937A0020917A0026FDFCCF209181
:1014F000780030917900620F731F0197009771F7A0
:1015000010927C0080917A008F7780937A00769594
:1015100067957695679580E090E00E941989089517
:1015200080E00E94410A20917C0230917D0240912E
:101530007E0250917F020E94FD8A21EE3AE744E943
:101540005EE30E94B28708950F931F93CF93DF93BA
:10155000CFE1D0E00BE51EE0C093510187EC90E0B5
:101560000E9445098091510185FD0DC0C031D10512
:1015700021F02CF00B54110904C004EC19E00253C3
:1015800011092197E9CFB80180E090E00E94198904
:1015900020E030E04AE754E40E947C88DF91CF915C
:1015A0001F910F910895CF93DF93EC01888199816A
:1015B000009799F08736904121F01982188283E0D4
:1015C00011C0623171F40E94A40A60931F247093C9
:1015D0002024809321249093222487E690E199830C
:1015E000888381E0DF91CF91089580917B008860AE
:1015F00080937B0089EC80937C0085E080937A0067
:1016000080917A00806880937A0080917B0087FFC8
:10161000FCCF80917B0085FFFCCF80917A008064B5
:1016200080937A0080917A0086FDFCCF80917A00C9
:10163000806480937A0080917A0086FDFCCF60916F
:1016400078007091790080917A008F7780937A008A
:1016500080E090E00E94198927ED33EA40E95FE3DA
:101660000E94FD8A26E636E648E853E40E94B187E8
:101670000895BF92CF92DF92EF92FF920F931F9344
:10168000CF93DF93CDB7DEB729970FB6F894DEBFBF
:101690000FBECDBF6C011092BE098FEF898708E89D
:1016A0001BE1B12C7E0189E0E80EF11C89858823BD
:1016B000E9F1E8E0BE16E1F1BE016F5F7F4FC701BF
:1016C0000E94DF5D89858F3F11F08E3F19F4809372
:1016D000BE092CC0CE010196C114D10471F40E9440
:1016E000F85D8093AA28FE013196A2EAB8E28191C2
:1016F0008D93EE15FF05D9F71DC00E94F85DF80126
:101700008083FE01319620E030E0A8014850510965
:101710008191DA01A20FB31F8C932F5F3F4F2830C6
:101720003105B1F7B394075F1F4FC0CF8B2D03C0B6
:1017300088E001C081E029960FB6F894DEBF0FBEA5
:10174000CDBFDF91CF911F910F91FF90EF90DF9070
:10175000CF90BF90089583EC9EE09F938F930E945B
:10176000BE920F900F9008952F923F924F925F92EA
:101770006F927F928F929F92AF92BF92CF92DF92A1
:10178000EF92FF920F931F93CF93DF93EC014B01E6
:10179000009711F427E004C08130910549F426E058
:1017A0004AE250E06BE270E089E290E00E94BF5CA8
:1017B000CE010E94390B9E012154364F5901D901A7
:1017C0008C93CD2B69F098E8C92E9BE1D92EC0E807
:1017D000DBE1E12CF12C24E7222E2EE0322EA6C0F4
:1017E00082EA98E20E942D5FBC01882777FD8095F0
:1017F000982F0E941B896B017C01892869F020E0E9
:1018000030E048EC52E40E947C889F938F937F9352
:101810006F9381EB9EE0ACC0C2EAD8E20CEA1EE016
:1018200089911F928F931F930F930E94BE920F90E6
:101830000F900F900F90B8E2CA3ADB0789F720E0CB
:1018400030E048EC52E4C701B6010E947C889F93C7
:101850008F937F936F938CE99EE09F938F930E9469
:10186000BE920F900F900F900F900F900F9080915D
:10187000AA28882319F084E993E002C088E094E064
:101880009F938F9388E99EE09F938F930E94BE92CF
:101890000F900F900F900F9075C000E010E0FE01C8
:1018A000E00FF11F80811F928F93A0E8BEE0BF93ED
:1018B000AF930E94BE920F5F1F4F0F900F900F903B
:1018C0000F900830110559F720E030E048EC52E461
:1018D000C301B2010E947C889F938F937F936F9383
:1018E000A8E7BEE0BF93AF930E94BE920F900F9007
:1018F0000F900F900F900F90D6018C91882309F4D0
:1019000055C084E993E09F938F933F922F920E945A
:10191000BE920E94AB0BBFEFEB1AFB0AE9E0CE0EC2
:10192000D11C29960F900F900F900F90D5018C919C
:1019300090E0E816F906ECF5CE010E942D5FBC019F
:10194000882777FD8095982F0E941B892B013C01E9
:101950008114910409F4A1CF20E030E048EC52E476
:101960000E947C889F938F937F936F9385E89EE07E
:101970009F938F930E94BE920F900F900F900F90A5
:101980000F900F90DF91CF911F910F91FF90EF90EB
:10199000DF90CF90BF90AF909F908F907F906F908F
:1019A0005F904F903F902F900C94AB0B88E094E0A9
:1019B000AACFDF91CF911F910F91FF90EF90DF9011
:1019C000CF90BF90AF909F908F907F906F905F90DF
:1019D0004F903F902F900895CF93DF9300D0CDB7D5
:1019E000DEB78091A32889838091A9288A83CE01BC
:1019F00001960E9438520F900F90DF91CF91089579
:101A0000CF93DF93EC012091A2283091A32840913D
:101A1000A4285091A5286091A6287091A7288091AC
:101A2000A8289091A928AFEF0E942D8EE1F427E01D
:101A30004AE250E06BE270E089E290E00E94BF5C15
:101A400080E090E00E94390BC154D64F888349E072
:101A500050E06AE070E082EA98E20E943094DF9100
:101A6000CF910C94EC0CDF91CF9108951F920F92BF
:101A70000FB60F9211240BB60F92DF92EF92FF92E6
:101A80000F931F932F933F934F935F936F937F9386
:101A90008F939F93AF93BF93CF93DF93EF93FF9376
:101AA0008091AD2882608093AD288091580286FD98
:101AB0002B9A8091580287FD2B9A809184029091F5
:101AC00085021816190614F4749A739A8091C50940
:101AD0009091C60985FF02C07498739880910202A4
:101AE0009091030201979093030280930202892B45
:101AF00009F03DC18091D3099091D409019690934A
:101B0000D4098093D3098091232490912424A09117
:101B10002524B09126240196A11DB11D8093232474
:101B200090932424A0932524B093262480E190E070
:101B300090930302809302028091580280FD02C0BC
:101B40001D9B07C01092C3091092C20983B7817F01
:101B500009C081E090E09093C3098093C20983B7E4
:101B6000817F866083BF8091C5099091C60997FFE8
:101B700008C08091C2099091C309892B61F0749AC1
:101B8000739807E21BE1C4E3D4E234E0E32EF12CC6
:101B9000DD24D3941FC0739A7498F3CF8091D30936
:101BA0009091D40901960E94FE8B892BD1F0F80107
:101BB000608571856115710509F5F801608571858C
:101BC0006115710569F5065F1F4F2596FBE10F341E
:101BD0001F07D1F1F801608571856115710539F331
:101BE000DDCF77988091C5099091C60992FFDFCF2C
:101BF0007498F0928502E0928402D9CF8091D30943
:101C00009091D40901960E94FE8B892BB1F61C821B
:101C10001B82AE0162E186E192E00E944454CDCF86
:101C20008091D3099091D4090E94FE8B892B59F69B
:101C3000D8821A8309831C821B82AE0162E184E38D
:101C400092E00E944454BFCF60915E0270915F02A7
:101C500061157105A1F18091D3099091D4090E9479
:101C6000FE8B892B61F58091882890918928A0911D
:101C70008A28B0918B284091151C5091161C6091B8
:101C8000171C7091181C841B950BA60BB70B809327
:101C90004F1B9093501BA093511BB093521B8091EC
:101CA000882890918928A0918A28B0918B288093C8
:101CB000151C9093161CA093171CB093181C6091D0
:101CC0005C0270915D0261157105A1F18091D309EB
:101CD0009091D4090E94FE8B892B61F580918C280C
:101CE00090918D28A0918E28B0918F284091191C39
:101CF00050911A1C60911B1C70911C1C841B950B2D
:101D0000A60BB70B8093531B9093541BA093551BAA
:101D1000B093561B80918C2890918D28A0918E288D
:101D2000B0918F288093191C90931A1CA0931B1CB0
:101D3000B0931C1C8091580286FD2B98809158020C
:101D400090915902A0915A02B0915B0291FF0FC08D
:101D50000E94DE688A3119F0C1E0C80F01C0CBE0F3
:101D60000E9498678C2F0E94F6680E94E06740E00E
:101D700050E060E086E892E00E944454FF91EF91C9
:101D8000DF91CF91BF91AF919F918F917F916F9193
:101D90005F914F913F912F911F910F91FF90EF9085
:101DA000DF900F900BBE0F900FBE0F901F901895F5
:101DB0008091771B90913324891B08950E94D80E3F
:101DC000882371F0E0913324EF71F0E0E453F44E96
:101DD000808190E0209133242F5F20933324089555
:101DE0008FEF9FEF0895CF93DF93EC011092F009EE
:101DF0001092EF09888199810097C1F08A3793404A
:101E000021F01982188283E0B6C0613109F0B2C0B6
:101E1000F89478940E94DE0E99279093EB098093B2
:101E2000EA098D3009F441C08F3F49F40E94D80E71
:101E30008111EECF8AE793E0998388839BC082313A
:101E4000910509F458C08F37910509F050C0809171
:101E5000E8099091E909181619060CF560916D31A1
:101E600070916E3188E090E00E947A9260916D31BD
:101E700070916E3180E290E00E947A9260916D31B3
:101E800070916E3188E090E00E947A928091E8092A
:101E90009091E90901979093E9098093E80980916D
:101EA000E8099091E909CF9709F61092332410922E
:101EB000771B8091E8099091E909FC01E85BFB4DF3
:101EC00010829093F0098093EF091092E909109223
:101ED000E8098091AB289091AC28009709F4A6CF2F
:101EE00040E050E06091FE110E9444549FCF883042
:101EF000910571F5ACCF60916D3170916E318DE0CF
:101F000090E00E947A921092E7091092E60980917F
:101F1000E6099091E7092091E8093091E9098217D3
:101F200093070CF0BCCFFC01E85BFB4D8081609116
:101F30006D3170916E3190E00E947A928091E60945
:101F40009091E70901969093E7098093E609DFCF26
:101F500060916D3170916E310E947A928091E809A2
:101F60009091E9092091EA09FC01E85BFB4D20838F
:101F7000019691CF81E0DF91CF9108958091C209C0
:101F80009091C309892BD1F0809158029091590208
:101F9000A0915A02B0915B0293FD10C00E94986715
:101FA00083B7817F866083BFF89483B7816083BFE6
:101FB0007894889583B78E7F83BF78940895CF9364
:101FC000DF93EC0188819981009719F08A3990415B
:101FD00099F40E9455660E94BE0F40E050E065E80B
:101FE00080910212909103120E9444548AE990E178
:101FF0009983888381E003C01982188283E0DF918E
:10200000CF910895CF93DF9300D0CDB7DEB7892B62
:1020100081F05F934F9381E79EE09F938F93698355
:102020007A830E94BE920F900F900F900F907A814A
:1020300069817F936F938EE69EE09F938F930E94BA
:10204000BE920F900F900F900F900F900F90DF9116
:10205000CF910895FF920F931F93CF93DF930E9428
:10206000556680EB0E94BA5F81111CC00E941E6001
:1020700080911D2090911E20816090931E2080935E
:102080001D208DE993E09F938F938EE69EE09F93B2
:102090008F930E94BE920F900F900F900F90C1E00F
:1020A000D0E002C0C0E0D0E0FEB08F2D8470F82EEA
:1020B000729A0E9455668EE40E94BA5F811116C022
:1020C0000E941E6080911D2090911E20826090933E
:1020D0001E2080931D208E010F5F1F4F43E259E0A9
:1020E00065EA73E0CE010E940210E801F11001C020
:1020F00072980E9455668EEE0E94BA5F811116C0DA
:102100000E941E6080911D2090911E2084609093FB
:102110001E2080931D208E010F5F1F4F43E259E068
:102120006DEA73E0CE010E940210E8010E9455663C
:1021300086EA0E94BA5F811116C00E941E608091DB
:102140001D2090911E20886090931E2080931D205A
:102150008E010F5F1F4F43E259E064EB73E0CE0145
:102160000E940210E8010E9455668CE30E94BA5F4B
:1021700081111EC00E941E6080911D2090911E2022
:10218000806190931E2080931D208E010F5F1F4F52
:1021900043E259E06CEB73E0CE010E94021086E648
:1021A0009EE09F938F930E94BE920F900F90E80144
:1021B0000E94556682ED0E94BA5F811116C00E948E
:1021C0001E6080911D2090911E20806290931E20A1
:1021D00080931D208E010F5F1F4F43E259E064EC96
:1021E00073E0CE010E940210E8010E94556680E86B
:1021F0000E94BA5F811116C00E941E6080911D204E
:1022000090911E20916090931E2080931D208E013E
:102210000F5F1F4F43E259E06DEC73E0CE010E9467
:102220000210E8010E94556680ED0E94BA5F81119C
:1022300016C00E941E6080911D2090911E20806813
:1022400090931E2080931D208E010F5F1F4F43E24D
:1022500059E063ED73E0CE010E940210E8010E9494
:1022600055668CEE0E94BA5F811116C00E941E60F6
:1022700080911D2090911E20926090931E2080934B
:102280001D208E010F5F1F4F43E259E06BED73E09D
:10229000CE010E940210E80107E010E00E9455669E
:1022A0008CE70E94BA5F811113C00E941E6080916A
:1022B0001D2090911E20806490931E2080931D20ED
:1022C00043E259E062EE73E0CE010E94021005C0C5
:1022D000015011090115110509F70E941E60DF91D7
:1022E000CF911F910F91FF900C94AB0BCF93DF9385
:1022F00000D0CDB7DEB74A8369830E94F55F69815C
:10230000862F0E9426604A81842F0E9426600F90AB
:102310000F90DF91CF910C941E60AF92BF92DF922D
:10232000EF92FF920F931F93CF93DF9300D01F92F2
:10233000CDB7DEB7182FD22E4A835B8369830E9404
:10234000F55F6981862F0E942660812F81600E943F
:102350001C604A81A42E5B81B52E00E010E0ED2CBC
:10236000F12C81E0E81AF1080D1580F40E151F0517
:1023700019F40E94416002C00E943760F501808319
:102380000F5F1F4FFFEFAF1ABF0AEECF0F900F90F6
:102390000F90DF91CF911F910F91FF90EF90DF9001
:1023A000BF90AF900C941E60AF92BF92CF92DF921D
:1023B000EF92FF920F931F93CF93DF93CDB7DEB7CA
:1023C00060970FB6F894DEBF0FBECDBFB82EA42E17
:1023D0006623E9F18E010F5F1F4F80E1F801119232
:1023E0008A95E9F728E0A80168E980EB0E948D1141
:1023F000BB2041F02BEE33E03F932F930E94AC9231
:102400000F900F906E01F8E0CF0ED11C52EFE52E29
:1024100053E0F52EF80181918F011F928F93FF9267
:10242000EF920E94AC920F900F900F900F900C15AE
:102430001D0581F788851F928F9327E434E03F9331
:102440002F930E94AC920F900F900F900F90AA20A4
:10245000E9F18E010F5F1F4F80E1F80111928A951B
:10246000E9F728E0A80160E880EB0E948D11BB200D
:1024700041F087EF93E09F938F930E94AC920F906F
:102480000F906E01F0E1CF0ED11C42EFE42E43E03D
:10249000F42EF80181918F011F928F93FF92EF929A
:1024A0000E94AC920F900F900F900F900C151D058D
:1024B00081F788851F928F9387E494E09F938F9391
:1024C0000E94AC920F900F900F900F9060960FB6F5
:1024D000F894DEBF0FBECDBFDF91CF911F910F915A
:1024E000FF90EF90DF90CF90BF90AF900895CF9383
:1024F000DF9300D0CDB7DEB71A82198222E0AE0199
:102500004F5F5F4F6AEA8EEE0E948D11898190E0E5
:10251000982F88272A81822B9093ED1B8093EC1BA8
:1025200022E0AE014F5F5F4F6CEA8EEE0E948D118C
:10253000898190E0982F88272A81822B9093EF1B26
:102540008093EE1B22E0AE014F5F5F4F6EEA8EEE8E
:102550000E948D11898190E0982F88272A81822BF3
:102560009093F11B8093F01B22E0AE014F5F5F4F11
:1025700060EB8EEE0E948D11898190E0982F882764
:102580002A81822B9093FF1B8093FE1B22E0AE01D9
:102590004F5F5F4F62EB8EEE0E948D11898190E05C
:1025A000982F88272A81822B9093011C8093001CEE
:1025B00022E0AE014F5F5F4F64EB8EEE0E948D1103
:1025C000898190E0982F88272A81822B9093031C81
:1025D0008093021C22E0AE014F5F5F4F66EB8EEEF0
:1025E0000E948D11898190E0982F88272A81822B63
:1025F0009093F31B8093F21B22E0AE014F5F5F4F7D
:1026000068EB8EEE0E948D11898190E0982F8827CB
:102610002A81822B9093F51B8093F41B22E0AE015C
:102620004F5F5F4F6AEB8EEE0E948D11898190E0C3
:10263000982F88272A81822B9093F91B8093F81B6F
:1026400022E0AE014F5F5F4F6CEB8EEE0E948D116A
:10265000898190E0982F88272A81822B9093FB1BF9
:102660008093FA1B22E0AE014F5F5F4F6EEB8EEE60
:102670000E948D11898190E0982F88272A81822BD2
:102680009093FD1B8093FC1B0F900F90DF91CF91D7
:1026900008952F923F924F925F926F927F928F9206
:1026A0009F92AF92BF92CF92DF92EF92FF920F93E1
:1026B0001F93CF93DF93CDB7DEB76A970FB6F89429
:1026C000DEBF0FBECDBF182F488F298F19821A8207
:1026D0001B828091101C811107C06A8F0E947712A3
:1026E00081E08093101C6A8D662309F46CC04EE271
:1026F00064EF8EEE0E94761169E07AE180E090E06E
:102700000E94985F22E0AE014F5F5F4F66EF8EEE52
:102710000E948D112981822F90E0A0E0B0E0222755
:10272000382F492F5A2F8A81282B8091021C909193
:10273000031C281B390B41095109A091001CB091C1
:10274000011C0E94DB8B6B017C018FE0F594E79408
:10275000D794C7948A95D1F76091FA1B7091FB1BAF
:10276000882777FD8095982F2BE0660F771F881FAD
:10277000991F2A95D1F72091FC1B3091FD1B44270E
:1027800037FD4095542F2C0D3D1D4E1D5F1D0E94A1
:10279000488CC20ED31ED092F71BC092F61B88E065
:1027A000C80ED11C34E0D594C7943A95E1F7EE24D5
:1027B000D7FCE094FE2CC092041CD092051CE09241
:1027C000061CF092071C012F0295000F000F007CE1
:1027D0000C5CA12FB0E0BD8BAC8BA3E0B0E0012E70
:1027E00002C0AA0FBB1F0A94E2F725E335E00E945E
:1027F000D48BDC01CB010296A11DB11D8C879D8776
:10280000AE87BF8780E593ECA0E0B0E004C0B5954B
:10281000A795979587951A95D2F7888B998BAA8B50
:10282000BB8B10E0188619861A861B86A8E02A2E14
:10283000312CAC89BD892A1A3B0A988D191709F4E5
:1028400036C1402F64EF8EEE0E9476116C857D8537
:102850008E859F850E94985F23E0AE014F5F5F4F9A
:1028600066EF8EEE0E948D11E091F61BF091F71B42
:10287000E05AFF409F01DF010E94BD8B6B017C018C
:102880008091EE1B9091EF1B9F8B8E8BA090EC1B89
:10289000B090ED1B2091F01B3091F11B0E94BD8B7D
:1028A0002B013C013DE075946794579447943A9509
:1028B000D1F7A091F21BB091F31BA70196016CE038
:1028C00055954795379527956A95D1F70E94E68BE0
:1028D000BB2797FDB095AB2F480E591E6A1E7B1E75
:1028E00092E0490E511C611C711CB2E07594679412
:1028F00057944794BA95D1F7A0E85A0E611C711C01
:10290000A091FE1BB091FF1BA30192010E94DB8BE3
:10291000DC01CB012FE0B695A795979587952A9571
:10292000D1F78C839D83AE83BF8329818A8190E018
:10293000A0E0B0E04424582E692E7A2E622A8B81C2
:10294000482A022C04C075946794579447940A94BB
:10295000D2F74501AA2497FCA094BA2C42E0880C37
:10296000991CAA1CBB1C4A95D1F7A091F41BB091ED
:10297000F51BA70196010E94E68B6B017C0157E1D4
:10298000F594E794D794C7945A95D1F72E893F8947
:10299000DF010E94BD8BEBE0959587957795679554
:1029A000EA95D1F7C60ED71EE81EF91E8C0C9D1CA9
:1029B000AE1CBF1C0C8804C0880C991CAA1CBB1C34
:1029C0000A94D2F792E0890E911CA11CB11CF2E08E
:1029D000B594A79497948794FA95D1F74818590815
:1029E0006A087B08A3019201688979898A899B8991
:1029F0000E94EE8B97FD0DC0660F771F881F991FF1
:102A00002C813D814E815F810E94268C49015A01B3
:102A10000CC02C813D814E815F810E94268C490132
:102A20005A01880C991CAA1CBB1C9927B7FC9A95C3
:102A30008B2D7A2D692D9B01AC010E94EE8B9B01A1
:102A4000AC01AEEDBBE00E94DB8B6C01FF24D7FC38
:102A5000F094EF2CA3E4B3EEA50194010E94E98B5E
:102A6000BB2797FDB095AB2FC80ED91EEA1EFB1EE3
:102A7000AFECCA0EAEE0DA1EE11CF11CA4E0F59446
:102A8000E794D794C794AA95D1F7C80CD91CEA1C2F
:102A9000FB1C88859985AA85BB858C0D9D1DAE1D67
:102AA000BF1D88879987AA87BB871F5FC6CE112362
:102AB00091F0212F30E040E050E0688579858A85EB
:102AC0009B850E94268C2093081C3093091C409300
:102AD0000A1C50930B1CA98DAA2389F16091081C34
:102AE0007091091C80910A1C90910B1C6115710555
:102AF0008105910521F10E941B8920E836EE45EC05
:102B000057E40E947C8821E03EED42E45EE30E94AF
:102B1000608B9B01AC0160E070E080E89FE30E9465
:102B2000B1872BE43AE34DEB57E30E947C88609336
:102B30000C1C70930D1C80930E1C90930F1C6A96B6
:102B40000FB6F894DEBF0FBECDBFDF91CF911F91BE
:102B50000F91FF90EF90DF90CF90BF90AF909F903C
:102B60008F907F906F905F904F903F902F9008953F
:102B70000F931F93CF93DF9300D000D000D0CDB739
:102B8000DEB78E010F5F1F4F86E0F80111928A9524
:102B9000E9F780911E1B811113C040E061E386EAD2
:102BA0000E9476114AE06CE286EA0E94761181E08A
:102BB00080931E1B6CE77EE380E090E00E94985FAC
:102BC00048E06DE286EA0E9476116CE77EE380E0E1
:102BD00090E00E94985F26E0A80162E386EA0E94E6
:102BE0008D1147E06DE286EA0E9476118A8190E0BD
:102BF000982F88272981822B9093191B8093181B6B
:102C00002C8130E0322F22274B81242B30931B1B49
:102C100020931A1B4E8150E0542F44276D81462B80
:102C200050931D1B40931C1B5F934F933F932F9317
:102C30009F938F938BEF93E09F938F930E94AC921F
:102C40000FB6F894DEBF0FBECDBF26960FB6F89430
:102C5000DEBF0FBECDBFDF91CF911F910F910895C1
:102C6000CF92DF92EF92FF920F931F93CF93DF9358
:102C7000CDB7DEB72A970FB6F894DEBF0FBECDBF33
:102C80008E010F5F1F4F86E0F80111928A95E9F7D8
:102C900041E062E08CE30E94761148E560E08CE35D
:102CA0000E94761162E174E380E090E00E94985FF8
:102CB00026E0A80163E08CE30E948D1143E062E00E
:102CC0008CE30E947611098110E0102F00278A8181
:102CD000082B1093F91A0093F81AEB80F12CFE2CB4
:102CE000EE248C81E82AF092FB1AE092FA1ACD8049
:102CF000D12CDC2CCC248E81C82AD092FD1AC09213
:102D0000FC1AB801882777FD8095982F0E941B89AF
:102D10009B01AC01B701882777FD8095982F2F8301
:102D2000388749875A870E941B892F8138854985B2
:102D30005A850E94258820EE3EE245E652E40E9434
:102D4000FD8A20E030E044E353E40E94B2879F9381
:102D50008F937F936F93DF92CF92FF92EF921F93A7
:102D60000F9389E094E09F938F930E94AC920FB6EB
:102D7000F894DEBF0FBECDBF2A960FB6F894DEBF23
:102D80000FBECDBFDF91CF911F910F91FF90EF90BC
:102D9000DF90CF900895CF93DF93EC0188819981E4
:102DA0000097F9F08338904121F01982188283E06E
:102DB00063C085ED99E00E94EA56892BE1F080918D
:102DC000C5099091C60993FD18C08091C5099091DD
:102DD000C60994FD43C08091C5099091C60995FD2F
:102DE00044C060E870E085ED99E00E94C35683E836
:102DF00090E19983888381E03FC080911D2082FF0C
:102E0000E4CF21E048E061E083E00E944913809133
:102E10000F1C8F9380910E1C8F9380910D1C8F93AC
:102E200080910C1C8F9380910B1C8F9380910A1CB6
:102E30008F938091091C8F938091081C8F9385EC50
:102E40009EE09F938F930E94BE928DB79EB70A9685
:102E50000FB6F8949EBF0FBE8DBFB7CF80911D20D7
:102E600083FFB9CF0E94B815B6CF80911D2084FF93
:102E7000B8CF0E943016B5CFDF91CF910895CF9390
:102E8000C82F8CEE0E941C608C2F0E94266065E388
:102E900075E080E090E00E94985F8DEE0E941C60DB
:102EA0000E943760C82F0E9441602C2F30E0322FE3
:102EB0002227A901482BCA01CF910895CF93DF9310
:102EC000C82F8CEE0E941C608C2F0E94266062E14D
:102ED00074E380E090E00E94985F8CEE0E941C609A
:102EE00080E00E94266065E375E080E090E00E944B
:102EF000985F8DEE0E941C600E943760C82F0E9470
:102F00003760D82F0E9441604D2F50E060E070E0A4
:102F1000762F652F542F44276C2B482BCB01BA01F9
:102F2000DF91CF9108952F923F924F925F926F92CF
:102F30007F928F929F92AF92BF92CF92DF92EF9249
:102F4000FF920F931F93CF93DF93CDB7DEB7CD548E
:102F5000D1090FB6F894DEBF0FBECDBF809100023D
:102F600090910102892BD1F110920102109200027E
:102F70008CEE0E941C608EE10E9426606BE17EE474
:102F800080E090E00E94985F82EA0E943F17909351
:102F9000D2098093D10984EA0E943F179093D00907
:102FA0008093CF0986EA0E943F179093CE098093C1
:102FB000CD0988EA0E943F179093CC098093CB09F2
:102FC0008AEA0E943F179093CA098093C9098CEA44
:102FD0000E943F179093C8098093C70988E40E9414
:102FE0005E176FAB78AF89AF9AAF88E50E945E1726
:102FF0004B015C018091C9099091CA0920E030E041
:1030000040E050E0BA0126962FAF269727963FAFB3
:10301000279728964FAF289729965FAF29972A962A
:103020006FAF2A972B967FAF2B979C0140E050E023
:1030300060E070E080E090E008E00E94CF8D0E94A8
:103040007B8D3901B42FA52FF62FE72F8C0194012A
:10305000A50160E070E080E090E05301CB2EDA2E15
:10306000EF2EFE2E0E94068E29833A832A011B0131
:103070004C01B101C401315041095F4F6F4F7F4F87
:103080008F4F9F4FA1E0B0E02596BFAFAEAF259721
:1030900021153F4F4F4F5140610571058105910545
:1030A00009F020F425961FAE1EAE259725966EAC2E
:1030B0007FAC25978091C7099091C8095C01C12C0C
:1030C000D12CE12CF12C00E010E029813A81A20101
:1030D000B101C4010E949E8CD22EE32EF42E052F46
:1030E000162FB72FF82FE92FA0E00E942D8E84F421
:1030F0002150310940485F4F6F4F7F4F8F4F9F4F97
:10310000D22EE32EF42E052F162FB72FF82FE92FEE
:103110002D2D3E2D4F2D502F612F7B2F8F2F9E2F2A
:1031200007E10E94E88D2B8F3C8F4D8F5E8F6F8F54
:1031300078A389A39AA32053384F4F4F5F4F6F4F07
:103140007F4F8F4F9F4F2B8B3C8B4D8B5E8B6F8BAD
:10315000788F898F9A8F2056304F4F4F5F4F6F4F28
:103160007F4F8F4F9F4F243D3043410551056105EF
:1031700071058105910541F038F025966EAC7FAC64
:103180002597FFEF6F1A7F0A8091CF099091D009A0
:103190009C0140E050E060E070E080E090E000E101
:1031A0000E94CF8D2B833C834D835E836A87798712
:1031B0008F8398874091CB095091CC09A980BA8020
:1031C0006201710184019A0140E050E060E070E02A
:1031D00080E090E00E949E8CD22EE32EF42E052FEC
:1031E000162FB72FF82FE92FA0E00E942D8E5CF448
:1031F000AFE70E940F8ED22EE32EF42E052F162F4E
:10320000B72FF82FE92F2D2D3E2D4F2D502F612F49
:103210007B2F8F2F9E2F07E00E94E88D59016A01B6
:103220007B018C012B813C814D815E816A85798592
:103230008F8198850E94068E2B833C834D835E830D
:103240006F8378878F87988B2E5F3F4F434051095C
:103250006E4F7F4F8F4F9F4F22303105494F5F4F49
:10326000644071058105910521F018F01FEF611A86
:10327000710A8091D1099091D209BC0180E090E05F
:1032800020E030E840E050E00E94F78C29873A8740
:103290004B875C876A8B798B8D879E874091CD09A0
:1032A0005091CE09A980BA806201710184019A010E
:1032B00040E050E060E070E080E090E00E949E8C92
:1032C000D22EE32EF42E052F162FB72FF82FE92F2D
:1032D000A0E00E942D8E84F421503F4F4F4F5F4F4E
:1032E0006F4F7F4F8F4F9F4FD22EE32EF42E052F1F
:1032F000162FB72FF82FE92F2D2D3E2D4F2D502FA4
:10330000612F7B2F8F2F9E2F08E00E94E88D59019F
:103310006A017B018C0129853A854B855C856A8928
:1033200079898D859E850E94068E29873A874B87ED
:103330005C876D877E87898B9A8B2F5F3F4F4140DB
:1033400051096109710981099109213030484C4FB7
:103350005F47614071058105910521F018F0BFEFCD
:103360006B1A7B0A2B893C894D895E896F89788D20
:10337000898D9A8D2F3C37404105510561057105B6
:103380008105910511F00CF0A5C1A980BA806201F8
:10339000710184019501A201B101C4010E949E8CBA
:1033A000A12CB12CC12C10E8D12EE12CF12C00E085
:1033B00010E00E94618C2BAF3CAF4DAF5EAF6FAFA2
:1033C00021967FAF219722968FAF229723969FAFAA
:1033D0002397AB8CBC8CCD8CDE8CEF8CF8A009A134
:1033E0001AA19501A601B701C8010E949E8C59013E
:1033F0006A017B01E82F192F02E00E94CF8D0E2F6A
:103400000E94068E69017A01162F272EF82FE92FC8
:10341000322E8D2C942EAF2CB62E072F582EB92F6E
:10342000A0E00E942D8E5CF4A1E00E940F8E322E4F
:10343000832E942EA52EB62E072F582EB92F232D6E
:10344000382D492D5A2D6B2D702F852D9B2F01E086
:103450000E94E88D2E962FAF2E972D963FAF2D9779
:1034600049A75AA76BA77CA78DA79EA7522E432ECC
:103470004BA35CA36DA37EA38FA398A7B22D960147
:10348000A701612F722D8F2F9E2FA0E00E942D8EFD
:103490004CF4A3E00E940F8E69017A01162FB72F1A
:1034A000F82FE92F9601A701612F7B2F8F2F9E2FD9
:1034B00002E00E94E88D2FA738AB49AB5AAB6BAB4B
:1034C0007CAB8DAB9EAB19014A01B62FA72F24967A
:1034D0008FAF2497F92F2B893C894D895E896F899D
:1034E000788D898D9A8D24323A4F4F4F5F4F6F4FB1
:1034F0007F4F8F4F9F4F0CF08CC02B8D3C8D4D8D8F
:103500005E8D6F8D78A189A19AA12455324F4F4FBE
:103510005F4F6F4F7F4F8F4F9F4F59016A017B0164
:103520008C010E949E8C19014A01B62FA72FFC0125
:1035300003E00E94CF8D51016401EB2EFA2E8F0122
:103540000E941B8E59016A017B018C012E962FADC2
:103550002E972D963FAD2D9749A55AA56BA57CA515
:103560008DA59EA50E94068E522E432E4BA35CA3D2
:103570006DA37EA38FA398A79101A4016B2F7A2F2F
:10358000CF0102E00E94CF8D51016401EB2EFA2E93
:103590008F010E941B8E02E00E94CF8D0E2F0E9491
:1035A0001B8EF22E032F142FD52EE62EB72FF82FB9
:1035B000E92FA0E00E942D8E5CF4A1E00E940F8E06
:1035C000F22E032F142FD52EE62EB72FF82FE92F2A
:1035D0002F2D302F412F5D2D6E2D7B2F8F2F9E2F66
:1035E00001E00E94E88D59016A017B018C012FA541
:1035F00038A949A95AA96BA97CA98DA99EA90E949D
:10360000068E19014A01B62FA72F24968FAF249753
:10361000F92F2B813C814D815E816F8178858F856B
:103620009889A52CB42CCBA0DCA0EDA0FEA00FA106
:1036300018A50E941B8E2B833C834D835E836F8372
:1036400078878F87988B29853A854B855C856D8532
:103650007E8589899A8951016401EB2EFA2E249680
:103660000FAD24971F2F0E941B8E29873A874B8707
:103670005C876D877E87898B9A8B2B893C894D89E6
:103680005E896F89788D898D9A8DABACBCACCDACE1
:10369000DEACEFAC2196FFAC219722960FAD2297BE
:1036A00023961FAD23970E941B8E2056304F4F4FFD
:1036B0005F4F6F4F7F4F8F4F9F4F243D30434105EA
:1036C0005105610571058105910521F018F02FEF75
:1036D000621A720A6FA978AD89AD9AADAB01BC01CF
:1036E00080E090E0DC0124964FAF249725965FAFF1
:1036F000259726966FAF269727967FAF2797289610
:103700008FAF289729969FAF29972A96AFAF2A9710
:103710002B96BFAF2B97A984BA84CB84DC84ED842D
:10372000FE8409891A899A01AB0160E070E080E0AB
:1037300090E00E949E8CF22E032F142FD52EE62EA1
:10374000B72FF82FE92FA0E00E942D8E84F421508E
:103750003109404E5F4F6F4F7F4F8F4F9F4FF22E7B
:10376000032F142FD52EE62EB72FF82FE92F2F2D4C
:10377000302F412F5D2D6E2D7B2F8F2F9E2F05E13A
:103780000E94E88DAB80BC80CD80DE80EF80F88425
:103790000F8518890E941B8EF22E032F142FD52E11
:1037A000E62EB72FF82FE92FA0E00E942D8E84F48B
:1037B000215030484F4F5F4F6F4F7F4F8F4F9F4F7C
:1037C000F22E032F142FD52EE62EB72FF82FE92F28
:1037D0002F2D302F412F5D2D6E2D7B2F8F2F9E2F64
:1037E0000FE00E94E88D69017A018B018A83998339
:1037F00029011A014B015C01285E3340410951093E
:103800006109710981099109283D304D41405105F7
:10381000610571058105910521F018F0BFEF6B1A64
:103820007B0A0E941E60672859F09601A701B80123
:103830008A8199810E947B8D29011A014B015C01CB
:103840009201A101B401C5010E94158920E030E078
:1038500048EC52E40E947C88C35BDF4F0FB6F894BB
:10386000DEBF0FBECDBFDF91CF911F910F91FF90B3
:10387000EF90DF90CF90BF90AF909F908F907F9010
:103880006F905F904F903F902F9008954F925F926E
:103890006F927F928F929F92AF92BF92CF92DF9260
:1038A000EF92FF922B013C0169017A0123EC35EF85
:1038B0004CE851E4C701B6010E94FD8A4B015C014E
:1038C00028EB3EE143E753E4C701B6010E94B2870B
:1038D0009B01AC01C501B4010E947C880E94E9886B
:1038E0004B015C0120E030E048EC52E4C301B2013E
:1038F0000E947C8821E835E943EC50E40E94FD8A6F
:10390000A50194010E94FD8A4B015C0123E333E988
:1039100048E853E4C701B6010E94B2879B01AC019D
:10392000C501B4010E947C8823E333EB48E553E4EE
:103930000E94FD8AFF90EF90DF90CF90BF90AF90F4
:103940009F908F907F906F905F904F9008954F92CF
:103950005F926F927F928F929F92AF92BF92CF921F
:10396000DF92EF92FF9269017A010E947F8A20E044
:1039700030E040E050E40E94B18722E93CE54EEDA2
:103980005EE30E947C884B015C0123EC35EF4CE840
:1039900051E4C701B6010E94FD8A2B013C0128EBCE
:1039A0003EE143E753E4C701B6010E94B2879B01A1
:1039B000AC01C301B2010E947C889B01AC01C5012E
:1039C000B4010E94B2876B017C0128EB3EE143E722
:1039D00053E40E94FD8A4B015C01A701960163EC50
:1039E00075EF8CE891E40E94B1879B01AC01C501A1
:1039F000B4010E947C88FF90EF90DF90CF90BF9041
:103A0000AF909F908F907F906F905F904F900895B0
:103A10004F925F926F927F928F929F92AF92BF92DE
:103A2000CF92DF92EF92FF922B013C0169017A0164
:103A300023EC35EF4CE851E4C701B6010E94FD8A42
:103A40004B015C0128EB3EE143E753E4C701B601BB
:103A50000E94B2879B01AC01C501B4010E947C8821
:103A60000E94E9884B015C0120E030E048EC52E420
:103A7000C301B2010E947C88A50194010E94FD8AC5
:103A800020E030E040E251E40E94B18724EE38E3C8
:103A90004EE05FE30E94FD8A9B01AC01C701B601C5
:103AA0000E94B287FF90EF90DF90CF90BF90AF90D1
:103AB0009F908F907F906F905F904F90089580E8D7
:103AC0000E941C6081110DC08EEF0E942660811142
:103AD00008C06BE17EE480E090E00E94985F0C9467
:103AE0001E600E941E6080912F2490913024A0912E
:103AF0003124B09132240196A11DB11D80932F2451
:103B000090933024A0933124B09332240895FC0183
:103B1000DC0182E020E041E39D91292798E0322FEB
:103B2000330F27FF03C0232F242701C0232F9150D9
:103B3000B1F7815089F781E090E03281231711F0CD
:103B400080E090E00895DF92EF92FF920F931F9331
:103B5000CF93DF930E945F1D80E80E941C6081115B
:103B60006DC08AEF0E942660811168C08FE00E94BC
:103B70002660811163C065E375E080E090E00E94FB
:103B8000985F81E80E941C60811158C00E943760D4
:103B9000C82F0E9437600E943760D82F0E9437607C
:103BA0000E943760182F0E9437600E944160082FE2
:103BB00080E80E941C60811141C08CEF0E94266049
:103BC00081113CC089EC0E942660811137C065E3F9
:103BD00075E080E090E00E94985F81E80E941C60A0
:103BE0000E943760E82E0E943760D82E0E9437600E
:103BF0000E943760F82E0E9441601F92DF921F9250
:103C0000EF921F920F931F921F931F92DF931F92A9
:103C1000CF931F928F931F92FF928EE194E09F9318
:103C20008F930E94AC920E941E608DB79EB7429601
:103C30000FB6F8949EBF0FBE8DBF17C00E941E60C6
:103C400080912F2490913024A0913124B09132247E
:103C50000196A11DB11D80932F2490933024A09331
:103C60003124B09332240E945F1D20E030E040E018
:103C700050E060E070E080E090E0DF91CF911F9134
:103C80000F91FF90EF90DF900895EF92FF920F93C6
:103C90001F93CF93DF9300D01F92CDB7DEB78C0177
:103CA00080E80E941C60811154C00115110551F07B
:103CB00085EE0E94266081114CC061E077E980E0CA
:103CC00090E009C083EE0E942660811142C069E93C
:103CD0007AEB81E090E00E94985F81E80E941C608E
:103CE000811137C00E943760F82E89830E943760A7
:103CF000E82E8A830E9441608B830E941E60CE0161
:103D000001960E94871D892B21F16E2D70E07F297D
:103D10006C7F80E090E0012B69F00E94198920E01F
:103D200030E04AEF5AE30E94FD8A20E030E040ECA8
:103D300050E40CC00E94198922E538EB4FE25BE3A6
:103D40000E94FD8A26E636E64BE352E40E94B187E4
:103D50001BC00E941E6080912F2490913024A0915E
:103D60003124B09132240196A11DB11D80932F24DE
:103D700090933024A0933124B09332240E945F1D8D
:103D800060EF7FEF89E794E40F900F900F90DF9141
:103D9000CF911F910F91FF90EF9008950F931F9374
:103DA000CF93DF93729A8091580283FF08C08EE40C
:103DB0000E94BA5F811167C0C0E5D0E00AC0C0E5CB
:103DC000D0E087EE93E00E94450921972097C9F73C
:103DD000EECF87EE93E00E94450921972097C9F71F
:103DE0008FE40E94BA5F0E943760082F0F730E9411
:103DF0003760182F0E943760D82F0E944160C82F6B
:103E00000E941E608091580283FF7298602F70E0BC
:103E1000762F6627610F711D80E090E00E9419895E
:103E200020E134E048EC5BE30E94FD8A6093111CC2
:103E30007093121C8093131C9093141C6D2F70E0D0
:103E4000762F66276C0F711D769567957695679529
:103E500080E090E00E94198924EA3CEF44E25CE3B0
:103E60000E94FD8A20E030E040E252E40E94B187E7
:103E70006093AE287093AF288093B0289093B128B8
:103E800080E090E002C081E090E0DF91CF911F914F
:103E90000F9108957298729A8EE40E94BA5F80EA38
:103EA0000E94266080E00E94266080E00E942660DA
:103EB0008FE40E94BA5F0E9437608EE40E94BA5F6E
:103EC00080E80E94266080E00E94266080E00E94D8
:103ED00026600E941E6080E090E0089589E59EE0E3
:103EE0009F938F930E94BE92809173020F900F90C8
:103EF000882361F01F928F9386E59EE09F938F93B6
:103F00000E94BE920F900F900F900F90089581E342
:103F10009EE09F938F930E94BE9289E09EE09F93C4
:103F20008F930E94BE9282EE9DE09F938F930E949A
:103F3000BE9287EA9DE09F938F930E94BE9285E791
:103F40009DE09F938F930E94BE9289E39DE09F9393
:103F50008F930E94BE9283E19DE09F938F930E9476
:103F6000BE928DED9CE09F938F930E94BE928091B4
:103F70001D2090911E20827091702DB73EB7205F5A
:103F80003F4F0FB6F8943EBF0FBE2DBF892B41F0B7
:103F90008DEA9CE09F938F930E94BE920F900F90AA
:103FA00081E89CE09F938F930E94BE9285E49CE001
:103FB0009F938F930E94BE928CE19CE09F938F937E
:103FC0000E94BE9280EF9BE09F938F930E94BE92CF
:103FD00081EC9BE09F938F930E94BE928FE89BE0C1
:103FE0009F938F930E94BE928EE59BE09F938F9349
:103FF0000E94BE9284E29BE09F938F930E94BE92A8
:104000008EEE9AE09F938F930E94BE928EEB9AE081
:104010009F938F930E94BE9282E99AE09F938F9321
:104020000E94BE9283E69AE09F938F930E94BE9275
:104030008AE29AE09F938F930E94BE9281EF99E06B
:104040009F938F930E94BE928AEB99E09F938F93E8
:104050000E94BE9289E899E09F938F930E94BE923E
:104060008DB79EB780960FB6F8949EBF0FBE8DBFDA
:104070008AE599E09F938F930E94BE928BE299E02C
:104080009F938F930E94BE9284E099E09F938F93B9
:104090000E94BE928EEC98E09F938F930E94BE92F6
:1040A00088E998E09F938F930E94BE9282E698E001
:1040B0009F938F930E94BE9289E398E09F938F9382
:1040C0000E94BE9281E098E09F938F930E94BE92DF
:1040D00086ED97E09F938F930E94BE922DB73EB7D7
:1040E0002E5E3F4F0FB6F8943EBF0FBE2DBF089512
:1040F0008DE494E00C94E2924F925F926F927F92E3
:104100008F929F92AF92BF92CF92DF92EF92FF92E7
:10411000CF93DF93CDB7DEB728970FB6F894DEBF05
:104120000FBECDBF8091232490912424A0912524FB
:10413000B091262489839A83AB83BC834090232447
:10414000509024246090252470902624809123246C
:1041500090912424A0912524B09126248D839E83C0
:10416000AF83B88760912324709124248091252403
:10417000909126242CE3822E912CA12CB12CA50108
:1041800094010E94268C7F936F9330E1C32E3EE012
:10419000D32EE12CF12C6D817E818F819885A70132
:1041A00096010E94268CA50194010E94268C3F93C3
:1041B0002F9340E8842E41E5942EAA24A394B12C99
:1041C000C301B201A50194010E94268CA7019601AA
:1041D0000E94268C3F932F9369817A818B819C81E9
:1041E000A50194010E94268C3F932F9380EB97E0CA
:1041F0009F938F930E94BE920FB6F894DEBF0FBEBE
:10420000CDBF28960FB6F894DEBF0FBECDBFDF91AD
:10421000CF91FF90EF90DF90CF90BF90AF909F90A5
:104220008F907F906F905F904F900895E3E7F1E358
:10423000808191818234924479F0E357F143FF9376
:10424000EF9382E997E09F938F930E94BE920F9025
:104250000F900F900F9008953A96E53F81E4F8078C
:1042600038F30895CF93DF93EC018C9A0E94900A63
:104270009F938F937F936F9386E897E09F938F939D
:104280000E94BE920F900F900F900F900F900F9082
:10429000209719F00E94AB0B08C084E897E09F9329
:1042A0008F930E94BE920F900F9081E00E94410A6E
:1042B000209178023091790240917A0250917B02EC
:1042C0000E94FD8A9F938F937F936F9388E797E077
:1042D0009F938F930E94BE920F900F900F900F901C
:1042E0000F900F90209719F00E94AB0B08C086E743
:1042F00097E09F938F930E94BE920F900F9082E061
:104300000E94410A20917402309175024091760218
:10431000509177020E94FD8A9F938F937F936F93B2
:104320008AE697E09F938F930E94BE920F900F9022
:104330000F900F900F900F90209719F00E94AB0BE9
:1043400008C088E697E09F938F930E94BE920F90DB
:104350000F9083E00E94410A9F938F937F936F9306
:1043600089E597E09F938F930E94BE928C980F905F
:104370000F900F900F900F900F90209719F00E94C0
:10438000AB0B08C087E597E09F938F930E94BE9286
:104390000F900F9080911D2087FF83C021E042E1A4
:1043A00061E080ED0E947E619F938F937F936F9376
:1043B0008AE497E09F938F930E94BE920F900F9094
:1043C0000F900F900F900F90209719F00E94AB0B59
:1043D00008C088E497E09F938F930E94BE920F904D
:1043E0000F9021E042E162E080ED0E947E619F93A8
:1043F0008F937F936F938BE397E09F938F930E94AC
:10440000BE920F900F900F900F900F900F902097EB
:1044100019F00E94AB0B08C089E397E09F938F933C
:104420000E94BE920F900F9021E042E163E080ED88
:104430000E947E619F938F937F936F938CE297E0AE
:104440009F938F930E94BE920F900F900F900F90AA
:104450000F900F90CD2B19F00E94AB0B08C08AE291
:1044600097E09F938F930E94BE920F900F9021E050
:1044700042E164E080ED0E947E619F938F937F9381
:104480006F938DE197E09F938F930E94BE920F9060
:104490000F900F900F900F900F90DF91CF910C9491
:1044A000AB0BCD2BD1F3DF91CF9108950F931F93D9
:1044B000CF93DF93882389F049E050E06FEF70E0FD
:1044C00082EA98E20E94009249E050E06AE070E0DF
:1044D00082EA98E20E94309413C0C2EAD8E208E16E
:1044E00017E089911F928F931F930F930E94BE92A2
:1044F0000F900F900F900F9088E2CA3AD80789F773
:10450000DF91CF911F910F910C94AB0BCF92DF9263
:10451000EF92FF92CF93DF936B017C0160FF11C09C
:104520008AE894E09F938F938EE69EE09F938F930B
:104530000E94BE920F900F900F900F9081E090E03C
:1045400002C080E090E0C1FE09C0EC01219643E288
:1045500059E06FE874E00E940210CE01C2FE09C06B
:10456000EC01219643E259E067E974E00E940210F1
:10457000CE01C3FE09C0EC01219643E259E06FE988
:1045800074E00E940210CE01C4FE09C0EC01219625
:1045900043E259E063EA74E00E940210CE01C5FED6
:1045A00009C0EC01219643E259E066EA74E00E94FA
:1045B0000210CE01C6FE09C0EC01219643E259E08B
:1045C0006AEA74E00E940210CE01C7FE09C0EC0145
:1045D000219643E259E060EB74E00E940210CE01A4
:1045E000D0FE09C0EC01219643E259E068EB74E08B
:1045F0000E940210CE01D1FE09C0EC01219643E2D7
:1046000059E060EC74E00E940210CE01D2FE09C0B5
:10461000EC01219643E259E064EC74E00E94021040
:10462000CE0120911D2030911E2024703270232B4A
:1046300059F0D3FE09C0EC01219643E259E06AEC3F
:1046400074E00E940210CE0120911D2023FF0BC0B8
:10465000D4FE09C0EC01219643E259E06FEC74E00E
:104660000E940210CE0120911D2024FF0BC0D5FE18
:1046700009C0EC01219643E259E065ED74E00E9427
:104680000210CE01D6FE09C0EC01219643E259E0AA
:104690006DED74E00E940210CE01B701A60144271F
:1046A0005078452B462B472B61F043E259E068EEEA
:1046B00074E0DF91CF91FF90EF90DF90CF900C945A
:1046C0000210CD28CE28CF2841F483E197E09F93B4
:1046D0008F930E94BE920F900F90DF91CF91FF9029
:1046E000EF90DF90CF9008950F931F93CF93DF93B8
:1046F0008C01C0E0D0E00115110509F48AC06EE01C
:1047000077E0C8010E94DF91892B09F4C16066E05F
:1047100077E0C8010E94DF91892B09F4C2606EEF37
:1047200076E0C8010E94DF91892B09F4C4606AEF2A
:1047300076E0C8010E94DF91892B09F4C86067EF19
:1047400076E0C8010E94DF91892B09F4C06163EF14
:1047500076E0C8010E94DF91892B09F4C0626DEEFA
:1047600076E0C8010E94DF91892B09F4C06465EEF0
:1047700076E0C8010E94DF91892B09F4C0686DEDD5
:1047800076E0C8010E94DF91892B09F4D16069EDC0
:1047900076E0C8010E94DF91892B09F4D26063EDB5
:1047A00076E0C8010E94DF91892B09F4D4606EEC99
:1047B00076E0C8010E94DF91892B09F4D86068EC8B
:1047C00076E0C8010E94DF91892B09F4D06160EC8A
:1047D00076E0C8010E94DF91892B09F4D06265EB75
:1047E00076E0C8010E94DF91892B09F4D06464EA65
:1047F00076E0C8010E94DF91892B09F4D0686091AE
:1048000071027091720280E090E00E94F3918C013D
:1048100072CFCE01DF91CF911F910F910895AF928A
:10482000BF92CF92DF92EF92FF920F931F93CF939D
:10483000DF93F22E032F142FE52ED62EA72EB82E9F
:10484000C92E217030E040E050E060E070E080E090
:1048500090E0A0E00E942D8E89F0E9EFF4E0FF9354
:10486000EF93EEE6FEE0FF93EF930E94BE920F906F
:104870000F900F900F90E1E0F0E002C0E0E0F0E078
:1048800080911D2080FF17C02F2D247030E040E064
:1048900050E060E070E080E090E0A0E00E942D8EAB
:1048A00051F0EF01219643E259E06DEF74E0CF0142
:1048B0000E940210FE012F2D227030E040E050E0F7
:1048C00060E070E080E090E0A0E00E942D8E51F06A
:1048D000EF01219643E259E061E075E0CF010E94CB
:1048E0000210FE012F2D287030E040E050E060E023
:1048F00070E080E090E0A0E00E942D8E51F0EF018A
:10490000219643E259E069E175E0CF010E9402106F
:10491000FE012F2D207130E040E050E060E070E0BB
:1049200080E090E0A0E00E942D8E51F0EF012196F2
:1049300043E259E064E075E0CF010E940210FE01FD
:104940002F2D207230E040E050E060E070E080E029
:1049500090E0A0E00E942D8E51F0EF01219643E2FD
:1049600059E067E075E0CF010E940210FE012F2D93
:10497000207430E040E050E060E070E080E090E0E3
:10498000A0E00E942D8E51F0EF01219643E259E004
:104990006DE075E0CF010E940210FE012F2D2078FE
:1049A00030E040E050E060E070E080E090E0A0E0C7
:1049B0000E942D8E51F0EF01219643E259E063E110
:1049C00075E0CF010E940210FE0120E0302F31700F
:1049D00040E050E060E070E080E090E0A0E00E9405
:1049E0002D8E51F0EF01219643E259E066E175E02A
:1049F000CF010E940210FE0120E0302F327040E013
:104A000050E060E070E080E090E0A0E00E942D8E39
:104A100051F0EF01219643E259E06BE175E0CF01DF
:104A20000E940210FE0120E0302F347040E050E080
:104A300060E070E080E090E0A0E00E942D8E51F0F8
:104A4000EF01219643E259E062E275E0CF010E9456
:104A50000210FE0120E0302F387040E050E060E0AE
:104A600070E080E090E0A0E00E942D8E51F0EF0118
:104A7000219643E259E065E275E0CF010E94021001
:104A8000FE0120E0302F307140E050E060E070E047
:104A900080E090E0A0E00E942D8E51F0EF01219681
:104AA00043E259E06AE275E0CF010E940210FE0184
:104AB00020E0302F307240E050E060E070E080E0B5
:104AC00090E0A0E00E942D8E51F0EF01219643E28C
:104AD00059E061E375E0CF010E940210FE0120E081
:104AE00030E040E050E06D2D647070E080E090E0D8
:104AF000A0E00E942D8E51F0EF01219643E259E093
:104B000068E375E0CF010E940210FE0180911D2034
:104B100081FF17C020E0302F307440E050E060E0AB
:104B200070E080E090E0A0E00E942D8E51F0EF0157
:104B3000219643E259E06CE375E0CF010E94021038
:104B4000FE0180911D2090911E2090FF17C020E053
:104B500030E040E05E2D507160E070E080E090E079
:104B6000A0E00E942D8E51F0EF01219643E259E022
:104B70006FE375E0CF010E940210FE0180911D20BD
:104B800090911E2090FF17C020E030E040E05E2DA5
:104B9000507260E070E080E090E0A0E00E942D8E16
:104BA00051F0EF01219643E259E062E475E0CF0154
:104BB0000E940210FE0180911D2090911E2090FF06
:104BC00017C020E030E040E05E2D507460E070E0FF
:104BD00080E090E0A0E00E942D8E51F0EF01219640
:104BE00043E259E068E475E0CF010E940210FE0143
:104BF00020E0302F307840E050E060E070E080E06E
:104C000090E0A0E00E942D8E51F0EF01219643E24A
:104C100059E063E575E0CF010E940210FE0120E03B
:104C200030E0412F417050E060E070E080E090E0C3
:104C3000A0E00E942D8E51F0EF01219643E259E051
:104C400068E575E0CF010E940210FE0120E030E02F
:104C5000412F427050E060E070E080E090E0A0E022
:104C60000E942D8E51F0EF01219643E259E06BE551
:104C700075E0CF010E940210FE0120E030E0412FDC
:104C8000447050E060E070E080E090E0A0E00E94BE
:104C90002D8E51F0EF01219643E259E06EE575E06B
:104CA000CF010E940210FE0180911D2087FF17C0D6
:104CB00020E030E0412F487050E060E070E080E09C
:104CC00090E0A0E00E942D8E51F0EF01219643E28A
:104CD00059E061E675E0CF010E940210FE0180916B
:104CE0001D2087FF17C020E030E0412F407150E0C9
:104CF00060E070E080E090E0A0E00E942D8E51F036
:104D0000EF01219643E259E065E675E0CF010E948C
:104D10000210FE0180911D2087FF17C020E030E0C7
:104D2000412F407250E060E070E080E090E0A0E051
:104D30000E942D8E51F0EF01219643E259E069E681
:104D400075E0CF010E940210FE0180911D2087FFB7
:104D500017C020E030E0412F407450E060E070E088
:104D600080E090E0A0E00E942D8E51F0EF012196AE
:104D700043E259E06DE675E0CF010E940210FE01AA
:104D800080911D2082FF17C020E030E0412F407845
:104D900050E060E070E080E090E0A0E00E942D8EA6
:104DA00051F0EF01219643E259E06DE376E0CF0147
:104DB0000E940210FE0180911D2082FF17C020E09A
:104DC00030E040E05E2D517060E070E080E090E007
:104DD000A0E00E942D8E51F0EF01219643E259E0B0
:104DE00061E775E0CF010E940210FE0180911D2055
:104DF00090911E2090FF17C020E030E040E05E2D33
:104E0000527060E070E080E090E0A0E00E942D8EA3
:104E100051F0EF01219643E259E064E775E0CF01DC
:104E20000E940210FE0180911D2090911E2090FF93
:104E300017C020E030E040E05E2D547060E070E08C
:104E400080E090E0A0E00E942D8E51F0EF012196CD
:104E500043E259E06CE775E0CF010E940210FE01C9
:104E600080911D2090911E2091FF1EC020E030E017
:104E700040E05E2D587060E070E080E090E0A0E0DF
:104E80000E942D8E89F043E259E065E875E0CF017C
:104E9000DF91CF911F910F91FF90EF90DF90CF9016
:104EA000BF90AF900C9402102F2D302F412F5E2D0C
:104EB0006D2D7A2D8B2D9C2DA0E00E942D8E41F41E
:104EC0008FE996E09F938F930E94BE920F900F9070
:104ED000DF91CF911F910F91FF90EF90DF90CF90D6
:104EE000BF90AF9008958F929F92BF92DF92EF9202
:104EF0000F931F93CF93DF93EC014B01FB011082C3
:104F00006AE976E00E94DF91892B61F580911D208E
:104F10007DE4D72EE0E8EE2E82FD02C004E001C061
:104F200004E810E0B12C81FF02C060ECE62E26E020
:104F30004AE250E06BE270E089E290E00E94BF5CE0
:104F400081E090E00E94390B882311F05DE5D52EB9
:104F500080911D2090911E2090FD16E091FF07C0CA
:104F6000186005C0D12CE12C00E010E0B12C68E9FC
:104F700076E0CE010E94DF91892B61F481E0F4019B
:104F80008083609171027091720280E090E00E94D3
:104F9000F391EC0166E976E0CE010E94DF91892B66
:104FA00061F48FEFF401808360917102709172025D
:104FB00080E090E00E94F391EC01209709F424C175
:104FC00062E976E0CE010E94DF91892B19F4FD2D74
:104FD000F160DF2E6EE876E0CE010E94DF91892B32
:104FE00019F48D2D8460D82E6BE876E0CE010E94F6
:104FF000DF91892B19F4ED2DE260DE2E69E876E071
:10500000CE010E94DF91892B19F4FD2DF860DF2E6F
:1050100066E876E0CE010E94DF91892B19F48D2D90
:105020008061D82E60E876E0CE010E94DF91892B66
:1050300019F4ED2DE062DE2E6AE776E0CE010E94E3
:10504000DF91892B19F4FD2DF064DF2E67E776E000
:10505000CE010E94DF91892B19F48D2D8068D82E06
:1050600062E776E0CE010E94DF91892B19F4EE2DE4
:10507000E160EE2E6BE676E0CE010E94DF91892B97
:1050800019F4FE2DF260EF2E68E676E0CE010E9464
:10509000DF91892B19F48E2D8460E82E63E676E08B
:1050A000CE010E94DF91892B19F4EE2DE860EE2EDF
:1050B0006CE576E0CE010E94DF91892B19F4FE2D7C
:1050C000F061EF2E65E576E0CE010E94DF91892B3D
:1050D00019F48E2D8062E82E61E576E0CE010E9403
:1050E000DF91892B19F4EB2DE460BE2E6EE476E09F
:1050F000CE010E94DF91892B19F4FE2DF064EF2E72
:1051000069E476E0CE010E94DF91892B19F48E2D9F
:105110008068E82E66E476E0CE010E94DF91892B5C
:1051200009F4016063E476E0CE010E94DF91892BEF
:1051300009F4026060E476E0CE010E94DF91892BE1
:1051400009F404606CE376E0CE010E94DF91892BC4
:1051500009F4086068E376E0CE010E94DF91892BB4
:1051600009F4006164E376E0CE010E94DF91892BAF
:1051700009F4006260E376E0CE010E94DF91892BA2
:1051800009F400646EE276E0CE010E94DF91892B83
:1051900009F400686BE276E0CE010E94DF91892B72
:1051A00009F4116063E276E0CE010E94DF91892B61
:1051B00009F412606AE176E0CE010E94DF91892B4A
:1051C00009F4146061E176E0CE010E94DF91892B41
:1051D00009F418606EE076E0CE010E94DF91892B21
:1051E00009F4106168E076E0CE010E94DF91892B1E
:1051F00009F410626DEF75E0CE010E94DF91892BFA
:1052000009F0D2CE1064D0CE2D2D3E2DA8016B2DED
:1052100070E080E090E0DF91CF911F910F91EF90CF
:10522000DF90BF909F908F9008955F926F927F92D2
:105230008F929F92AF92BF92CF92DF92EF92FF92A6
:105240000F931F93CF93DF93782EC7E2DBE100E04B
:1052500010E0F7EFEF2EF5E0FF2E8170582E872D2E
:105260008270682EA2EECA2EA5E0DA2EBAEEAB2E20
:10527000B5E0BB2E88EE882E85E0982E772051F081
:105280001F930F93FF92EF920E94BE920F900F9088
:105290000F900F905520A1F089858F9388858F936B
:1052A000BF92AF920E94BE920F900F900F900F90FE
:1052B0006620C1F09F928F920E94BE920F900F9035
:1052C000662081F0DF92CF920E94BE9228813981C0
:1052D0004A815B816C817D818E819F810E940F2438
:1052E0000F900F900E94AB0B0F5F1F4F2A96043058
:1052F000110521F6DF91CF911F910F91FF90EF9053
:10530000DF90CF90BF90AF909F908F907F906F90E5
:105310005F90089582ED95E09F938F930E94BE92D7
:105320000E9478208EE09BE19F938F938AEC95E01A
:105330009F938F930E94BE9260915202709153028C
:10534000809154029091550228EE33E040E050E005
:105350000E94268C5F934F933F932F938AEB95E0A7
:105360009F938F930E94BE9281EB95E09F938F93C2
:105370000E94BE920E942A1080911D202DB73EB738
:10538000225F3F4F0FB6F8943EBF0FBE2DBF80FF88
:1053900005C041E061E081E00E94D4118DEA95E012
:1053A0009F938F930E94BE9280E00E9456220E949B
:1053B0007C20809157021F928F9384EA95E09F93FF
:1053C0008F930E94BE928091C1091F928F938BE9A7
:1053D00095E09F938F930E94BE92809183028F935A
:1053E000809182028F93809181028F9380918002BD
:1053F0008F938DE895E09F938F930E94BE921F92AA
:1054000080E48F9385E795E09F938F930E94BE92EF
:105410008091B3281F928F938091B2281F928F930F
:1054200082E695E09F938F930E94BE9280915602F0
:105430001F928F9389E595E09F938F930E94BE9270
:105440008091580290915902A0915A02B0915B024A
:105450002DB73EB7225E3F4F0FB6F8943EBF0FBE4A
:105460002DBF96FF03C08EE895E002C081E995E06C
:105470009F938F938FE495E09F938F930E94BE92AA
:1054800083E00E9415290F900F900F900F901D9BA5
:1054900003C08EE895E002C081E995E09F938F9369
:1054A00083E495E09F938F930E94BE9289E395E0F9
:1054B0009F938F930E94BE92809158020F900F90FD
:1054C0000F900F900F900F9081FF09C083E395E03C
:1054D0009F938F930E94BE920F900F9013C080FFF6
:1054E00003C08EE895E002C081E995E09F938F9319
:1054F0008FE295E09F938F930E94BE920F900F9042
:105500000F900F908091580290915902A0915A02E9
:10551000B0915B0297FF03C08EE895E002C081E97D
:1055200095E09F938F9386E295E09F938F930E94DF
:10553000BE928FE195E09F938F930E94BE926091FF
:10554000C5097091C60980E090E00E9486220E9401
:10555000AB0B0F900F900F900F900F900F907799CB
:1055600003C08EE895E002C081E995E09F938F9398
:1055700086E195E09F938F930E94BE920E944B0913
:105580000E94F50A9F938F937F936F9388E095E035
:105590009F938F930E94BE920E94A40A9F938F9321
:1055A0007F936F938AEF94E09F938F930E94BE92B4
:1055B00081E090E00E943221809188289091892892
:1055C000A0918A28B0918B28BF93AF939F938F931C
:1055D0008CEE94E09F938F930E94BE9280919D28C1
:1055E0008F9380919C288F9380919B288F9380919B
:1055F0009A288F9388ED94E09F938F930E94BE9298
:1056000080918C2890918D28A0918E28B0918F2820
:10561000BF93AF939F938F938AEC94E09F938F9364
:105620000E94BE928DB79EB782960FB6F8949EBF29
:105630000FBE8DBF8091A1288F938091A0288F935A
:1056400080919F288F9380919E288F9386EB94E082
:105650009F938F930E94BE9261E070E080E090E0A3
:105660000E94B40B0F900F900F900F900F900F901F
:1056700061E070E081E090E00C94B40BF894E0E01D
:10568000F0E081E2809357008491E2E0F0E041E2B3
:10569000409357004491E4E0F0E091E2909357008A
:1056A000E49190E0A0E0B0E0DC019927882750E089
:1056B00060E070E0762F652F542F4427840F951FEC
:1056C000A61FB71F8E0F911DA11DB11D8093C81B72
:1056D0009093C91BA093CA1BB093CB1B78940895D9
:1056E000CF93DF93CDB7DEB761970FB6F894DEBFE7
:1056F0000FBECDBF48E250E06EE170E087E29BE173
:105700000E9412942091271B3091281B4091291B45
:1057100050912A1B60912B1B70912C1B80912D1B8B
:1057200090912E1BAFEF0E942D8E09F05DC08DE48D
:105730008093271B80E88093281B84E08093291B9B
:1057400010922A1B10922B1B10922C1B10922D1BB7
:1057500010922E1B8CE390E09093301B80932F1BB4
:105760001092311B1092321B1092331B1092341B7B
:105770001092351B1092361B1092371B1092381B5B
:1057800010923A1B1092391B10923B1B10923C1B3B
:1057900010923D1B10923E1B10923F1B1092401B1B
:1057A0001092411B1092421B1092441B1092431BFB
:1057B0001092451B1092461B1092471B1092481BDB
:1057C0001092491B10924A1B10924B1B10924C1BBB
:1057D00010924E1B10924D1B48E250E06EE170E0BB
:1057E00087E29BE10E94309444E050E06AE170E07F
:1057F000CE010B960E9412948B859C85AD85BE854B
:105800008F3F2FEF9207A207B207A9F48AE090E436
:10581000A0E0B0E08093580290935902A0935A02FE
:10582000B0935B0244E050E06AE170E088E592E00A
:105830000E94309408C08093580290935902A0931C
:105840005A02B0935B0242E050E066E570E0CE01A0
:105850000F960E9412948F8598898F3F2FEF9207A1
:1058600069F41092C6091092C50942E050E066E55D
:1058700070E085EC99E00E94309404C09093C609D2
:105880008093C50949E050E06AE070E082EA98E25E
:105890000E9412940E94EC0C44E050E06AE470E034
:1058A000CE010B960E9412948B859C85AD85BE859A
:1058B00044E050E06AE470E08F3F9F4FAF4FBF4F2E
:1058C00029F488E792E00E94309404C088E792E0CF
:1058D0000E94129444E050E066E470E0CE010B9622
:1058E0000E9412948B859C85AD85BE8544E050E076
:1058F00066E470E08F3F9F4FAF4FBF4F29F484E7BE
:1059000092E00E94309404C084E792E00E941294D6
:1059100044E050E06EE470E0CE010B960E941294D9
:105920008B859C85AD85BE8544E050E06EE470E0DB
:105930008F3F9F4FAF4FBF4F29F48CE792E00E94FB
:10594000309404C08CE792E00E94129441E050E051
:1059500069E170E0CE0141960E941294898941E08C
:1059600050E069E170E08F3F29F481EC99E00E94FA
:10597000309404C081EC99E00E94129441E050E020
:1059800068E170E0CE0141960E941294898941E05D
:1059900050E068E170E08F3F29F487E592E00E94D3
:1059A000309404C087E592E00E94129441E050E0F8
:1059B00067E170E0CE0141960E941294898941E02E
:1059C00050E067E170E08F3F29F486E592E00E94A5
:1059D000309404C086E592E00E9412944AE050E0C0
:1059E00060E070E0CE0101960E94129489814AE045
:1059F00050E060E070E08F3F29F48EE09BE10E9470
:105A0000309404C08EE09BE10E94129444E050E088
:105A100062E570E0CE010B960E9412948B859C8506
:105A2000AD85BE8544E050E062E570E08F3F9F4F5A
:105A3000AF4FBF4F29F480E892E00E94309404C039
:105A400080E892E00E94129444E050E063E170E04C
:105A5000CE010B960E9412948B859C85AD85BE85E8
:105A600044E050E063E170E08F3F9F4FAF4FBF4F86
:105A700029F482E592E00E94309404C082E592E02D
:105A80000E94129461960FB6F894DEBF0FBECDBF90
:105A9000DF91CF910895CF92DF92EF92FF926091C4
:105AA00071027091720280E090E00E94F39165E9CA
:105AB00075E00E940792892B09F01FC18DE4809345
:105AC000271B80E88093281B84E08093291B109279
:105AD0002A1B10922B1B10922C1B10922D1B109224
:105AE0002E1B8CE390E09093301B80932F1B109221
:105AF000311B1092321B1092331B1092341B1092E8
:105B0000351B1092361B1092371B1092381B1092C7
:105B10003A1B1092391B10923B1B10923C1B1092A7
:105B20003D1B10923E1B10923F1B1092401B109287
:105B3000411B1092421B1092441B1092431B109267
:105B4000451B1092461B1092471B1092481B109247
:105B5000491B10924A1B10924B1B10924C1B109227
:105B60004E1B10924D1B48E250E06EE170E087E260
:105B70009BE10E9430948AE090E4A0E0B0E0809342
:105B8000580290935902A0935A02B0935B0244E0EA
:105B900050E06AE170E088E592E00E943094109253
:105BA000C6091092C50942E050E066E570E085EC58
:105BB00099E00E94309442E2C42EDD24DA944CEC49
:105BC000E42E4BE3F42EC0927802D0927902E09258
:105BD0007A02F0927B0244E050E06AE470E088E7E9
:105BE00092E00E943094C0927402D0927502E092CA
:105BF0007602F092770244E050E066E470E084E7D9
:105C000092E00E94309487ED94E3AFEEBCE3809382
:105C10007C0290937D02A0937E02B0937F0244E0C9
:105C200050E06EE470E08CE792E00E9430948AE9E4
:105C300099E9A9E1B0E48093800290938102A09356
:105C40008202B093830244E050E062E570E080E8B5
:105C500092E00E9430941092C10980E00E943A6A5A
:105C600041E050E069E170E081EC99E00E943094FD
:105C70008AE1809357020E94E16841E050E068E1C8
:105C800070E087E592E00E9430948FE080935602A6
:105C900041E050E067E170E086E592E00E943094D8
:105CA0008AE0EEE0FBE1DF011D928A95E9F74AE028
:105CB00050E060E070E0CF010E94309480EA96E806
:105CC000A1E0B0E08093520290935302A09354025B
:105CD000B093550244E050E063E170E082E592E069
:105CE0000E94309481E00E94562280E090E0FF9074
:105CF000EF90DF90CF900C94000DFF90EF90DF902D
:105D0000CF9008952F923F924F925F926F927F9221
:105D10008F929F92AF92BF92CF92DF92EF92FF92BB
:105D20000F931F93CF93DF93CDB7DEB72B970FB6AB
:105D3000F894DEBF0FBECDBF9B878A874A01FC0166
:105D400080819181892B11F00C941E416091710228
:105D500070917202CA010E94F39160E470E0C40184
:105D60000E942692009759F460916D3170916E31C6
:105D70008AE090E00E947A9281E00C942341813085
:105D8000910561F4F401B0801B2D110F110B012F4F
:105D9000412E512E612E712EA12EBCC08230910554
:105DA000B9F4F4018081992787FD9095982F882771
:105DB0002181820F911D27FD9A95B82E192F092F49
:105DC000000F000B402E502E602E702EA02EA2C071
:105DD00083309105B1F5F4012081922F990F990B31
:105DE000392F492F592F692F792F892F00E10E94D0
:105DF000CF8D19012A013B01B82FA92F2181922FA4
:105E0000990F990B392F492F592F692F792F892FE6
:105E100008E00E94CF8D59016A017B018C0191013C
:105E2000A201B3018B2F9A2F0E94068EA2801A2DF9
:105E3000110F110BB12EC12ED12EE12EF12E012FFB
:105E400055C004970CF45DC0F4012081922F990F86
:105E5000990B392F492F592F692F792F892F08E155
:105E60000E94CF8D19012A013B01B82FA92F218152
:105E7000922F990F990B392F492F592F692F792F6D
:105E8000892F00E10E94CF8D59016A017B018C01AD
:105E90009101A201B3018B2F9A2F0E94068EA3803D
:105EA0001A2D110F110BB12EC12ED12EE12EF12E74
:105EB000012F0E94068E19012A013B01B82FA92F3C
:105EC0002281922F990F990B392F492F592F692F22
:105ED000792F892F08E00E94CF8D59016A017B013B
:105EE0008C019101A201B3018B2F9A2F0E94068E83
:105EF000B22E132F042F452E562E672E782EA92E44
:105F000009C07AE0B72E10E000E0412C512C612C42
:105F1000712CA12C0E94AB0B2B2D312F402F542D17
:105F2000652D762D872D9A2D2736FFE63F07FCE657
:105F30004F075105610571058105910511F40C9418
:105F40002B3B2736EFE63E07ECE64E075105610591
:105F500071058105910511F008F096C12936F2E727
:105F60003F0741055105610571058105910511F452
:105F70000C94483E2936E2E73E074105510561058C
:105F800071058105910511F008F0A6C02536F4E6EB
:105F90003F0741055105610571058105910509F42A
:105FA00057C62536E4E63E074105510561057105F2
:105FB0008105910509F0B8F5A6E70E942D8E11F430
:105FC0000C949F380E942D8E09F068F4A8E60E9478
:105FD0002D8E09F483C6A5E70E942D8E11F40C9432
:105FE00089380C941C412B2D312F402F542D652DB9
:105FF000762D872D9A2D2A33F6E23F07410551056C
:10600000610571058105910509F41FC324363146E8
:1060100041055105610571058105910511F40C9447
:10602000C13E0C941C412B2D312F402F542D652D3A
:10603000762D872D9A2D2737FFE63F07410551051D
:10604000610571058105910511F40C946C3C2737AD
:10605000EFE63E0741055105610571058105910592
:1060600009F0C8F42436F9E63F07410551056105FA
:1060700071058105910511F40C94623825363E4670
:1060800041055105610571058105910511F40C94D7
:10609000A03C0C941C412B2D312F402F542D652DED
:1060A000762D872D9A2D2333F1E73F0741055105C2
:1060B000610571058105910511F40C94C13E2536E9
:1060C000324741055105610571058105910511F4BE
:1060D0000C946A3D0C941C412B2D312F402F542DD4
:1060E000652D762D872D9A2D2837F4E63F07F1E6AA
:1060F0004F075105610571058105910509F4B5C288
:106100002837E4E63E07E1E64E07510561057105D3
:106110008105910511F008F050C02837F4E73F07DA
:1061200041055105610571058105910509F48DC28F
:106130002837E4E73E0741055105610571058105F2
:10614000910509F0C8F42337F2E73F0741055105EF
:10615000610571058105910511F40C94993E233771
:10616000334741055105610571058105910511F41C
:106170000C94AD3E0C941C412B2D312F402F542DEF
:10618000652D762D872D9A2D2133F4E63F07F1E614
:106190004F075105610571058105910509F469C233
:1061A0002336344641465105610571058105910547
:1061B00011F40C94C13E0C941C412B2D312F402F17
:1061C000542D652D762D872D9A2D2336FDE63F071C
:1061D000F8E64F075105610571058105910509F440
:1061E00040C32336EDE63E07E8E64E07510561055C
:1061F00071058105910509F0C8F42236F5E63F07DF
:10620000F4E64F075105610571058105910509F413
:106210001FC5223732474546510561057105810585
:10622000910511F40C94C53B0C941C412B2D312F7E
:10623000402F542D652D762D872D9A2D2336F2E390
:106240003F07F9E64F075105610571058105910585
:1062500009F42FC22436E3E63E07ECE64E0751056B
:10626000610571058105910511F40C94283B2D36CB
:10627000354748465105610571058105910511F0C5
:106280000C941C410C94D73E2B2D312F402F542DB4
:10629000652D762D872D9A2D2136EDE63E07E5E713
:1062A0004E07E8E65E07610571058105910511F469
:1062B0000C948A3C2136FDE63F07F5E74F07F8E6E8
:1062C0005F07610571058105910511F008F0DAC0DD
:1062D0002437E8E73E07E4E74E07510561057105FD
:1062E0008105910509F497C72437F8E73F07F4E7DC
:1062F0004F075105610571058105910511F008F001
:1063000055C02133E1E33E07E1E74E075105610542
:1063100071058105910511F40C94063C2133F1E3DC
:106320003F07F1E74F0751056105710581059105AB
:1063300009F0D0F42537E3E63E07EDE64E075105B8
:10634000610571058105910511F40C94063C20331B
:10635000314341475105610571058105910511F4EE
:106360000C94C53B0C941C412B2D312F402F542DE8
:10637000652D762D872D9A2D2037E5E63E07E2E73D
:106380004E075105610571058105910511F40C94C5
:106390006A3D2C3634474447510561057105810536
:1063A000910511F40C9445400C941C412B2D312F78
:1063B000402F542D652D762D872D9A2D2936ECE60C
:1063C0003E07E1E64E07E3E65E07610571058105DC
:1063D000910509F47BC22936FCE63F07F1E64F0739
:1063E000F3E65F07610571058105910509F0E0F4A9
:1063F0002437E4E63E07E7E74E07510561057105DE
:106400008105910511F40C94934024373F464F4683
:106410005246610571058105910511F00C941C41EE
:106420000C9400000C941E412B2D312F402F542D25
:10643000652D762D872D9A2D2633E9E63E07E5E773
:106440004E07E5E65E07610571058105910509F4D2
:1064500049C42037FCE63F07F5E64F07F8E65F073B
:10646000610571058105910509F438C42E36314660
:1064700048465346610571058105910509F49FC69B
:106480000C941C412B2D312F402F542D652D762D32
:10649000872D9A2D2437F3E73F07F5E64F07F2E7FC
:1064A0005F07610571058105910511F40C941A3D92
:1064B0002437E3E73E07E5E64E07E2E75E076105BE
:1064C00071058105910511F008F055C02337F2E7F9
:1064D0003F07F7E74F07F0E75F07610571058105A3
:1064E000910511F40C941D3D2337E2E73E07E7E7E1
:1064F0004E07E0E75E07610571058105910509F02A
:10650000C8F42237F7E73F07F0E74F075F07610559
:1065100071058105910509F4A8C123373546424725
:106520005047610571058105910511F40C94873F71
:106530000C941C412B2D312F402F542D652D762D81
:10654000872D9A2D2436FDE63F07F3E64F07F2E745
:106550005F07610571058105910509F4CEC42136F7
:106560003C4645465247610571058105910509F490
:10657000D6C30C941C412B2D312F402F542D652D4B
:10658000762D872D9A2D2437F2E73F07F1E64F0746
:10659000F5E75F07610571058105910509F408C5F7
:1065A0002437E2E73E07E1E64E07E5E75E076105CF
:1065B00071058105910509F0C8F42437F3E73F0719
:1065C000F5E64F07F4E75F07610571058105910561
:1065D00009F44CC6273730474847544761057105D1
:1065E0008105910509F4C1C50C941C412B2D312F57
:1065F000402F542D652D762D872D9A2D2F36FCE6B4
:106600003F07FFE54F07F6E75F0761057105810565
:10661000910509F41DC42C36E1E63E07E4E74E0778
:10662000E8E75E07610571058105910511F40C9499
:106630000F402237374640475547610571058105B0
:10664000910511F00C941C41E0C783E080939028E1
:10665000109292281092912840E958E262E184E376
:1066600092E00E9444540C941E410E94B8150C9470
:106670001E4121E042E161E080ED0E947E6121E067
:1066800042E161E080ED0E947E6121E042E161E053
:1066900080ED0E947E6121E042E161E080ED0E9498
:1066A0007E6121E042E161E080ED0E947E610C9418
:1066B0001E41609171027091720280E090E00E9430
:1066C000F3916CE975E00E940792892B09F0C5C02F
:1066D000609171027091720280E090E00E94F391EB
:1066E0005C01009709F497C060EE73E00E94079286
:1066F000892BE1F488EE93E0A0E0B0E080935202B1
:1067000090935302A0935402B093550268EE73E045
:1067100080E090E00E94A55F44E050E063E170E01B
:1067200082E592E00E9430940C941E4162EA75E08A
:10673000C5010E940792892BE1F480E197E2A0E075
:10674000B0E08093520290935302A0935402B0930E
:10675000550260E177E280E090E00E94A55F44E0AE
:1067600050E063E170E082E592E00E9430940C9486
:106770001E4165EA75E0C5010E940792892BE1F48C
:1067800080EA96E8A1E0B0E0809352029093530231
:10679000A0935402B093550260EA76E881E090E05D
:1067A0000E94A55F44E050E063E170E082E592E082
:1067B0000E9430940C941E4169EA75E0C5010E9464
:1067C0000792892BE1F480E89AE1A6E0B0E080939B
:1067D000520290935302A0935402B093550260E882
:1067E0007AE186E090E00E94A55F44E050E063E13A
:1067F00070E082E592E00E9430940C941E4187EF95
:1068000092E09F938F930E94BE920E94AB0B0F90D9
:106810000F900C941E41609152027091530280912E
:1068200054029091550228EE33E040E050E00E947F
:10683000268C5F934F933F932F9383EF92E09F9328
:106840008F930E94BE920E94AB0B0F900F900F90FF
:106850000F900F900F900C941E410E942A100C94E0
:106860001E410E9430160C941E416091710270917D
:10687000720280E090E00E94F3918C016EE875E076
:106880000E940792892B19F477980C941E4161E9B4
:1068900075E0C8010E940792892B19F4779A0C942D
:1068A0001E41779903C08EE895E002C081E995E02A
:1068B0009F938F9380EA94E09F938F930E94BE9260
:1068C0000F900F900F900F900C941E4160917102E9
:1068D0007091720280E090E00E94F3918C0168E573
:1068E00075E00E940792892B09F077C060917102D0
:1068F0007091720280E090E00E94F3918C01009709
:1069000011F40C941E416DEA75E00E940792892BE8
:10691000B1F482E29FEFACECBBE3809378029093FA
:106920007902A0937A02B0937B0244E050E06AE4DB
:1069300070E088E792E00E9430940C941E4163EB73
:1069400075E0C8010E940792892BB1F482E29FEFA3
:10695000ACECBAE38093780290937902A0937A0228
:10696000B0937B0244E050E06AE470E088E792E094
:106970000E9430940C941E41C8010E94DD902B01AE
:106980003C0120E030E0A9010E9478888823D9F0FA
:1069900081E00E94410A9B01AC01C301B2010E9447
:1069A0007C88609378027093790280937A02909346
:1069B0007B0244E050E06AE470E088E792E00E94E5
:1069C00030940C941E4186EE92E09F938F930E9428
:1069D000BE920F900F900C941E416BE575E0C801BC
:1069E0000E940792892B09F077C060917102709123
:1069F000720280E090E00E94F3918C01009711F404
:106A00000C941E416DEA75E00E940792892BB1F447
:106A100082E29FEFACECBBE380937402909375022B
:106A2000A0937602B093770244E050E066E470E011
:106A300084E792E00E9430940C941E4163EB75E071
:106A4000C8010E940792892BB1F482E29FEFACEC5F
:106A5000BAE38093740290937502A0937602B09388
:106A6000770244E050E066E470E084E792E00E9440
:106A700030940C941E41C8010E94DD902B013C0112
:106A800020E030E0A9010E9478888823D9F082E0D4
:106A90000E94410A9B01AC01C301B2010E947C88A3
:106AA00060937402709375028093760290937702DC
:106AB00044E050E066E470E084E792E00E943094A5
:106AC0000C941E4189ED92E09F938F930E94BE9299
:106AD0000F900F900C941E4163E575E0C8010E9471
:106AE0000792892B09F073C0609171027091720254
:106AF00080E090E00E94F3918C01009711F40C94D7
:106B00001E416DEA75E00E940792892BB1F487ED72
:106B100094E3AFEEBCE380937C0290937D02A0935C
:106B20007E02B0937F0244E050E06EE470E08CE7B8
:106B300092E00E9430940C941E4163EB75E0C80112
:106B40000E940792892B51F48AEC92E09F938F93D5
:106B50000E94BE920F900F900C941E41C8010E949B
:106B6000DD902B013C0120E030E0A9010E947888F3
:106B7000882319F180E00E94410A4B015C0121EE5B
:106B80003AE744E95EE3C301B2010E94B187A5017F
:106B900094010E947C8860937C0270937D028093B4
:106BA0007E0290937F0244E050E06EE470E08CE758
:106BB00092E00E9430940C941E418DEB92E09F93E2
:106BC0008F930E94BE920F900F900C941E410E94D2
:106BD000900A9F938F937F936F9386EB92E09F939E
:106BE0008F930E94BE9282E00E94410A209174021B
:106BF0003091750240917602509177020E94FD8A91
:106C0000162F072FF82EE92E81E00E94410AEF92FD
:106C1000FF920F931F932091780230917902409157
:106C20007A0250917B020E94FD8A9F938F937F93FB
:106C30006F938AEA92E09F938F930E94BE920E9484
:106C4000AB0B0FB6F894DEBF0FBECDBF0C941E4148
:106C5000609171027091720280E090E00E94F39165
:106C60000097C1F00E9474232091C5093091C60994
:106C70008217930709F19093C6098093C50942E0F2
:106C800050E066E570E085EC99E00E94309489E977
:106C900094E002C082E994E09F938F930E94BE9299
:106CA0006091C5097091C60980E090E00E9486223B
:106CB0000E94AB0B0F900F9087E894E09F938F9307
:106CC0000E94BE926FEF7FEF80E090E00E948622EC
:106CD0000E94AB0B0F900F900C941E410E94871FD7
:106CE0000C941E41F4018481843329F440E061E076
:106CF00080E00E94D41180917302882311F40C94D7
:106D00001E411F928F9384E894E09F938F930E947B
:106D1000BE920F900F900F900F900C941E41F401B3
:106D20008481893709F080C060917102709172028C
:106D300080E090E00E94F3918C016EE875E00E9483
:106D40000792892B51F48091580290915902A09199
:106D50005A02B0915B02906410C061E975E0C8010D
:106D60000E940792892BD1F4809158029091590288
:106D7000A0915A02B0915B029F7B8093580290933E
:106D80005902A0935A02B0935B0244E050E06AE1DA
:106D900070E088E592E00E94309446C068EB75E0B0
:106DA000C8010E940792892B21F58091261B8F93A1
:106DB0008091251B8F938091241B8F938091231B9F
:106DC0008F938091221B8F938091211B8F938091B1
:106DD000201B8F9380911F1B8F938FE792E09F93CF
:106DE0008F930E94BE920FB6F894DEBF0FBECDBF48
:106DF0001BC08091580290915902A0915A02B09103
:106E00005B0296FF03C08EE895E002C081E995E041
:106E10009F938F938BE792E09F938F930E94BE92F4
:106E20000F900F900F900F9080917302882311F4B0
:106E30000C941E411F928F9381E894E09F938F934F
:106E40000E94BE920F900F900F900F900C941E41D5
:106E5000F40184818737E9F56091710270917202C3
:106E600080E090E00E94F3910097D9F00E94DD90BD
:106E70002B013C0120E030E0A9010E9478888823A2
:106E800081F0409280025092810260928202709260
:106E9000830244E050E062E570E080E892E00E9406
:106EA0003094809183028F93809182028F9380919E
:106EB00081028F93809180028F938DE692E09F9361
:106EC0008F930E94BE920F900F900F900F900F9093
:106ED0000F9080917302882311F40C941E411F922D
:106EE0008F938EE794E09F938F930E94BE920F90B2
:106EF0000F900F900F900C941E4160917102709151
:106F0000720280E090E00E94F3918C016EE875E0DF
:106F10000E940792409058025090590260905A0285
:106F200070905B02892B19F4689457F809C061E9E5
:106F300075E0C8010E940792892B99F4E89457F8EC
:106F4000409258025092590260925A0270925B022B
:106F500044E050E06AE170E088E592E00E943094FD
:106F600013C057FE03C08EE895E002C081E995E0AA
:106F70009F938F9389E692E09F938F930E94BE9296
:106F80000F900F900F900F9080917302882311F44F
:106F90000C941E411F928F938BE794E09F938F93E5
:106FA0000E94BE920F900F900F900F900C941E4174
:106FB000609171027091720280E090E00E94F39102
:106FC0005C016EEB75E00E940792892B11F489E158
:106FD00008C062EC75E0C5010E940792892B49F454
:106FE00080E18093C4001092C50082E08093C000CD
:106FF00055C066EC75E0C5010E940792892B11F41B
:1070000088E0EFCF6BEC75E0C5010E940792892BF9
:1070100039F060ED75E0C5010E940792892B11F4EB
:1070200083E0DFCF8091C400893141F484E692E0AF
:107030009F938F930E94BE920F900F908091C400F7
:10704000803141F48FE592E09F938F930E94BE922E
:107050000F900F908091C400883041F489E592E050
:107060009F938F930E94BE920F900F908091C400C7
:10707000833041F483E592E09F938F930E94BE9208
:107080000F900F908091C400883041F48DE492E01D
:107090009F938F930E94BE920F900F9080917302E6
:1070A000882311F40C941E411F928F9388E794E07B
:1070B0009F938F930E94BE920F900F900F900F900E
:1070C0000C941E41609171027091720280E090E018
:1070D0000E94F3916DEA75E00E940792892B11F4EA
:1070E00081E001C080E00E945622809173028823D3
:1070F00011F40C941E411F928F9385E794E09F93A7
:107100008F930E94BE920F900F900F900F900C944F
:107110001E410E947C2080917302882311F40C94FC
:107120001E411F928F9382E794E09F938F930E945A
:10713000BE920F900F900F900F900C941E410E94E2
:10714000782080917302882311F40C941E411F92C1
:107150008F938FE694E09F938F930E94BE920F903F
:107160000F900F900F900C941E41609171027091DE
:10717000720280E090E00E94F3910E94E1908031E1
:1071800070F48093C1090E943A6A41E050E069E1DD
:1071900070E081EC99E00E9430940C941E41809143
:1071A000C1091F928F9383E492E09F938F930E9473
:1071B000BE920F900F900F900F900C941E41609113
:1071C00071027091720280E090E00E94F3910E943F
:1071D000E19095EF980F903170F4809357020E94E0
:1071E000E16841E050E068E170E087E592E00E94EC
:1071F00030940C941E41809157021F928F938AE322
:1072000092E09F938F930E94BE920F900F900F90E9
:107210000F900C941E41609171027091720280E097
:1072200090E00E94F391009789F04AE050E0BC01A1
:107230008EE09BE10E9417924AE050E060E070E02F
:107240008EE09BE10E9430940C941E418EE09BE105
:107250009F938F9385ED95E09F938F930E94AC92BF
:107260000F900F900F900F900C941E41609171023F
:107270007091720280E090E00E94F3915C0160EEF8
:1072800073E00E940792892BD9F4219A80915802C9
:1072900090915902A0915A02B0915B028061809353
:1072A000580290935902A0935A02B0935B0244E0B3
:1072B00050E06AE170E088E592E00E943094BEC739
:1072C0006CE575E0C5010E940792892BD9F4229ADA
:1072D0008091580290915902A0915A02B0915B029C
:1072E00080628093580290935902A0935A02B093FF
:1072F0005B0244E050E06AE170E088E592E00E94C1
:1073000030949CC762EC73E0C5010E940792892B00
:10731000D9F4239A8091580290915902A0915A026F
:10732000B0915B0280648093580290935902A093BD
:107330005A02B0935B0244E050E06AE170E088E5F5
:1073400092E00E9430947AC76FEF74E0C5010E940A
:107350000792892BD9F4239A80915802909159026F
:10736000A0915A02B0915B0280688093580290937A
:107370005902A0935A02B0935B0244E050E06AE1E4
:1073800070E088E592E00E94309458C76CE679E09E
:10739000C5010E940792892B71F581E08093342406
:1073A00087E29BE190933624809335241092382411
:1073B000109237248091580290915902A0915A025C
:1073C000B0915B0291608093580290935902A09310
:1073D0005A02B0935B0244E050E06AE170E088E555
:1073E00092E00E94309444E354E262E184E392E04C
:1073F0000E94445423C769EE73E0C5010E940792BE
:10740000892B11F5E7E5FBE1119211922BE1E737AA
:10741000F207D1F78091580290915902A0915A0237
:10742000B0915B0292608093580290935902A093AE
:107430005A02B0935B0244E050E06AE170E088E5F4
:1074400092E00E943094FAC661E975E0C5010E949D
:107450000792409158025091590260915A027091DE
:107460005B02892BC1F44F705C7F409358025093AC
:10747000590260935A0270935B022B9A44E050E0E9
:107480006AE170E088E592E00E943094809199284A
:107490000E94F668D3C644FF03C08EE895E002C0A0
:1074A00081E995E09F938F938FE292E09F938F9372
:1074B0000E94BE92809158020F900F900F900F90F3
:1074C00085FF03C08EE895E002C081E995E09F93B7
:1074D0008F9384E292E09F938F930E94BE9280915B
:1074E00058020F900F900F900F9086FF03C08EE808
:1074F00095E002C081E995E09F938F9389E192E046
:107500009F938F930E94BE92809158020F900F908C
:107510000F900F9087FF03C08EE895E002C081E9CD
:1075200095E09F938F938EE092E09F938F930E94BC
:10753000BE928091580290915902A0915A02B09146
:107540005B020F900F900F900F9090FF03C08EE89A
:1075500095E002C081E995E09F938F9383E092E0EC
:107560009F938F930E94BE928091580290915902EE
:10757000A0915A02B0915B020F900F900F900F9064
:1075800091FF03C08EE895E002C081E995E09F93EA
:107590008F9388EF91E09F938F930E94BE9280918A
:1075A000580290915902A0915A02B0915B020F903B
:1075B0000F900F900F9091FF41C68DED95E00E94C6
:1075C000E29257E5A52E5BE1B52E0BE010E065EEEB
:1075D000862E65E0962EF50180819181F2E0AF0E56
:1075E000B11C9F938F931F930F939F928F920E9432
:1075F000AC920F5F1F4F0F900F900F900F900F9056
:107600000F900B31110539F719C68BE694E09F9363
:107610008F930E94BE92809173020F900F908823E7
:1076200061F01F928F9388E694E09F938F930E945E
:10763000BE920F900F900F900F9088E10FB6F894C4
:1076400080936000109260000FBE0C94007CF6C521
:107650000E942F61F3C5609171027091720280E007
:1076600090E00E94F3918C016EE875E00E94079211
:10767000892BE9F40E94E0678091580290915902A9
:10768000A0915A02B0915B028D7F81608093580275
:1076900090935902A0935A02B0935B0244E050E0E9
:1076A0006AE170E088E592E00E943094C7C561E924
:1076B00075E0C8010E940792892BE1F40E94986747
:1076C0008091580290915902A0915A02B0915B02A8
:1076D0008C7F8093580290935902A0935A02B093E2
:1076E0005B0244E050E06AE170E088E592E00E94CD
:1076F0003094A4C560EF75E0C8010E940792892B01
:10770000E9F40E9498678091580290915902A091E3
:107710005A02B0915B028E7F8260809358029093F0
:107720005902A0935A02B0935B0244E050E06AE130
:1077300070E088E592E00E94309480C58091580204
:1077400081FF0FC080EF95E09F938F9384EF91E0CE
:107750009F938F930E94BE920F900F900F900F9067
:107760006DC580FF03C08EE895E002C081E995E019
:107770009F938F9380EF91E09F938F930E94BE928F
:107780000F900F900F900F9059C5809132248F93D6
:10779000809131248F93809130248F9380912F2476
:1077A0008F9380912E248F9380912D248F9380919D
:1077B0002C248F9380912B248F9380912A248F9354
:1077C000809129248F93809128248F93809127245E
:1077D0008F9385E494E09F938F930E94BE92809153
:1077E00073020FB6F894DEBF0FBECDBF882309F435
:1077F00025C51F928F9382E494E09F938F930E94FC
:10780000BE920F900F900F900F9018C5F89481E0E2
:1078100090E029E0FC0120935700C895E02C80E01F
:1078200090E0FC0120935700C895F02C7894F894D0
:1078300083E090E0FC0120935700C895002D82E082
:1078400090E0FC0120935700C895102D789480910A
:10785000CB1B8F938091CA1B8F938091C91B8F93F1
:107860008091C81B8F9328E334E03F932F930E94AD
:10787000BE921F92EF921F92FF921F920F931F9240
:107880001F9381E194E09F938F930E94BE920E9488
:107890001621809166001F928F9385E094E09F935C
:1078A0008F930E94BE920E94AB0B809173020FB621
:1078B000F894DEBF0FBECDBF882309F4BFC41F926A
:1078C0008F9382E094E09F938F930E94BE920F90DB
:1078D0000F900F900F90B2C460E070E080E090E0F5
:1078E0000E94B40B60E070E081E090E00E94B40B75
:1078F00080917302882309F4A1C41F928F938FEFA4
:1079000093E09F938F930E94BE920F900F900F90E1
:107910000F9094C40E944A1F0E94AB0B8091730287
:10792000882309F48BC41F928F938CEF93E09F936D
:107930008F930E94BE920F900F900F900F907EC475
:10794000609171027091720280E090E00E94F39168
:1079500065EF75E00E940792892B31F5F8948CEF62
:1079600099E00E9431555C01009769F0C5010F96BE
:107970000E943558B50184E092E00E94EB54C501A5
:107980000E94D955F0CF8CEF99E00E94BE55892B0B
:1079900029F08CEF99E00E946A55F5CF8CEF99E0C1
:1079A0000E942D55789434C08CEF99E00E94315597
:1079B0005C010BEF15E0A114B10451F1F5018681D2
:1079C0001F928F9380851F928F9385811F928F9333
:1079D00081851F928F9387811F928F9384811F923D
:1079E0008F9383811F928F9382811F928F938285C1
:1079F0001F928F931F930F930E94AC92C5010E9418
:107A0000D9555C010FB6F894DEBF0FBECDBFD3CF02
:107A100080917302882309F411C41F928F9389EF18
:107A200093E09F938F930E94BE920F900F900F90C0
:107A30000F9004C40E944B2D01C46091710270919B
:107A4000720280E090E00E94F3918C016AE376E09C
:107A50000E940792892BD1F480915802909159028B
:107A6000A0915A02B0915B02977F80935802909345
:107A70005902A0935A02B0935B0244E050E06AE1DD
:107A800070E088E592E00E943094D8C363EB75E023
:107A9000C8010E940792892BD1F4809158029091DD
:107AA0005902A0915A02B0915B02986080935802EB
:107AB00090935902A0935A02B0935B0244E050E0C5
:107AC0006AE170E088E592E00E943094B7C30E94BA
:107AD0004B09B4C3609171027091720280E090E032
:107AE0000E94F391FC0120812332B1F44AE050E07E
:107AF00060E070E001960E94958E1B01609171021A
:107B00007091720280E090E00E94F391F4E02F16F1
:107B100031040CF094C002C0212C312C009709F4E0
:107B20008EC01982BE016F5F7F4F0E9473272901AB
:107B30003A014B01B82FA92F8AE0829DF001839D65
:107B4000F00D1124E95DF44E20812A8331813B83BD
:107B500082818C8393819D8324812E8335813F8311
:107B600086818887978199879201A301B4018B2F21
:107B70009A2FAA80BB80CC80DD80EE80FF800885B4
:107B800019850E94248E09F45DC08981882351F1F2
:107B90008CF02A81422A3B81532A8C81682A9D815C
:107BA000792A2E81822A3F81932A8885B82B99854C
:107BB000A92B18C040945094609470948094909431
:107BC000B095A0952A8142223B8153228C81682264
:107BD0009D8179222E8182223F8193228885B8233C
:107BE0009985A92340825182628273828482958220
:107BF000B683A78348E250E06EE170E087E29BE144
:107C00000E94309481EF93E09F938F930E94BE92E5
:107C10008AE0829DF001839DF00D1124E95DF44E10
:107C20002081318142815381648175818681978170
:107C30000E940F240E94AB0B0F900F9003C082E0B4
:107C40000E94152985EE93E09F938F930E94BE9228
:107C50002FEF3FEF4FEF5FEF6FEF7FEF8FEF9FEF74
:107C60000E940F240E94AB0B809173020F900F9023
:107C7000882309F4E3C21F928F9382EE93E09F93CF
:107C80008F930E94BE920F900F900F900F90D6C2CC
:107C9000609171027091720280E090E00E94F39115
:107CA000FC0120812332A1F44AE050E060E070E062
:107CB00001960E94958E8B01609171027091720203
:107CC00080E090E00E94F39104301105ECF402C0D2
:107CD00000E010E00097C1F04AE050E060E070E0A2
:107CE0000E94C98F2AE0209FF001219FF00D1124EE
:107CF000E95DF44E7187608748E250E06EE170E024
:107D000087E29BE10E94309481E00E9415298091D6
:107D10007302882309F492C21F928F938FED93E030
:107D20009F938F930E94BE920F900F900F900F9091
:107D300085C20E946E5880917302882309F47EC226
:107D40001F928F938CED93E09F938F930E94BE922E
:107D50000F900F900F900F9071C20E948A2980910E
:107D60007302882309F46AC21F928F9389ED93E00E
:107D70009F938F930E94BE920F900F900F900F9041
:107D80005DC280E090E00E943221809173028823DE
:107D900009F454C21F928F9386ED93E09F938F93C3
:107DA0000E94BE920F900F900F900F9047C280914B
:107DB0001D2081FF2DC00E94CE1E892B49F5809188
:107DC000141C8F938091131C8F938091121C8F939E
:107DD0008091111C8F938BEC93E09F938F930E9463
:107DE000BE928091B1288F938091B0288F9380911B
:107DF000AF288F938091AE288F938EEB93E09F9363
:107E00008F930E94BE920FB6F894DEBF0FBECDBF17
:107E10000E94AB0B80911D2090911E2090FF63C0AB
:107E200081E090E00E94451E3B014C0180E090E023
:107E30000E94451E1B012C010E94A31D9F928F9240
:107E40007F926F928DEA93E09F938F930E94BE92F0
:107E50005F924F923F922F928DE993E09F938F9381
:107E60000E94BE92222D332D442D552D662D772D47
:107E7000882D992D0E94461C9F938F937F936F931B
:107E800082E993E09F938F930E94BE92222D332D1F
:107E9000442D552D662D772D882D992D0E94A71CD8
:107EA0009F938F937F936F9384E893E09F938F9337
:107EB0000E94BE92222D332D442D552D662D772DF7
:107EC000882D992D0E94081D9F938F937F936F9308
:107ED00081E793E09F938F930E94BE920FB6F89430
:107EE000DEBF0FBECDBF0E94AB0B80917302882313
:107EF00009F4A4C11F928F938EE693E09F938F9312
:107F00000E94BE920F900F900F900F9097C180919A
:107F10001D2082FF2BC021E048E061E083E00E9449
:107F2000491380910F1C8F9380910E1C8F93809129
:107F30000D1C8F9380910C1C8F9380910B1C8F9341
:107F400080910A1C8F938091091C8F938091081C4B
:107F50008F9387E593E09F938F930E94BE920E9438
:107F6000AB0B0FB6F894DEBF0FBECDBF80911D20C6
:107F700090911E2091FF41C00E949317B62EA72E0C
:107F8000982E892E20E030E048EC52E4D501F4012F
:107F90006B2F7A2F8F2F9E2F0E94FD8A20E836EEBE
:107FA00045EC57E40E947C8821E03EED42E45EE32C
:107FB0000E94608B9B01AC0160E070E080E89FE371
:107FC0000E94B1872BE43AE34DEB57E30E947C8893
:107FD0009F938F937F936F938F929F92AF92BF9255
:107FE0008EE393E09F938F930E94BE920E94AB0B0F
:107FF0000FB6F894DEBF0FBECDBF80917302882309
:1080000009F41CC11F928F938BE393E09F938F938E
:108010000E94BE920F900F900F900F900FC1609131
:1080200071027091720280E090E00E94F3916FE320
:1080300076E00E940792892BB1F4609171027091F1
:10804000720280E090E00E94F391009709F4F6C07C
:108050000E94E190803108F0F1C090915201982B7C
:1080600090935201EBC0809152018F701F928F93B9
:1080700083EE91E09F938F930E94BE920E94AB0B80
:108080000F900F900F900F90D9C060917102709176
:10809000720280E090E00E94F391009711F14AE0B3
:1080A00050E060E070E00E94958E603198F460933B
:1080B00056021F926F938EE293E09F938F930E94DC
:1080C000BE9241E050E067E170E086E592E00E94F8
:1080D000309411C0809156021F928F9385E293E0F5
:1080E00006C0809156021F928F938CE193E09F937C
:1080F0008F930E94BE920F900F900F900F900E944E
:10810000AB0B80917302882309F498C01F928F9360
:1081100089E193E09F938F930E94BE920F900F90FE
:108120000F900F908BC0609171027091720280E08D
:1081300090E00E94F3918C016EE875E00E94079236
:10814000892BE1F40E94496680915802909159026E
:10815000A0915A02B0915B02906180935802909373
:108160005902A0935A02B0935B0244E050E06AE1E6
:1081700070E088E592E00E94309460C061E975E0AB
:10818000C8010E940792892B81F5F8940E945766D6
:1081900088E10FB6F89480936000109260000FBEE3
:1081A00084B7877F84BF809160008861809360007E
:1081B0001092600078948091580290915902A09199
:1081C0005A02B0915B029F7E8093580290935902AD
:1081D000A0935A02B0935B0244E050E06AE170E081
:1081E00088E592E00E94309429C064E476E0C801FA
:1081F0000E940792409158025091590260915A0290
:1082000070915B02892B21F454FF18C0F894FFCFC2
:1082100054FF03C08EE895E002C081E995E09F938A
:108220008F938FED91E09F938F930E94BE920F905A
:108230000F900F900F9002C00E946E1FEA85FB8581
:108240001182108283E02B960FB6F894DEBF0FBE2A
:10825000CDBFDF91CF911F910F91FF90EF90DF90F5
:10826000CF90BF90AF909F908F907F906F905F90D6
:108270004F903F902F9008950F931F93CF93DF93CC
:10828000EC018A0188819981009711F18137904131
:1082900021F01982188283E020C06231E9F4A8013C
:1082A00062E170E08DEE99E00E94822E84E080937E
:1082B000902810929228109291281093942800935D
:1082C000932840E958E262E184E392E00E9444543A
:1082D00081E790E19983888381E0DF91CF911F91BD
:1082E0000F9108950E943D666C9A6B9A6A9A6F9AF4
:1082F000729A749A739A779A809880B3897F80BBB8
:108300008398849887E080937E00549A0E943E2B45
:108310000E94702B81E00E94B50980E090E00E94ED
:10832000000D60915202709153028091540290911D
:1083300055020E94A55F0E94A40A60931F247093B7
:10834000202480932124909322248091580286FD3A
:10835000239A0895CF93DF93EC0188819981009748
:1083600041F08C35904109F48CC01982188283E069
:1083700093C00E9472418091580280FD05C081FF28
:1083800001C01D9B0E949867809170008C7F809334
:1083900070008091B60080628093B6001092B200A7
:1083A00082E08093B1008091B6008770E1F7809100
:1083B000700081608093700069E679E080E090E071
:1083C0000E9427660E94782080E00E94562280EE5C
:1083D0009EE09F938F930E94BE920E942A108091EC
:1083E0001D200F900F9086FD0E94DB6080911D2064
:1083F00090911E2090FD0E945F1D80911D2087FF9F
:1084000006C021E04CE061E080ED0E947E61809139
:10841000C1090E943A6A809157020E94E1680E9455
:10842000DE688093EC09809157020E94E168809198
:10843000C1091F928F938091EC091F928F9389E459
:1084400096E09F938F930E94AC921092EE09109247
:10845000ED090F900F900F900F900F900F9088E400
:1084600092E09093AC288093AB2883E290E09093C5
:10847000FF118093FE118CE590E19983888381E060
:108480000BC06332E1F748E454E260E070E08DEE47
:1084900099E00E94822EE3CFDF91CF910895843638
:1084A000910514F19F938F938BE596E09F938F93A3
:1084B0000E94AC928091272490912824A091292495
:1084C000B0912A240196A11DB11D80932724909379
:1084D0002824A0932924B0932A240F900F900F9062
:1084E0000F9081E090E0089580E090E008952F9251
:1084F0003F924F925F926F927F928F929F92AF9234
:10850000BF92CF92DF92EF92FF920F931F93CF9380
:10851000DF93CDB7DEB7C859D1090FB6F894DEBFE7
:108520000FBECDBFCF56DF4F99838883C159D0404E
:108530008A01633871F481EF99E0C856DF4F688390
:10854000C859D0400E948752C856DF4F6881C85929
:10855000D040CF56DF4FA881B981C159D0402D916D
:108560003C912930B0E13B0709F4C9C340F421151F
:10857000310581F027343E4009F407C4FBC32B3199
:1085800040E1340709F4D7C32232304111F40C948E
:108590008F4FF0C34AEE52E061E870E081EF99E05E
:1085A0000E946D5287E49EE0A1C3E3E0F0E0EC0F8F
:1085B000FD1FE20FF31F1082C9010E944F42892B59
:1085C00089F720E030E040E050E0C357DF4F68819A
:1085D000CD58D040627070E080E090E0A0E00E9452
:1085E0002D8E09F084C6C557DF4F2881CB58D04067
:1085F000287030E040E050E060E070E080E090E023
:10860000A0E00E942D8EA1F127E04AE250E06BE24B
:1086100070E089E290E00E94BF5C82EA98E20E94EA
:108620002D5FBC01882777FD8095982F0E941B89BC
:1086300020E030E048EC52E40E947C889F938F93C6
:108640007F936F938FE896E09F938F931F9287E7B6
:108650008F93CE018E0D9F1D03969F938F930E9443
:108660000F93E80EF91E0FB6F894DEBF0FBECDBF14
:10867000C557DF4F2881CB58D040207130E040E013
:1086800050E060E070E080E090E0A0E00E942D8E7D
:10869000F1F126E04AE250E06BE270E089E290E01E
:1086A0000E94BF5C81E090E00E94390B8093C0097A
:1086B00080E89BE10E942D5FBC01882777FD8095B3
:1086C000982F0E941B8920E030E048EC52E40E9481
:1086D0007C889F938F937F936F9389E996E09F9314
:1086E0008F931F9287E78F93C7010296E1E0F0E036
:1086F000EC0FFD1F8E0F9F1F9F938F930E940F9370
:10870000E80EF91E0FB6F894DEBF0FBECDBF272DC1
:1087100030E040E050E060E070E080E090E0A0E019
:108720000E942D8E01F10E94F50A9F938F937F93F3
:108730006F9384EA96E09F938F931F9287E78F93BE
:10874000C701029641E050E04C0F5D1F840F951F5A
:108750009F938F930E940F93E80EF91E0FB6F89423
:10876000DEBF0FBECDBFC557DF4F2881CB58D040ED
:10877000207430E040E050E060E070E080E090E0A5
:10878000A0E00E942D8E31F1809122248F93809160
:1087900021248F93809120248F9380911F248F9385
:1087A00082EB96E09F938F931F9287E78F93C70189
:1087B0000296A1E0B0E0AC0FBD1F8A0F9B1F9F93F4
:1087C0008F930E940F93E80EF91E0FB6F894DEBF48
:1087D0000FBECDBFC557DF4F2881CB58D040207882
:1087E00030E040E050E060E070E080E090E0A0E049
:1087F0000E942D8E41F1F8948091882890918928CB
:10880000A0918A28B0918B287894BF93AF939F93BF
:108810008F9380EC96E09F938F931F9287E78F93BF
:10882000C701029621E030E02C0F3D1F820F931FFD
:108830009F938F930E940F93E80EF91E0FB6F89442
:10884000DEBF0FBECDBF20E0C457DF4F3881CC580C
:10885000D040317040E050E060E070E080E090E0B7
:10886000A0E00E942D8E09F054C520E0C457DF4FD0
:108870003881CC58D040327040E050E060E070E089
:1088800080E090E0A0E00E942D8E09F0B5C520E0C8
:10889000C457DF4F3881CC58D040347040E050E0AE
:1088A00060E070E080E090E0A0E00E942D8E09F092
:1088B000D4C520E0C457DF4F3881CC58D040387041
:1088C00040E050E060E070E080E090E0A0E00E94D6
:1088D0002D8E09F0F1C520E0C457DF4F3881CC5808
:1088E000D040307140E050E060E070E080E090E027
:1088F000A0E00E942D8E09F052C620E0C457DF4F41
:108900003881CC58D040307240E050E060E070E0F8
:1089100080E090E0A0E00E942D8E09F070C620E07B
:1089200030E040E050E0C357DF4F6881CD58D04081
:10893000647070E080E090E0A0E00E942D8E09F06D
:108940008CC620E0C057DF4F3881C059D04040E08E
:1089500050E060E070E080E090E0A0E00E942D8EAA
:1089600009F0E8C620E0CA56DF4F3881C659D0402A
:1089700040E050E060E070E080E090E0A0E00E9425
:108980002D8E09F005C720E030E0402F417050E007
:1089900060E070E080E090E0A0E00E942D8E09F0A1
:1089A00025C720E030E0402F427050E060E070E0EA
:1089B00080E090E0A0E00E942D8E09F04AC720E000
:1089C00030E0C657DF4F4881CA58D04050E060E0E1
:1089D00070E080E090E0A0E00E942D8E09F06CC76E
:1089E00020E030E0402F487050E060E070E080E030
:1089F00090E0A0E00E942D8E09F088C720E030E0D2
:108A0000402F407150E060E070E080E090E0A0E036
:108A10000E942D8E09F0AAC720E030E0402F40725E
:108A200050E060E070E080E090E0A0E00E942D8ED9
:108A300009F0CCC720E030E0402F407450E060E007
:108A400070E080E090E0A0E00E942D8E09F0EFC77A
:108A5000F02FF078BF2E20E030E04F2F50E060E0A4
:108A600070E080E090E0A0E00E942D8E11F00C9468
:108A7000484D212F2170C22E20E030E040E05C2DD7
:108A800060E070E080E090E0A0E00E942D8E11F0A8
:108A90000C94554D20E030E04B2D50E060E070E04C
:108AA00080E090E0A0E00E942D8E11F00C94634DC8
:108AB00020E030E040E05C2D60E070E080E090E09D
:108AC000A0E00E942D8E11F00C94984D20E030E033
:108AD00040E0512F527060E070E080E090E0A0E054
:108AE0000E942D8E11F00C94CD4D20E030E040E03E
:108AF000512F547060E070E080E090E0A0E00E94B0
:108B00002D8E11F00C94004E20E030E040E0512F0B
:108B1000507160E070E080E090E0A0E00E942D8E57
:108B200011F00C94334E20E030E040E0512F5072B1
:108B300060E070E080E090E0A0E00E942D8E11F0F7
:108B40000C94724E20E030E040E0512F507460E011
:108B500070E080E090E0A0E00E942D8E11F00C9477
:108B6000B14E20E030E040E0512F587060E070E0FE
:108B700080E090E0A0E00E942D8E11F00C94F04E69
:108B800020E030E040E05D2D60E070E080E090E0CB
:108B9000A0E00E942D8E11F00C94214F779A8091C5
:108BA000C5099091C60992FD749AC557DF4F288177
:108BB000CB58D040C457DF4F3881CC58D040A801A3
:108BC000C357DF4F6881CD58D040CD56DF4F7881F5
:108BD000C359D040CC56DF4F8881C459D040CB56C2
:108BE000DF4F9881C559D040A0E08E010D5F1F4F27
:108BF0000E942D8E11F00C945D4F80915602806181
:108C000089838091E5098A83F801EE0DFF1D1082AA
:108C10008091C5099091C60987010D5F1F4F80FFA4
:108C20000CC01F930F9387E598E09F938F930E944A
:108C3000AC920F900F900F900F90B801CE0101965B
:108C40000E94B65B8091580282FF0AC028E834E295
:108C5000A801BE016F5F7F4F81E692E00E944B60EA
:108C60008091C5099091C60982FD73980E94E067C2
:108C700081EF99E00E9489528091580290915902A7
:108C8000A0915A02B0915B0290FF40C03FEFE31AFF
:108C9000F30A0E94DE68D82E89E10E94F6684091AE
:108CA00058025091590260915A0270915B0250FF34
:108CB00029C073988091E5098F5F8093E5098A83C5
:108CC000B7016F5F7F4FCE0101960E94B65B81EFC7
:108CD00099E00E94895240E050E065E880910212DC
:108CE000909103120E94445489E090E1CF56DF4FE7
:108CF000A881B981C159D0408D939C9338C0E12C93
:108D0000F12CCDCF8D2D0E94F668739A8091C20907
:108D10009091C309892B11F00E9498678091E50911
:108D20008F5F8093E5098091C5099091C60982FF04
:108D300039CC739A37CC8DED99E00E94EA56892B95
:108D4000B1F00E94E0678091580287FD2B9860E4A3
:108D500070E08DED99E00E94C35682E290E1CF561B
:108D6000DF4FE881F981C159D0409183808381E050
:108D70000C94A24FCF56DF4FA881B981C159D04082
:108D80001D921C9283E00C94A24F623181F7C09037
:108D90005802D0905902E0905A02F0905B02D1FC48
:108DA00001CCF8018081813091F50180F281E02DC4
:108DB0002081C557DF4F2883CB58D0403181C4571D
:108DC000DF4F3883CC58D040028113814481C35790
:108DD000DF4F4883CD58D0405581CD56DF4F588363
:108DE000C359D0408681CC56DF4F8883C459D040C8
:108DF0009781CB56DF4F9883C559D040208431846A
:108E0000C257DF4F19821882CE58D0406AC08230D4
:108E1000E9F4A381B481C257DF4FB983A883CE5848
:108E2000D040212C312CB1E0C557DF4FB883CB584F
:108E3000D040C457DF4F1882CC58D04000E010E833
:108E4000C357DF4F1882CD58D0403CC08330F9F073
:108E5000843009F0A7CB212C312CC257DF4F198267
:108E60001882CE58D040E5E0C557DF4FE883CB5895
:108E7000D040C457DF4F1882CC58D04000E010E0FB
:108E8000F2E0C357DF4FF883CD58D0401BC0212CF0
:108E9000312CC257DF4F19821882CE58D04025E0BE
:108EA000C557DF4F2883CB58D040C457DF4F1882B7
:108EB000CC58D04000E010E031E0C357DF4F38839A
:108EC000CD58D040CD56DF4F1882C359D040CC5634
:108ED000DF4F1882C459D040CB56DF4F1882C55996
:108EE000D04080901F2490902024A0902124B09006
:108EF0002224409080025090810260908202709003
:108F000083022DEC3CEC4CE45EE3C301B2010E9411
:108F1000B2879B01AC01C501B4010E943E8A87FD66
:108F20000BC0E894E0F8C0925802D0925902E09247
:108F30005A02F0925B024AC0A3019201C501B4013A
:108F40000E94788887FF42C080912B2490912C2426
:108F5000A0912D24B0912E240196A11DB11D8093C6
:108F60002B2490932C24A0932D24B0932E24E0FC4A
:108F700019CB6894E0F8C0925802D0925902E0925E
:108F80005A02F0925B0245E4C557DF4F4883CB5845
:108F9000D04050E2C457DF4F5883CC58D04000E057
:108FA00010E084E0C357DF4F8883CD58D040CD56C2
:108FB000DF4F1882C359D040CC56DF4F1882C459B6
:108FC000D040CB56DF4F1882C559D040902F9470B7
:108FD000C657DF4F9883CA58D04020E030E0492F71
:108FE00050E060E070E080E090E0A0E00E942D8E14
:108FF00009F08C9AC557DF4FA881CB58D040A0729A
:109000007A2E2A2F30E040E050E060E070E080E00F
:1090100090E0A0E00E942D8E11F00E94F50AC45746
:10902000DF4FB881CC58D040B074C057DF4FB88301
:10903000C059D04020E03B2F40E050E060E070E0BD
:1090400080E090E0A0E00E942D8E11F00E94CE1EE4
:10905000C457DF4FE881CC58D040E078CA56DF4F84
:10906000E883C659D04020E03E2F40E050E060E069
:1090700070E080E090E0A0E00E942D8E51F00E9410
:10908000900A6093952870939628809397289093E0
:109090009828C557DF4F2881CB58D040217030E049
:1090A00040E050E060E070E080E090E0A0E00E94EE
:1090B0002D8EF1F08EE09BE19F938F938FE696E0EB
:1090C0009F938F931F9287E78F93CE0103969F9371
:1090D0008F930E940F936C010E944F420FB6F89439
:1090E000DEBF0FBECDBF892B09F05CCA760102C07E
:1090F000E12CF12CC557DF4F2881CB58D04022708E
:1091000030E040E050E060E070E080E090E0A0E01F
:109110000E942D8ED1F1C701029667E776E041E00B
:1091200050E04C0F5D1F840F951F0E94109253E07A
:10913000E50EF11C22EAA22E28E2B22E32EFC32E57
:1091400033E0D32E47E7942ED5018D915D011F9218
:109150008F93DF92CF921F929F92C7010296E1E018
:10916000F0E0EC0FFD1F8E0F9F1F9F938F930E94C7
:109170000F93E80EF91E0FB6F894DEBF0FBECDBFF9
:109180003AEAA31638E2B306F9F6C557DF4F28814D
:10919000CB58D040247030E040E050E060E070E018
:1091A00080E090E0A0E00E942D8E09F447C0C70146
:1091B00002966BE776E041E050E04C0F5D1F840FB4
:1091C000951F0E94109254E0E50EF11C4E018AE7B3
:1091D000880E911C80E1D4011D928A95E9F728E060
:1091E000A40168E980EB0E948D115401B8E0AB0E38
:1091F000B11C82EFC82E83E0D82E97E7692EF401C8
:1092000081914F011F928F93DF92CF921F926F92A5
:10921000C701029621E030E02C0F3D1F820F931F03
:109220009F938F930E940F93E80EF91E0FB6F89448
:10923000DEBF0FBECDBF8A149B0409F7512F5078B3
:10924000D52E20E030E040E060E070E080E090E08B
:10925000A0E00E942D8EE1F48091C2099091C30993
:109260009F938F9380E896E09F938F931F9287E759
:109270008F93CE018E0D9F1D03969F938F930E9417
:109280000F93E80EF91E0FB6F894DEBF0FBECDBFE8
:1092900020E030E040E050E0C357DF4F6881CD5818
:1092A000D040617070E080E090E0A0E00E942D8EE0
:1092B00009F487C9E3E0F0E0EC0FFD1FEE0DFF1DA0
:1092C00080E28083EBE4F4E2808197012F5F3F4FDF
:1092D0007901882309F469C98081A1E0B0E0AC0F6D
:1092E000BD1FAE0DBF1D12968C933196EDCFCE01F2
:1092F0008E0D9F1D67E876E003960E94109297E01E
:10930000E90EF11CC7010E944F42892B09F04AC99E
:109310006AC92114310409F4A8CAF8944090882835
:109320005090892860908A2870908B28789480913A
:10933000781B9091791BA0917A1BB0917B1BA301A4
:109340009201281B390B4A0B5B0BCA01B9010E9421
:1093500019894B015C01B10180E090E00E941989FC
:109360009B01AC01C501B4010E947C88B82EC92EB6
:109370009F938F937F936F938BEC96E09F938F9344
:109380001F9287E78F939E012E0D3F1D2D5F3F4F4C
:109390003F932F93C856DF4F6883C859D040C956B2
:1093A000DF4F7883C759D0400E940F93E80EF91E13
:1093B000C856DF4F6881C859D040C956DF4F788101
:1093C000C759D040862F972FAB2DBC2D80939A285C
:1093D00090939B28A0939C28B0939D284092781B43
:1093E0005092791B60927A1B70927B1B0FB6F89497
:1093F000DEBF0FBECDBF39CA2114310409F447CAFC
:10940000F89480914F1B9091501BA091511BB091EB
:10941000521B78949F938F9380915F028F938091DA
:109420005E028F9388ED96E09F938F931F9287E75C
:109430008F93C7010296A1E0B0E0AC0FBD1F8A0F69
:109440009B1F9F938F930E940F93E80EF91E0FB6F8
:10945000F894DEBF0FBECDBF1ACAF89480918C2855
:1094600090918D28A0918E28B0918F287894BF93E9
:10947000AF939F938F9388EE96E09F938F931F9265
:1094800087E78F93C701029621E030E02C0F3D1F44
:10949000820F931F9F938F930E940F93E80EF91EE4
:1094A000C7010E944F420FB6F894DEBF0FBECDBF7A
:1094B000892B09F077C8FDC92114310409F40BCABE
:1094C000F89440908C2850908D2860908E28709051
:1094D0008F28789480917C1B90917D1BA0917E1B9E
:1094E000B0917F1BA3019201281B390B4A0B5B0B28
:1094F000CA01B9010E9419894B015C01B10180E0E8
:1095000090E00E9419899B01AC01C501B4010E9441
:109510007C88B82EC92E9F938F937F936F9383EF90
:1095200096E09F938F931F9287E78F939E012E0D56
:109530003F1D2D5F3F4F3F932F93C856DF4F6883EA
:10954000C859D040C956DF4F7883C759D0400E94D0
:109550000F93E80EF91EC856DF4F6881C859D040F6
:10956000C956DF4F7881C759D040862F972FAB2D32
:10957000BC2D80939E2890939F28A093A028B09301
:10958000A12840927C1B50927D1B60927E1B7092A2
:109590007F1B0FB6F894DEBF0FBECDBF9CC923283A
:1095A00009F4ABC9F8948091531B9091541BA0917E
:1095B000551BB091561B78949F938F9380915D02B9
:1095C0008F9380915C028F9380E097E09F938F93BD
:1095D0001F9287E78F93C7010296A1E0B0E0AC0F1E
:1095E000BD1F8A0F9B1F9F938F930E940F93E80EBE
:1095F000F91E0FB6F894DEBF0FBECDBF7EC98091B5
:10960000232490912424A0912524B0912624BF9353
:10961000AF939F938F9380E197E09F938F931F92D7
:1096200087E78F93C701029621E030E02C0F3D1FA2
:10963000820F931F9F938F930E940F93E80EF91E42
:10964000C7010E944F420FB6F894DEBF0FBECDBFD8
:10965000892B11F00C94D24262C980912E248F93F1
:1096600080912D248F9380912C248F9380912B2493
:109670008F9380912A248F93809129248F938091B6
:1096800028248F93809127248F938BE197E09F93D9
:109690008F931F92B7E7CB2ECF92C7010296A1E01E
:1096A000B0E0AC0FBD1F8A0F9B1F9F938F930E944A
:1096B0000F93E80EF91EC7010E944F420FB6F894AF
:1096C000DEBF0FBECDBF892B11F00C94D24280912A
:1096D0001D2090911E2090FF34C9809132248F93D9
:1096E000809131248F93809130248F9380912F2407
:1096F0008F938FE397E09F938F931F92CF92C70131
:10970000029621E030E02C0F3D1F820F931F9F93A4
:109710008F930E940F93E80EF91EC7010E944F42DB
:109720000FB6F894DEBF0FBECDBF892B11F00C949D
:10973000D24207C98091141C8F938091131C8F9380
:109740008091121C8F938091111C8F9381E597E07B
:109750009F938F931F9287E78F93C7010296A1E093
:10976000B0E0AC0FBD1F8A0F9B1F9F938F930E9489
:109770000F93E80EF91EC7010E944F420FB6F894EE
:10978000DEBF0FBECDBF892B11F00C94D242EAC8C8
:10979000809198288F93809197288F938091962815
:1097A0008F93809195288F938CE597E09F938F936B
:1097B0001F9287E78F93C701029621E030E02C0FBC
:1097C0003D1F820F931F9F938F930E940F93E80E6C
:1097D000F91EC7010E944F420FB6F894DEBF0FBEBC
:1097E000CDBF892B11F00C94D242CDC881E00E94EC
:1097F000410A209178023091790240917A02509189
:109800007B020E94FD8A9F938F937F936F9389E6DB
:1098100097E09F938F931F9287E78F93C7010296DC
:10982000A1E0B0E0AC0FBD1F8A0F9B1F9F938F93E9
:109830000E940F93E80EF91EC7010E944F420FB617
:10984000F894DEBF0FBECDBF892B11F00C94D2422D
:10985000A8C882E00E94410A2091740230917502EA
:1098600040917602509177020E94FD8A9F938F93D8
:109870007F936F9386E797E09F938F931F9287E77D
:109880008F93C701029621E030E02C0F3D1F820F1D
:10989000931F9F938F930E940F93E80EF91EC701A9
:1098A0000E944F420FB6F894DEBF0FBECDBF892B8A
:1098B00011F00C94D24283C883E00E94410A9F9326
:1098C0008F937F936F9383E897E09F938F931F927B
:1098D00087E78F93C7010296A1E0B0E0AC0FBD1FF0
:1098E0008A0F9B1F9F938F930E940F93E80EF91E80
:1098F0008C98C7010E944F420FB6F894DEBF0FBE8E
:10990000CDBF892B11F00C94D2426AC880911D20E2
:1099100087FF74C821E042E161E080ED0E947E6132
:109920009F938F937F936F9380E997E09F938F939B
:109930001F9287E78F93C701029621E030E02C0F3A
:109940003D1F820F931F9F938F930E940F93E80EEA
:10995000F91EC7010E944F420FB6F894DEBF0FBE3A
:10996000CDBF892B11F00C94D24248C880911D20A4
:1099700087FF52C821E042E162E080ED0E947E61F3
:109980009F938F937F936F938EE997E09F938F932D
:109990001F9287E78F93C7010296A1E0B0E0AC0F5A
:1099A000BD1F8A0F9B1F9F938F930E940F93E80EFA
:1099B000F91EC7010E944F420FB6F894DEBF0FBEDA
:1099C000CDBF892B11F00C94D24226C880911D2066
:1099D00087FF30C821E042E163E080ED0E947E61B4
:1099E0009F938F937F936F938CEA97E09F938F93CE
:1099F0001F9287E78F93C701029621E030E02C0F7A
:109A00003D1F820F931F9F938F930E940F93E80E29
:109A1000F91EC7010E944F420FB6F894DEBF0FBE79
:109A2000CDBF892B11F00C94D2420C941A45809131
:109A30001D2087FF0DC821E042E164E080ED0E9417
:109A40007E619F938F937F936F938AEB97E09F93B1
:109A50008F931F9287E78F93C7010296A1E0B0E032
:109A6000AC0FBD1F8A0F9B1F9F938F930E940F9374
:109A7000E80EF91EC7010E944F420FB6F894DEBFF0
:109A80000FBECDBF892B11F00C94D2420C94284507
:109A900080911D2082FD02C00C94394546E061E0B2
:109AA00083E00E9449130C94394580911D2082FD6A
:109AB00002C00C944A4521E046E061E083E00E9448
:109AC00049130C944A4580911D2082FD02C00C94DC
:109AD000584580910B1C8F9380910A1C8F93809125
:109AE000091C8F938091081C8F9388EC97E09F93BB
:109AF0008F931F9287E78F93C701029641E050E052
:109B00004C0F5D1F840F951F9F938F930E940F939F
:109B1000E80EF91EC7010E944F420FB6F894DEBF4F
:109B20000FBECDBF892B11F00C94D2420C94584536
:109B300080911D2082FD02C00C94664580910F1C0F
:109B40008F9380910E1C8F9380910D1C8F93809129
:109B50000C1C8F9380ED97E09F938F931F9287E764
:109B60008F93C7010296E1E0F0E0EC0FFD1F8E0F2E
:109B70009F1F9F938F930E940F93E80EF91EC701BA
:109B80000E944F420FB6F894DEBF0FBECDBF892BA7
:109B900011F00C94D2420C94664580911D20909156
:109BA0001E2090FD02C00C94754580E090E00E945C
:109BB000451E9F938F937F936F938BED97E09F93B9
:109BC0008F931F9287E78F93C701029641E050E081
:109BD0004C0F5D1F840F951F9F938F930E940F93CF
:109BE000E80EF91EC7010E944F420FB6F894DEBF7F
:109BF0000FBECDBF892B11F00C94D2420C94754549
:109C000080911D2090911E2090FD02C00C948445EF
:109C100081E090E00E94451E9F938F937F936F9306
:109C20008BEE97E09F938F931F9287E78F93C701E7
:109C30000296E1E0F0E0EC0FFD1F8E0F9F1F9F9357
:109C40008F930E940F93E80EF91EC7010E944F42A6
:109C50000FB6F894DEBF0FBECDBF892B11F00C9468
:109C6000D2420C94844580911D2090911E2090FD3D
:109C700002C00C94934581E090E00E94451E4B0188
:109C80005C0180E090E00E94451E9B01AC01C50193
:109C9000B4010E94461C9F938F937F936F938CEF28
:109CA00097E09F938F931F9287E78F93C701029648
:109CB00041E050E04C0F5D1F840F951F9F938F93E1
:109CC0000E940F93E80EF91EC7010E944F420FB683
:109CD000F894DEBF0FBECDBF892B11F00C94D24299
:109CE0000C94934580911D2090911E2090FD02C000
:109CF0000C94A24581E090E00E94451E4B015C015E
:109D000080E090E00E94451E9B01AC01C501B401BA
:109D10000E94A71C9F938F937F936F9387E098E097
:109D20009F938F931F9287E78F93C7010296E1E07D
:109D3000F0E0EC0FFD1F8E0F9F1F9F938F930E94EB
:109D40000F93E80EF91EC7010E944F420FB6F89418
:109D5000DEBF0FBECDBF892B11F00C94D2420C9404
:109D6000A24580911D2090911E2090FD02C00C9470
:109D7000B14581E090E00E94451E4B015C0180E00E
:109D800090E00E94451E9B01AC01C501B4010E94F8
:109D9000081D9F938F937F936F9385E198E09F9326
:109DA0008F931F9287E78F93C701029641E050E09F
:109DB0004C0F5D1F840F951F9F938F930E940F93ED
:109DC000E80EF91EC7010E944F420FB6F894DEBF9D
:109DD0000FBECDBF892B11F00C94D2420C94B1452B
:109DE00080911D2090911E2091FD02C00C94C045D1
:109DF0000E9493179F938F937F936F9388E298E0CD
:109E00009F938F931F9287E78F93C7010296E1E09C
:109E1000F0E0EC0FFD1F8E0F9F1F9F938F930E940A
:109E20000F93E80EF91EC7010E944F420FB6F89437
:109E3000DEBF0FBECDBF892B11F00C94D2420C9423
:109E4000C045C257DF4FA881B981CE58D040169681
:109E50008C9116971F928F9315968C9115971F9240
:109E60008F9313968C9113971F928F9312968C91C8
:109E70001F928F9389E398E09F938F931F9287E7B8
:109E80008F93C7010296E1E0F0E0EC0FFD1F8E0F0B
:109E90009F1F9F938F930E940F93E80EF91EC70197
:109EA0000E944F420FB6F894DEBF0FBECDBF892B84
:109EB00011F00C94D2420C94CE458091C50990913A
:109EC000C60982FD0CC08091580280FD08C081FD4A
:109ED00002C00C94FD451D9902C00C94FD451F93D2
:109EE0000F9380E598E09F938F930E94AC928091AE
:109EF00073020F900F900F900F90882311F40C9421
:109F0000FD451F928F938DED9EE09F938F930E944E
:109F1000BE920F900F900F900F900C94FD458DED19
:109F200099E00E94EA56892B11F40C94B7460E94DE
:109F300098678091580287FD02C00C94D2422B9AF8
:109F40000C94D242C856DF4F0FB6F894DEBF0FBE56
:109F5000CDBFDF91CF911F910F91FF90EF90DF90D8
:109F6000CF90BF90AF909F908F907F906F905F90B9
:109F70004F903F902F9008950C94B0524F925F9263
:109F80006F927F928F929F92AF92BF92CF92DF9209
:109F9000EF92FF920F931F93CF93DF93CDB7DEB76E
:109FA00060970FB6F894DEBF0FBECDBF6B010E9465
:109FB000DE68E82FF0E0EE0FFF1FEF5BF44E8081CC
:109FC00091810196918380838091C5099091C60902
:109FD00081FD74988090580290905902A0905A0286
:109FE000B0905B020E940A5B7C01FC018081982F8B
:109FF00092959F70913099F48F7051F48091251B48
:10A000009091261B01969093261B8093251B07C1D8
:10A01000B60182EB98E20E942652892B51F0809182
:10A02000231B9091241B01969093241B8093231B48
:10A03000F6C0D501C4011EE0B695A7959795879502
:10A040001A95D1F7F82FF1708F2E8CEF99E00E94BE
:10A0500031558C01009709F448C0B601C801029639
:10A060000E942652892BE9F1980143E859E060E00B
:10A0700074E6C8010F960E94B157F7019181F8016B
:10A080008481981321C082858F5F82878091211BF4
:10A090009091221B01969093221B8093211B84E0B8
:10A0A0000E94275CF801208530E02817390708F066
:10A0B000A9C184E00E94275CF8018087F7018081B4
:10A0C0008F70F8018187ABC0F801128684E00E948E
:10A0D000275CF8018087F70180818F70F801818704
:10A0E00092C1C8010E94D955B4CF84E092E00E9489
:10A0F000C6548C01009709F492C0B601C8010296BB
:10A100000E941D52F70181818150F801848380E013
:10A1100091E0A0E0B0E083879487A587B687128698
:10A1200084E00E94275CF8018087F70180818F70AE
:10A13000F8018187B8018CEF99E00E949155980150
:10A1400043E859E060E074E6C8010F960E94B157F9
:10A1500099249394F7018181F8018483F701808128
:10A160008F70F801878384E00E94275CF801858363
:10A1700083E00E94275C5C01F801868387818F3031
:10A1800009F0912CF7014180F8018481481A512C83
:10A19000612C712C76E0440C551C661C771C7A955A
:10A1A000D1F72385348545855685A0ECB0E00E9423
:10A1B000DB8BBB27A92F982F872F480E591E6A1EAD
:10A1C0007B1E43865486658676868091C50990916C
:10A1D000C60981FD2EC08091580280FD2AC081FDF4
:10A1E00026C08091580290915902A0915A02B091D4
:10A1F0005B0297FDD2C0992091F082E080933424D5
:10A20000109236241092352410933824009337246A
:10A2100044E354E262E184E392E00E94445480917A
:10A22000C5099091C60981FFF0C0749AEEC01D9BCC
:10A23000D8CFA4E6B0E0A30192010E94DB8B672F88
:10A24000782F892F992724E630E040E050E00E94E3
:10A25000268C7F936F93452C562C672C77245F9226
:10A260004F92BB24BF92AF92F80185811F928F93CA
:10A27000F70180818F701F928F9381811F928F933E
:10A28000F60181811F928F9380811F928F93C70166
:10A2900002969F938F9388E698E09F938F930E94F6
:10A2A000AC92809173020FB6F894DEBF0FBECDBFA3
:10A2B000882361F01F928F938AED9EE09F938F9386
:10A2C0000E94BE920F900F900F900F9080915802B5
:10A2D00090915902A0915A02B0915B0296FF2DC055
:10A2E000882059F1F7012081322F3F70832F90E0B1
:10A2F0000297D4F08FEF830F207F822B808381EF32
:10A3000099E00E94BC4F80911F1B9091201B0196E9
:10A310009093201B80931F1B8091C5099091C609C3
:10A3200096FF0BC0739809C08091251B9091261B46
:10A3300001969093261B8093251B80911D2086FFFC
:10A3400050CF0E94CD60C70105960E949960F70129
:10A3500081811F928F93F80186811F928F9385814F
:10A360001F928F938CEA98E09F938F931F9280E1C6
:10A370008F939E012F5F3F4F6901DF922F930E94C1
:10A380000F9382E00E94B360C6010E9499600FB6ED
:10A39000F894DEBF0FBECDBF24CF8EE09BE12091AD
:10A3A0000E1B222309F427CF9F938F938FEB98E006
:10A3B0009F938F93FE0131966F01DF92EF930E947E
:10A3C0004C935C01B601C70102960E9431920F9036
:10A3D0000F900F900F900F900F90009709F40BCFF4
:10A3E00095012F5F3F4F280F391FA9012F5F3F4F66
:10A3F000FA0180818032C9F362E18CE092E00E9430
:10A400004454F9CE812C912CA5CE60960FB6F894C9
:10A41000DEBF0FBECDBFDF91CF911F910F91FF9097
:10A42000EF90DF90CF90BF90AF909F908F907F90F4
:10A430006F905F904F9008950895FB012081FC017B
:10A440002083FB012181FC0121830895FC0190817F
:10A45000DB018C91981309C081E090E03181119665
:10A460002C91321721F080E0089580E090E008956B
:10A47000BC0182EB98E20C941D52DC011996ED911F
:10A48000FC911A970280F381E02D309709F009942E
:10A4900008950F931F93CF93DF9300D0CDB7DEB70E
:10A4A0008C0188E10E943A5CBC01CE0101960E94B9
:10A4B0001D52D8011996ED91FC911A970190F081E7
:10A4C000E02DBE016F5F7F4FC80109950F900F907F
:10A4D000DF91CF911F910F910895EF92FF920F930B
:10A4E0001F93CF93DF93EC018B017A0142E053E09D
:10A4F0000E949652FA86E98666E073E0C801DF9111
:10A50000CF911F910F91FF90EF900C94EF520C940C
:10A51000AE52CF93DF93EC0162EB78E288E10E94C8
:10A52000305CCE01DF91CF910C94B052EF92FF924C
:10A530000F931F93CF93DF93EC018B017A010E945D
:10A54000CB52F886EF826AE073E0C801DF91CF91C9
:10A550001F910F91FF90EF900C94EF520C94D352F7
:10A560000C945A6DDC011796ED91FC9118970190AF
:10A57000F081E02D0994DC011796ED91FC9118977C
:10A580000280F381E02D309709F00994089580E06E
:10A5900092E10C942D55FC0173836283BC0180E031
:10A5A00092E10C949155BC0180E092E10C947655B7
:10A5B000CF93DF93EC0180E092E10E943155009748
:10A5C00049F0FC01228133812C173D0729F00E94BC
:10A5D000D955F5CF80E090E0DF91CF9108950F93AA
:10A5E0001F93CF93DF938B010E94D852EC01009709
:10A5F00031F01D830C83C8010E948B6F8E83DF9125
:10A60000CF911F910F9108951F93CF93DF93EC018A
:10A61000162FEC81FD813097D1F090930312809337
:10A62000021282E08887CE0106960995992787FD58
:10A6300090950297029710F0133839F4BE01CE01BD
:10A64000DF91CF911F910C94315381E08887DF9186
:10A65000CF911F910895FC01208520FD0C94045397
:10A660000895CF92DF92EF92FF920F931F93CF93B3
:10A67000DF93EC016B01E0900212F0900312009165
:10A68000041210910512F801EC17FD0739F030970C
:10A6900009F44AC00190F081E02DF6CF209709F42B
:10A6A00043C08885882309F118860115110561F0DA
:10A6B000C017D10729F0AE0167E8C8010E942B53EB
:10A6C000F80100811181F1CFEC81FD81309769F0B3
:10A6D000CC15DD0551F0D0930312C093021240E077
:10A6E00050E063E8CE0106960995E0910412F091DE
:10A6F0000512CE17DF0769F48881998190930512BE
:10A70000809304120DC0808191818C179D0721F0E8
:10A71000FC013097C1F704C08881998191838083BF
:10A72000F0920312E0920212DF91CF911F910F91EC
:10A73000FF90EF90DF90CF9008951F93CF93DF931A
:10A7400010920E12C0910412D091051211E02097C0
:10A7500079F08985882341F01887198640E050E018
:10A7600062E8CE010E9404530990D881C02DEFCF3A
:10A77000DF91CF911F9108958091B11291E0980FD0
:10A780009093B112089560910212709103120C948B
:10A7900031538AE88093B1121092AF121092B01226
:10A7A00010920512109204121092031210920212CB
:10A7B000089580910E1281110E949D537091B012E4
:10A7C000772309F451C0E091AF122E2F30E085E0DD
:10A7D000E89FF0011124E15FFD4E608160930D124E
:10A7E0004181528150930C1240930B1283819481CA
:10A7F00090930A12809309122F5F3F4F2F713327D6
:10A800002093AF1271507093B012009731F5809180
:10A810000412909105129093081280930712809170
:10A82000071290910812892BF9F080910E12811174
:10A830000E949D5340910B1250910C1260910D1289
:10A8400080910712909108120E942B53E0910712F9
:10A85000F091081280819181DECF613819F421E0F6
:10A86000FC0120870E942B5380910E122091B01280
:10A8700090E0820F911D089580910E122091B012E8
:10A8800090E0820F911D08952091B0122032B9F00E
:10A89000E091AF12E20FEF71E093061235E0E39F13
:10A8A000F0011124E15FFD4E608352834183948364
:10A8B00083832F5F2093B01280E090E0089581E0C1
:10A8C00090E00895CF93DF93C0910212D0910312CC
:10A8D0000E942B53D0930312C0930212DF91CF91A9
:10A8E0000895AB013091041220910512E32FF22F4D
:10A8F000E817F907B1F0309721F00190F081E02DD1
:10A90000F7CF009771F0FC013083218390930512FB
:10A910008093041221E020871782168261E80C944C
:10A9200062540895009749F0FC012085215022309F
:10A9300020F421E0218720930E12089521E030E0D9
:10A94000FC018085811102C020E030E0C90108953A
:10A95000CF93DF93EC014A815B8160E070E08C81F2
:10A960009D810E9400922A813B8188819981289F44
:10A97000A001299F500D389F500D112460E070E018
:10A980008E819F81DF91CF910C940092FC01828196
:10A99000938120E030E028173907D1F0A481B581F8
:10A9A000A20FB31F4C91411110C081E08C938081A4
:10A9B0009181289FA001299F500D389F500D11248F
:10A9C00086819781840F951F08952F5F3F4FE3CFB6
:10A9D00080E090E00895FC01268137814281538117
:10A9E00080E090E084179507C9F02617370781F4B7
:10A9F000A481B581A80FB91F2C91121614F421500F
:10AA00002C930480F581E02DE80FF91F80810895D3
:10AA1000A081B1812A0F3B1F0196E4CF8FEF0895EB
:10AA2000FC018681978168177907A0F0A081B18128
:10AA300042815381A49F9001A59F300DB49F300D9A
:10AA40001124280F391F81E090E06217730720F06E
:10AA500080E0089580E090E00895FC01118210826A
:10AA60000895FC01808191810895FB01208131814D
:10AA7000FC01318320830895DC01ED91FC91309736
:10AA800031F080819181009729F0FC01FACF80E0BC
:10AA900090E00895CF010895DC01ED91FC911197AC
:10AAA0003097A9F020813181232B21F41D921C9233
:10AAB000CF010895A081B1818D919C911197892B2F
:10AAC00011F0FD01F7CF11821082CD01089580E0D1
:10AAD00090E00895DC01ED91FC911197309721F001
:10AAE000208131812D933C93CF010895DC01ED91BC
:10AAF000FC913097A9F0A0E0B0E020813181E61709
:10AB0000F70741F4109709F4DC012D933C9311826F
:10AB1000108208952115310519F0DF01F901EDCFFB
:10AB200008950F931F93CF93DF938C01EB010E9445
:10AB3000765519821882C8010E943C55009711F47D
:10AB4000F80101C0FC01D183C083DF91CF911F9137
:10AB50000F9108950F931F93CF93DF93EC018B0117
:10AB60000E94765588819981F801918380831983A9
:10AB70000883DF91CF911F910F910895DC01ED9132
:10AB8000FC9180E090E0309729F001960190F081EF
:10AB9000E02DF9CF0895FB01309719F4BA010C9418
:10ABA000AA5580819181DA018D939C9351834083D2
:10ABB0000895009721F0FC0180819181089580E043
:10ABC00090E008958091B4129091B512892B29F4E8
:10ABD0001092B3121092B21208950E94E564E091AF
:10ABE000B412F091B5122281338140815181240F3A
:10ABF000351F281B390B0480F581E02D309769F053
:10AC00004281538160817181460F571F481B590B48
:10AC10004217530780F79A01EECF280F391F309360
:10AC2000B3122093B212089586E892E00C949254E5
:10AC3000EF92FF920F931F93CF93DF938C01FC0150
:10AC400080819181009799F08A359105D9F0F801BA
:10AC50001182108283E068C08681978184179507EE
:10AC600009F049C00480F581E02D3097A9F71092D2
:10AC7000B5121092B4128AE590E0F80191838083B6
:10AC800081E052C0673891F16238A9F7C091B412DF
:10AC9000D091B512E12CF12C209769F3CE010E94DE
:10ACA0005C73892BF1F0AE0168E88E819F810E9470
:10ACB0004454892BA1F41F821E828C819D81E11452
:10ACC000F10421F0F7019583848304C09093B512B9
:10ACD0008093B4121D821C820E94E255D7CF0E943D
:10ACE00014567E010C80DD81C02DD6CFE091B412C8
:10ACF000F091B512BACFF093B512E093B412A481DB
:10AD0000B581109709F4B7CF16968D919C9117973E
:10AD10008417950711F0FD01F2CF14968D919C9147
:10AD2000159795838483EBCFDF91CF911F910F917E
:10AD3000FF90EF900895CF93DF93EC010E9414569B
:10AD40008E819F813091B4122091B512892B59F0D8
:10AD5000E32FF22F309739F0EC17FD0781F00480D4
:10AD6000F581E02DF7CF80910212909103129F831D
:10AD70008E833C832D83D093B512C093B412DF91A0
:10AD8000CF910C94E255CF93DF93EC010E943C737A
:10AD9000CE01DF91CF910C949B56CF93DF93EC01C2
:10ADA0000E944873CE01DF91CF910C949B56CF93B4
:10ADB000DF93EC010E945273CE01DF91CF910C948E
:10ADC0009B56FC0120813181260F371F3183208360
:10ADD0000C94E25521E030E0FC0186819781892BBB
:10ADE00011F020E030E0C9010895FC012281338197
:10ADF00080819181820F931F0895FC018081918150
:10AE0000089581E090E02091B4123091B512232B87
:10AE100011F480E090E008958091B4129091B51201
:10AE2000892B29F08091B2129091B312089580E09D
:10AE300090E00895CF93DF93EC01E091B412F0918C
:10AE4000B5128E179F0769F48C819D819093B5127E
:10AE50008093B4120DC0848195818C179D0721F0D9
:10AE6000FC013097C1F706C08C819D819583848356
:10AE70000E94E2551D821C821F821E82DF91CF91AB
:10AE80000895EF92FF920F931F93CF93DF938C015E
:10AE90007A01FC0180819181009741F08B3491050A
:10AEA00001F1F8011182108283E048C087EB92E142
:10AEB0000E943155EC01209751F06C817D81CE01CB
:10AEC00002960E94C3560990D881C02DF4CF81E02C
:10AED0008093B6128BE490E0F8019183808381E047
:10AEE0002DC06838E1F787EB92E10E943155EC0103
:10AEF000209781F3CE010296E816F906D9F4BE0137
:10AF000087EB92E10E947655E0900212F0900312D6
:10AF10008A859B859093031280930212EC85FD85B0
:10AF2000309719F08E859F850995F0920312E09273
:10AF30000212D0CF0990D881C02DDACFDF91CF9106
:10AF40001F910F91FF90EF9008951092B61287EB2A
:10AF500092E10E942D5560E070E080E992E00C944F
:10AF600071540F931F93CF93DF93EC010091021262
:10AF7000109103121B870A875D874C873F872E87B6
:10AF80008091B612882379F080E992E090930312C1
:10AF900080930212CE0102960E94C35610930312B0
:10AFA0000093021202C07D836C83BE0187EB92E1A5
:10AFB0000E947655BE0187EB92E1DF91CF911F9100
:10AFC0000F910C9491550F931F93CF93DF93EC0146
:10AFD0008091B612882391F0009102121091031211
:10AFE00080E992E09093031280930212CE010296C0
:10AFF0000E94CD561093031200930212BE0187EBFC
:10B0000092E10E947655BE0187EB92E1DF91CF91EC
:10B010001F910F910C9491550F931F93CF93DF9332
:10B02000EC018091B612882391F0009102121091E8
:10B03000031280E992E09093031280930212CE01F2
:10B0400002960E94D7561093031200930212BE017B
:10B0500087EB92E10E947655BE0187EB92E1DF918A
:10B06000CF911F910F910C949155CF93DF93EC01E9
:10B070008091B612882329F0CE0102960E941A57B9
:10B0800004C01F821E8219861886BE0187EB92E1DA
:10B09000DF91CF910C947655CF93DF93EC018091A3
:10B0A000B612882331F0CE010296DF91CF910C9435
:10B0B000EA5687EB92E10E943155009739F08C17E0
:10B0C0009D0739F0FC0180819181F7CF81E090E00C
:10B0D00002C080E090E0DF91CF9108952F923F92DF
:10B0E0004F925F926F927F928F929F92AF92BF9298
:10B0F000CF92DF92EF92FF920F931F93CF93DF9344
:10B10000CDB7DEB7E8970FB6F894DEBF0FBECDBF60
:10B11000E9EEFAE22081318142815381E5EEFAE2E3
:10B120005080418032802380E1EEFAE28081898381
:10B1300091819A83A281AB836380EDEDFAE2B081C5
:10B14000BC8381818D8392819E83A381AF83E9ED4E
:10B15000FAE2B081B8878181898792819A87A38139
:10B16000AB87E5EDFAE2B081BC8781818D87928162
:10B170009E87A381AF87E1EDFAE2B081B88B818130
:10B18000898B92819A8BA381AB8BEDECFAE2B08133
:10B19000BC8B81818D8B92819E8BA381AF8BE9ECDF
:10B1A000FAE2B081B88F8181898F92819A8FA381D1
:10B1B000AB8FE5ECFAE2B081BC8F81818D8F9281FB
:10B1C0009E8FA381AF8FE1ECFAE2B081B8A38181B9
:10B1D00089A392819AA3A381ABA3EDEBFAE2B0819C
:10B1E000BCA381818DA392819EA3A381AFA3E9EB30
:10B1F000FAE2B081B8A7818189A792819AA7A38139
:10B20000ABA7E5EBFAE2B081BCA781818DA7928163
:10B210009EA7A381AFA7E1EBFAE2B081B8AB818131
:10B2200089AB92819AAB7380EDEAFAE2B080A1809B
:10B2300092808380E9EAFAE2F080E180D280C380E4
:10B24000E5EAFAE2A081AFABB181B8AF1281038128
:10B250002BAB3CAB4DAB5EAB0E9413655EA95F931D
:10B260004DA94F933CA93F932BA92F932F923F9227
:10B270004F925F926F922B812F932A812F93298176
:10B280002F932F812F932E812F932D812F932C81FC
:10B290002F932B852F932A852F9329852F932885EC
:10B2A0002F932F852F932E852F932D852F932C85CC
:10B2B0002F932B892F932A892F9329892F932889BC
:10B2C0002F932F892F932E892F932D892F932C899C
:10B2D0002F932B8D2F932A8D2F93298D2F93288D8C
:10B2E0002F932F8D2F932E8D2F932D8D2F932C8D6C
:10B2F0002F932BA12F932AA12F9329A12F9328A11C
:10B300002F932FA12F932EA12F932DA12F932CA1FB
:10B310002F932BA52F932AA52F9329A52F9328A5EB
:10B320002F932FA52F932EA52F932DA52F932CA5CB
:10B330002F937F922AA92F9329A92F9328A92F937E
:10B340008F929F92AF92BF92CF92DF92EF92FF9235
:10B350000F931F9328AD2F932FA92F939F938F9314
:10B360007F936F93A3EBB8E28C911F928F93E2EBE4
:10B37000F8E280811F928F9385E59FE09F938F93E2
:10B380000E94BE92E9E1FBE220813181428153813A
:10B39000E5E1FBE25080418032802380E9E0FBE27E
:10B3A0009080818072806380E5E0FBE28081898308
:10B3B00091819A83A281AB83B381BC83E1E0FBE2FC
:10B3C00080818D8391819E83A281AF83B381B88771
:10B3D000EDEFFAE28081898791819A87A281AB871C
:10B3E000B381BC87E9EFFAE280818D8791819E87E6
:10B3F000A281AF87B381B88BE5EFFAE28081898BB8
:10B4000091819A8BB280A380E1EFFAE2F080E18033
:10B41000D280C380EDEEFAE2A081AB8BB181BC8B10
:10B42000128103810FB6F894DEBF0FBECDBF2BABE8
:10B430003CAB4DAB5EAB0E9413655EA95F934DA91B
:10B440004F933CA93F932BA92F932F923F924F925A
:10B450005F926F927F928F929F922C812F932B817C
:10B460002F932A812F9329812F9328852F932F8122
:10B470002F932E812F932D812F932C852F932B8506
:10B480002F932A852F9329852F9328892F932F85F2
:10B490002F932E852F932D852F93AF92BF922A89BC
:10B4A0002F9329892F93CF92DF92EF92FF920F93E0
:10B4B0001F932C892F932B892F939F938F937F9387
:10B4C0006F93A3EBB8E28C911F928F93E2EBF8E2BB
:10B4D00080811F928F9386EE9EE09F938F930E94B0
:10B4E000BE920FB6F894DEBF0FBECDBFE8960FB682
:10B4F000F894DEBF0FBECDBFDF91CF911F910F91AA
:10B50000FF90EF90DF90CF90BF90AF909F908F9083
:10B510007F906F905F904F903F902F90089580E3C1
:10B5200080936D130895CF93DF9360916D1370E056
:10B53000C0E3D0E0C61BD70B65547D4EAE010E9420
:10B54000F791CE01DF91CF910895CF92DF92EF92E4
:10B55000FF920F931F93CF93DF937C01C0907013E2
:10B56000D090711360916D1370E0E601E096C61BF8
:10B57000D70BC138D105D8F400E310E0061B170B38
:10B5800065547D4EA8010E94F7916091B9127091A7
:10B59000BA1280916E1390916F13680F791FA601F4
:10B5A000C701800F911F0E94F791CE0102C080E079
:10B5B00090E0DF91CF911F910F91FF90EF90DF907E
:10B5C000CF90089590916D13980F90936D130895F7
:10B5D00040917013509171134817590798F02091BA
:10B5E0006E1330916F13280F391F30936F13209310
:10B5F0006E13481B590B509371134093701381E0E5
:10B6000090E0089580E090E0089590937113809306
:10B610007013089580916E1390916F1385519D4E14
:10B62000089580916D1390E085549D4E089581E0BA
:10B6300090E02091B9123091BA122B5E324111F490
:10B6400080E090E008950E94175B892B61F0609183
:10B65000B9127091BA1240917013509171138BEE20
:10B6600092E10C94F79120916E1330916F13211594
:10B670003105B9F08091701390917113C096EBEE83
:10B68000F2E1AF014B5B52414817590734F4DF0137
:10B69000A20FB31F4C914193F4CF10926F131092ED
:10B6A0006E1308958091B9129091BA120895809105
:10B6B000701390917113089590916D1380E3891B1D
:10B6C000089520E380916D13281B80917013909151
:10B6D0007113820F911D08951F93CF93DF93EC0197
:10B6E00010916D13812F90E08C179D076CF00E94D4
:10B6F000615B8C0F9D1F8138910530F41C1B1093EA
:10B700006D1381E090E002C080E090E0DF91CF9186
:10B710001F910895CF93DF93ECEBF8E21192119211
:10B7200088E2EC3EF807D1F7C4EBD8E260E073E0C2
:10B73000CE010E941D52229688E2CC3BD807B1F779
:10B74000DF91CF91089510926F1310926E131092A3
:10B7500071131092701380E380936D138BEE92E15E
:10B760009093BA128093B9120C948A5BEF92FF9275
:10B770000F931F93CF93DF9300D0CDB7DEB78C012B
:10B7800069837A830E94A35B6981E62E7A81F72E12
:10B7900081E8E816F10418F080E8E82EF12CA70102
:10B7A000B8018091B9129091BA120E94F791F0926B
:10B7B0007113E0927013C7010F900F90DF91CF913A
:10B7C0001F910F91FF90EF9008950F931F93CF93C8
:10B7D000DF938C01EB010E94A35B1093BA120093DC
:10B7E000B912D0937113C0937013DF91CF911F9151
:10B7F0000F91089520E3ECEBF8E2DC0101900D924B
:10B800002A95E1F788E0E4EBF8E2DB0101900D9284
:10B810008A95E1F7089520E3FC01ACEBB8E20190D2
:10B820000D922A95E1F788E0FB01A4EBB8E20190C4
:10B830000D928A95E1F70895E82FF0E0EE0FFF1FD3
:10B84000E454F74D7183608381E090E00895E82F20
:10B85000F0E0EE0FFF1FE454F74D808191810895D1
:10B8600090E0880F991F8C57974D0E941D5281E0E0
:10B8700090E0089590E0880F991F8C57974D089598
:10B880008115910511F00197F1F70895E091EF28E6
:10B89000F091F02890818091EE2889230895E0911D
:10B8A000EC28F091ED2880819091EE28892B8083FF
:10B8B000E091F128F091F22880819091EE28892B77
:10B8C00080830895E091EC28F091ED28908180919B
:10B8D000EE28809589238083E091F128F091F22869
:10B8E00090818091EE2880958923808308951F930D
:10B8F000CF93DF93E091EC28F091ED289081809137
:10B90000EE28809589238083E091F128F091F22838
:10B9100080819091EE28892B80838FEB93E00E94A9
:10B92000405C1FB7F894E091F128F091F2289081E3
:10B930008091EE2880958923808383E890E00E949F
:10B94000405CE091EF28F091F028D081C091EE2882
:10B950001FBF78948BE393E00E94405CE091EF2856
:10B96000F091F02890818091EE28982319F08D2F86
:10B970008C2301C081E0DF91CF911F9108955093F6
:10B98000F2284093F1287093ED286093EC2890936F
:10B99000F0288093EF2881E001C0880F2A95EAF70C
:10B9A0008093EE280C94775CCF93DF93C82FDFB79A
:10B9B000F894E091F128F091F22880819091EE289E
:10B9C000892B808383E090E00E94405CCC2351F07F
:10B9D000E091F128F091F22880819091EE289095E5
:10B9E0009823908387E190E00E94405CE091EF28EB
:10B9F000F091F02880819091EE28892309F4C0E02D
:10BA000089E590E00E94405CE091F128F091F228F5
:10BA100080819091EE28909598239083DFBF8BE3EF
:10BA200090E00E94405C8C2FDF91CF910895CF93DE
:10BA3000DF93C82FD8E08C2F81700E94D45CC6950C
:10BA40008111C068D150B9F78C2FDF91CF91089543
:10BA50008FEF0C94175DDF92EF92FF920F931F937D
:10BA6000CF93DF93E82EEB010E94775C81112FC00A
:10BA700080EF0E94175DF12C10E488EFD82ED10ED4
:10BA800081E00E94D45C082F81E00E94D45C88236E
:10BA900019F0002361F01DC0011109C01E1528F026
:10BAA000888180FF04C0E11611F0F12E01E0802FA3
:10BAB0000E94D45C988196950111906898831150EA
:10BAC0001D11DECF21961111D8CF8F2D03C08FEF1E
:10BAD00001C08EEFDF91CF911F910F91FF90EF90FA
:10BAE000DF900895FF920F931F93CF93DF93F82E6B
:10BAF000EB010E94775C209769F085E50E94175D55
:10BB00008E01085F1F4F89910E94175DC017D107F2
:10BB1000D1F703C08CEC0E94175D8F2DDF91CF9180
:10BB20001F910F91FF900C94175D0F931F93CF936C
:10BB3000DF93DB01EC9111969C911197F0E0F92BCA
:10BB4000803181F4BF016E7FE3E0660F771FEA95D5
:10BB5000E1F716969C911697ECE0F0E0E91BF109ED
:10BB6000E60FF71FF7FF07C091E0EA019883F19510
:10BB7000E195F10902C0EA011882883279F414963D
:10BB80008C91982F9076903649F086FF02C0EE7F18
:10BB900005C085FF02C0EC7F01C0E87FCF0144E013
:10BBA000969587954A95E1F7D9018C93EF70E80156
:10BBB000E88380E0DF91CF911F910F9108950F935B
:10BBC0001F93CF93DF93EC018B01B80188810E9412
:10BBD0002B5D888381508D3F30F4F801808188325D
:10BBE00011F0803191F7DF91CF911F910F9108955E
:10BBF000CF93DF93EC010E94775CBE0184EB0E943F
:10BC0000725D81E00E94D45CC82F0E94775C81E065
:10BC1000C11101C080E0DF91CF9108951F93CF93B0
:10BC2000DF9300D0CDB7DEB7182F69837A830E94E7
:10BC3000775C0E94465C69817A81882341F084E4C4
:10BC40000E94725D113029F00E944F5C02C082E0B8
:10BC500001C080E00F900F90DF91CF911F91089568
:10BC60004F925F926F927F928F929F92AF92BF920C
:10BC7000CF92DF92EF92FF920F931F93CF93DF93B8
:10BC8000CDB7DEB729970FB6F894DEBF0FBECDBF94
:10BC90006C015B014A0189010E94775CB6018EEB61
:10BCA0000E94725DCE0101967C013E019AE0690E10
:10BCB000711C27010E94285DF70181937F01E61521
:10BCC000F705C1F769E070E0C2010E94CD778111EC
:10BCD00009C09401A501B201F60180810E94955D21
:10BCE00080E001C083E029960FB6F894DEBF0FBE56
:10BCF000CDBFDF91CF911F910F91FF90EF90DF901B
:10BD0000CF90BF90AF909F908F907F906F905F90FB
:10BD10004F9008955F926F927F928F929F92AF9211
:10BD2000BF92CF92DF92EF92FF920F931F93CF9328
:10BD3000DF93CDB7DEB729970FB6F894DEBF0FBEFD
:10BD4000CDBF582E6B015A01890160E070E08EEB87
:10BD50000E94725DCE0101967C014E019AE0890E2F
:10BD6000911C37010E94285DF70181937F01E8153E
:10BD7000F905C1F769E070E0C3010E94CD77811138
:10BD800008C09501A601B301852D0E94955D80E054
:10BD900001C083E029960FB6F894DEBF0FBECDBF79
:10BDA000DF91CF911F910F91FF90EF90DF90CF9097
:10BDB000BF90AF909F908F907F906F905F9008950D
:10BDC0000F931F93CF93DF93CDB7DEB728970FB6AE
:10BDD000F894DEBF0FBECDBF182F062F98E0ECE021
:10BDE000F3E0DE01119601900D929A95E1F7242F70
:10BDF000332727FD309541E752E0249FC001259F5E
:10BE0000900D349F900D112464E670E00E94128C16
:10BE1000CB0144E6049F800D911D1124FE01319653
:10BE2000AE01475F5F4F619170E02617370711F44D
:10BE3000019603C0E417F507B1F7112319F09195A6
:10BE40008195910928960FB6F894DEBF0FBECDBF3D
:10BE5000DF91CF911F910F910895EF92FF920F9371
:10BE60001F93CF93DF93CDB7DEB72B970FB6F89420
:10BE7000DEBF0FBECDBFF82EE92E682F792F88E0E8
:10BE80008F0D0E940E5E882319F084E391E243C077
:10BE900066E471E48FE090E00E94985F8E01075F96
:10BEA0001F4F9801AE01465F5F4FBE01655F7F4F38
:10BEB0008F2D9E2D0E94305E8111E7CF88E0ECE04F
:10BEC000F3E0DE01119601900D928A95E1F7498524
:10BED00021E732E0429FC001439F900D112464E6A8
:10BEE00070E00E94128C8A8594E6899F600D711D16
:10BEF0001124FE0131968191481303C06F5F7F4F7B
:10BF000003C0E017F107B9F78B85882319F0719505
:10BF100061957109CB012B960FB6F894DEBF0FBE69
:10BF2000CDBFDF91CF911F910F91FF90EF900895BA
:10BF3000DC01CB0181159105A105B10529F08150E6
:10BF40009040A040B040D9F708959B01AC011092F9
:10BF5000B90060E072E18AE790E00E94268C2051EF
:10BF600031094109510956954795379527952093F1
:10BF7000B800089594EA9093BC0040EA56E861E066
:10BF800070E09091BC0097FD0BC0415051096109D0
:10BF90007109411551056105710599F781E0089511
:10BFA0009091B900987F983011F09031B9F7809353
:10BFB000BB0084E88093BC0080EA96E8A1E0B0E092
:10BFC0002091BC0027FD08C00197A109B109009785
:10BFD000A105B105A9F7E2CF8091B900887F88312A
:10BFE00011F08034D9F680E0089524EA34E844E979
:10BFF0002093BC009091BC0097FFFCCF9091B900BA
:10C00000987F983011F0903199F78093BB0030936E
:10C01000BC009091BC0097FFFCCF9091B900987F35
:10C02000903211F0983539F44093BC009091BC00E7
:10C0300094FDFCCFDDCF08950C94BA5F84E9809322
:10C04000BC008091BC0084FDFCCF08958093BB00B0
:10C0500084E88093BC008091BC0087FFFCCF909166
:10C06000B900987F81E0983209F480E0089584EC6B
:10C070008093BC008091BC0087FFFCCF8091BB0007
:10C08000089584E88093BC008091BC0087FFFCCFBA
:10C090008091BB000895E0E1DC01FD91CD01F093BA
:10C0A0003F01E150C9F780913C018F7D80933C01B5
:10C0B00080913C01877F80933C01FB0180E191915D
:10C0C00090933E018150D9F780913C018068809324
:10C0D0003C0180913D0180FFFCCF4051510980918E
:10C0E0003C01806280933C0180913C01877F80937A
:10C0F0003C01141615069CF4FB0180E1919190938C
:10C100003E018150D9F780913C01806880933C01C9
:10C1100080913D0180FFFCCF40515109EACFF901E8
:10C1200080E190913E0191938150D9F781E090E0B8
:10C1300008950F931F93CF93DF93EC018CE70E9438
:10C14000F55F8CE70E9426608E01005F1F4F89918A
:10C150000E942660C017D107D1F7DF91CF911F91C0
:10C160000F910C941E60813019F440E050E002C041
:10C1700040EC50E060E070E08CE790E00C947611C9
:10C18000813019F44EE050E002C048E050E060E039
:10C1900070E08CE790E00C94761141E050E060E0B4
:10C1A00070E08CE790E00E9476116AE67AE080E029
:10C1B00090E00C94985F48E350E060E070E08CE71A
:10C1C00090E00E94761149E350E060E070E08CE777
:10C1D00090E00E94761144E150E060E070E08CE76E
:10C1E00090E00E94761148E750E060E070E08CE754
:10C1F00090E00E9476114EE550E060E070E08CE740
:10C2000090E00E9476114DE650E060E070E08CE72F
:10C2100090E00E9476116CE17AE186E090E00E9465
:10C22000985F4CE050E060E070E08CE790E00E94A6
:10C23000761141E050E060E070E08CE790E00E9411
:10C24000761146E050E060E070E08CE790E00E94FC
:10C2500076116AE67AE080E090E00C94985FCF93E4
:10C26000DF93CDB7DEB7A2970FB6F894DEBF0FBE4F
:10C27000CDBF81E1E0E4F9E0DE01529601900D923C
:10C280008A95E1F781E1E1E5F9E0DE01119601909F
:10C290000D928A95E1F70E94DB60CE0142960E94E2
:10C2A000996082E00E94B3606AE67AE080E090E004
:10C2B0000E94985FCE0101960E94996060E17EEA3B
:10C2C00088E290E00E94985F80E00E94C06060E198
:10C2D0007EEA88E290E00E94985F4EE050E060E0E5
:10C2E00070E08CE790E00E947611A2960FB6F89469
:10C2F000DEBF0FBECDBFDF91CF910895CF92DF9209
:10C30000EF92FF920F931F93CF93DF9300D01F9272
:10C31000CDB7DEB7F82E042F122F213031F02230A6
:10C3200031F0243031F0283031F090E005C091E058
:10C3300003C092E001C093E00C3059F00E3011F4CC
:10C34000946007C0003111F4986003C0023109F411
:10C350009C60613059F0623011F4906207C0633024
:10C3600011F4906403C0643009F490669068692FFA
:10C3700070E023E030E0AE014F5F5F4F8F2D90E023
:10C380000E948D1169E07AE180E090E00E94985F60
:10C390008F2D8160F82E0E94BA5F0E9437608983DA
:10C3A0000E9437608A83023119F40E9437608B83C0
:10C3B0000E94376087FDF1CF0E9441600E941E609D
:10C3C00069E07AE180E090E00E94985F8F2D0E9402
:10C3D000BA5F0E94376089830E9437608A83023186
:10C3E00019F40E9441608B830E9441600E941E608C
:10C3F00039812A81023149F5832F90E0A0E0B0E035
:10C400004B817727662731FF0EC030E0322F22277D
:10C41000620F731F811D911D640F711D811D911D80
:10C420008C6F9F6F0BC030E0322F2227620F731F7B
:10C43000811D911D640F711D811D911D0E941B891D
:10C4400020E83FEF4FEF57E420C0632F70E0762FD6
:10C450006627620F711D882777FD8095982F0E94AF
:10C460001B890C3029F420E030EE4FEF54E40DC06E
:10C470000E3029F420E038EF4FEF55E406C00031CC
:10C4800031F420E03EEF4FEF56E40E947C882FE627
:10C4900032E143E050E40E94FD8A6B017C01612F90
:10C4A00070E080E090E00E941B899B01AC01C70115
:10C4B000B6010E947C880F900F900F90DF91CF9172
:10C4C0001F910F91FF90EF90DF90CF900895E6E4D9
:10C4D000F1E08081208190813081829586958695DA
:10C4E000837022952F70822B832B92959F70892BBE
:10C4F00008950F931F93CF93DF9300D0CDB7DEB78E
:10C5000046E06CE080E00E94A96589E18093C40068
:10C510001092C50082E08093C00080E00E943466E3
:10C520000E94D56484B784B784B784B784B7E3E73F
:10C53000F1E322E432E4318320833A968DB79EB74B
:10C540000A97E817F907B8F382E699E09F938F936B
:10C5500082EA90E19F938F930E94BE920E94107492
:10C560000E94C95360E070E086E892E00E94715436
:10C570000E94A557E0911403F091150309950E94BC
:10C58000676290E00E944C74CE0101960E940A649A
:10C590000F900F900F900F90882341F082E890E168
:10C5A0009F938F930E94BE920F900F90CE010196A1
:10C5B0000E9438520E9418648C010E941464AE01DB
:10C5C0004F5F5F4FB8010E9400690E9484630E9420
:10C5D000E1680E941C640E943A6A85E790E19F939B
:10C5E0008F930E94BE928A811F928F9301E710E180
:10C5F0001F930F930E94BE9289811F928F931F9366
:10C600000F930E94BE928FE690E19F938F930E94BA
:10C61000BE920E945074E0915103F091520309952B
:10C62000E0914303F09144030995E0912A03F091CE
:10C630002B0309950E94416A182F0E94DE681F9201
:10C640001F931F928F93809150038F9380914F037C
:10C650008F93809142038F93809141038F9384E560
:10C6600090E19F938F930E94BE92E0915B03F091C3
:10C670005C030FB6F894DEBF0FBECDBF309791F0CC
:10C680000995BC0180E890E00E94FE8B7F936F9338
:10C6900081E490E19F938F930E94BE920F900F9040
:10C6A0000F900F908FE390E19F938F930E94BE9223
:10C6B00060E070E08CED92E00E94715480EF92E0B7
:10C6C0000E94207387E390E19F938F930E94BE9214
:10C6D0000F900F900F900F900F900F90DF91CF91D0
:10C6E0001F910F9108957F936F939F938F9381E391
:10C6F00090E19F938F930E94BE920F900F900F90A6
:10C700000F900F900F9008951F93CF93DF93CDB7A5
:10C71000DEB7A0970FB6F894DEBF0FBECDBF8DE594
:10C7200090E00E942A94182F282F35EF380F3031CF
:10C7300008F0982F9095291709F461C08DEB90E1CE
:10C740009F938F930E94BE92E2E0F1E10F900F90D1
:10C75000DE01119684918D93319681E1EA30F807DC
:10C76000C9F7F89448E050E069E770E0CE0101961F
:10C770000E943094E4EFF0E1DE01119684918D93F4
:10C78000319681E1E230F807C9F74EE050E06BE600
:10C7900070E0CE0101960E943094EAEEF0E1DE01F5
:10C7A000119684918D93319680E1E43FF807C9F7A3
:10C7B0004AE050E061E670E0CE0101960E943094BC
:10C7C0006DEC7BEA8BE590E00E94489460E070E0BD
:10C7D00089E590E00E94489460E088E590E00E943E
:10C7E0003A9460E070E08FE590E00E9448941AE18E
:10C7F0006AE175EE8DE590E00E9448947894812F6F
:10C80000A0960FB6F894DEBF0FBECDBFDF91CF91DB
:10C810001F910895F89442E050E069E770E00E94AB
:10C820001294789480E008958BE590E00C942A941B
:10C8300089E590E00C942A9488E590E00C94229489
:10C840004091012950910229609103297091042996
:10C8500090E0A0E0B0E0480F591F6A1F7B1F409393
:10C860000129509302296093032970930429409170
:10C87000FD285091FE286091FF2870910029480FF3
:10C88000591F6A1F7B1F4093FD285093FE28609319
:10C89000FF28709300292091A12A2223A1F0409122
:10C8A000F9285091FA286091FB287091FC28480FD4
:10C8B000591F6A1F7B1F4093F9285093FA286093F1
:10C8C000FB287093FC2808951F920F920FB60F92C9
:10C8D00011240BB60F922F933F934F935F936F9357
:10C8E0007F938F939F93AF93BF93EF93FF93809129
:10C8F000741390917513019690937513809374132C
:10C90000809173138F5F809373138038A9F4109212
:10C9100073138091012990910229A0910329B0916C
:10C9200004290196A11DB11D80930129909302292C
:10C93000A0930329B09304298091A12A8823E1F0D0
:10C94000809172138F5F809372138038A9F41092D4
:10C9500072138091F9289091FA28A091FB28B09148
:10C96000FC280196A11DB11D8093F9289093FA2807
:10C97000A093FB28B093FC280E940157892B11F04B
:10C980000E941456FF91EF91BF91AF919F918F91AB
:10C990007F916F915F914F913F912F910F900BBEBF
:10C9A0000F900FBE0F901F901895F8941092B6003C
:10C9B00016BC83EF87BD82E084BD94E095BD95B33E
:10C9C00095BB80936E007894089580917413909134
:10C9D0007513209174133091751382179307A9F77B
:10C9E0000895009751F022E330E000002150310912
:10C9F00021153105D1F70197F4CF08950F931F93B7
:10CA0000CF93DF93EC010E94E5648C010E94E56402
:10CA1000801B910B8C179D07C8F3DF91CF911F915D
:10CA20000F91089508950F931F93609101297091BC
:10CA300002298091032990910429009101291091E4
:10CA40000229209103293091042960177107820778
:10CA5000930759F71F910F9108951F920F920FB6E8
:10CA60000F9211241092B2020F900FBE0F901F90E0
:10CA700018951F920F920FB60F9211240BB60F92BA
:10CA80002F933F934F935F936F937F938F939F93D6
:10CA9000AF93BF93EF93FF93E091A802F091A902A7
:10CAA0008081E091B302F091B402309709F00995CA
:10CAB000FF91EF91BF91AF919F918F917F916F9176
:10CAC0005F914F913F912F910F900BBE0F900FBE32
:10CAD0000F901F9018951F920F920FB60F9211246E
:10CAE0001092BF020F900FBE0F901F9018951F92CB
:10CAF0000F920FB60F9211240BB60F922F933F9304
:10CB00004F935F936F937F938F939F93AF93BF9355
:10CB1000EF93FF93E091B502F091B6028081E0912E
:10CB2000C002F091C102309709F00995FF91EF9191
:10CB3000BF91AF919F918F917F916F915F914F9135
:10CB40003F912F910F900BBE0F900FBE0F901F9033
:10CB500018959DE0899FF0011124E855FD4FA281B1
:10CB6000B3811C92A481B5816C93A681B78188EDB5
:10CB70008C93A085B1854C931286148613860895F4
:10CB80009DE0899FF0011124E855FD4F81E08287E7
:10CB9000A081B1816C933A9680818111FDCF089577
:10CBA0001F93CF93DF93182FEB01FE01649166234F
:10CBB00029F0812F0E94C0652196F7CFDF91CF9198
:10CBC0001F9108951F93CF93DF93182FEB01888156
:10CBD000882369F08A3021F46DE0812F0E94C065BE
:10CBE00069916D30A1F3812F0E94C065F0CFDF9174
:10CBF000CF911F910895CF93DF93CDB7DEB79E01FC
:10CC0000285F3F4F4E815F8160E470E086E793E1EB
:10CC10000E947B9366E773E18D810E94E265DF915C
:10CC2000CF910895CF93C82F8A3031F46DE0809171
:10CC3000B6130E94C06502C08D3029F06C2F809120
:10CC4000B6130E94C06580E090E0CF9108959DE00A
:10CC5000899FF0011124E855FD4F7487638708957B
:10CC6000682F80E00C94C0658093B6138AE992E047
:10CC700090936E3180936D31089584B7877F84BF20
:10CC800088E10FB6F89480936000109260000FBEA8
:10CC900008952FE088E190E00FB6F894A89580936E
:10CCA00060000FBE209360000895A895089588E164
:10CCB0000FB6F89480936000109260000FBE089544
:10CCC000F89428E088E190E00FB6F894A895809356
:10CCD00060000FBE20936000FFCF80910C298091EF
:10CCE0000C2990E0089540E06FE181E491E00C941C
:10CCF000D66BE9E3F1E0808180818D7F80838DE0D8
:10CD000090E00197F1F723E040E06FE182E491E0E9
:10CD10000E94E06B83E090E00197F1F70895909115
:10CD2000390191FD0AC0282F803108F02FE040E042
:10CD30006FE085E491E00C94E06B089580913901F7
:10CD400081FD0EC040E06FE181E491E00E94D66B6E
:10CD5000282F2F7E81E090E0213021F080E008959F
:10CD600080E090E008958091390181FD10C040E09D
:10CD70006FE181E491E00E94D66B8F3131F0982F02
:10CD80009F7E915081E0923018F480E0089581E018
:10CD900008950E94B3668823E1F30895CF93DF934B
:10CDA000C82F0E94C9660E947366D82FC81789F1E0
:10CDB000C83019F40E94796625C0C93121F4863142
:10CDC00089F429E005C0C63169F4893159F426E0B7
:10CDD00040E06FE182E491E00E94E06BE3E0F0E08C
:10CDE0003197F1F72C2F40E06FE182E491E00E944F
:10CDF000E06BD83019F4E9E6F1E002C0E3E0F0E0DE
:10CE00003197F1F70E9473668C1719F083E490E074
:10CE100002C080E490E0DF91CF9108950E94C9663E
:10CE20001092A12A0E9479668091390182608093D4
:10CE300039018091242B8823D9F18091940090911D
:10CE400095004091352B5091362B84179507A0F40F
:10CE50008091012B9091022BA091032BB091042B78
:10CE60008C57914EAF4FBF4F8093012B9093022B65
:10CE7000A093032BB093042B209194003091950044
:10CE8000241B350B8091012B9091022BA091032B39
:10CE9000B091042B820F931FA11DB11D8093012B14
:10CEA0009093022BA093032BB093042B1092242B6E
:10CEB0008091262B8823D9F1809194009091950040
:10CEC0004091392B50913A2B84179507A0F480910B
:10CED000092B90910A2BA0910B2BB0910C2B8C5706
:10CEE000914EAF4FBF4F8093092B90930A2BA09385
:10CEF0000B2BB0930C2B2091940030919500241BA8
:10CF0000350B8091092B90910A2BA0910B2BB0919E
:10CF10000C2B820F931FA11DB11D8093092B9093A1
:10CF20000A2BA0930B2BB0930C2B1092262B089559
:10CF30008091A12A882381F080913A14811104C044
:10CF40000E94B366811106C081E08093381481E0AD
:10CF500090E008950E940E6780E090E0089580912F
:10CF600094009091950090933A2B8093392B21E077
:10CF70002093262B8091390181FD08C080913901D1
:10CF800081FD1AC086E10E94CE6616C02093A02AB9
:10CF900080919400909195009093362B8093352B3F
:10CFA0002093242B809139018D7F809339018091CA
:10CFB000A02A8111FCCFE2CF81E08093A12A0895BD
:10CFC0008091A12A81110AC080913A14882321F00E
:10CFD00081E08093391402C00E94AF6781E090E045
:10CFE00008951F93CF93DF931F92CDB7DEB78FB70E
:10CFF000898380913A14811126C0F8948091A12AE6
:10D00000882351F08091390181FD1BC00E94B366D5
:10D010008823B9F080E003C00E94E06781E020919E
:10D02000470191E02E3008F090E0192F1195811101
:10D030000E949867107429F089818FBF81E090E089
:10D0400004C089818FBF80E090E00F90DF91CF9185
:10D050001F91089580913914882321F00E94AF67B1
:10D060001092391480913814882321F00E940E67A1
:10D070001092381410923A1408950F931F93AB0135
:10D0800021E020933A140091E52A1091E62A20919C
:10D09000E72A3091E82A0F5F1F4F2F4F3F4F009331
:10D0A000E52A1093E62A2093E72A3093E82A22E023
:10D0B000260F27FF0CC080919E2A90919F2A0196EF
:10D0C00090939F2A80939E2A0FEF1FEF07C0BC0109
:10D0D00087EB93E10E94F79100E010E00E942A683C
:10D0E000C8011F910F91089580933C1408950E94E8
:10D0F0007366823011F0823111F480E0089581E08E
:10D10000089508958FEF80934E0122E044E060EF90
:10D110008CE691E00E94E06B25E041E06EE08CE25D
:10D1200090E00E94E06B80E880936F01809146015F
:10D1300080936D0121E045E060E284E491E00C948D
:10D14000E06B8DEF93E00197F1F70E94CC6B1092AA
:10D150001529109297291092192A109214291092C9
:10D160001329E9E3F1E080818E7F808380818D7FC8
:10D1700080838DE090E00197F1F7E9E3F1E08081B1
:10D180008160808323E040E06FE182E491E00E94CF
:10D19000E06B8DEF93E00197F1F780915D01809155
:10D1A0005E010E94826860E070E082EC92E00E9482
:10D1B00071540E94AF6781E090E0089580913B1424
:10D1C0000895CF93DF931F92CDB7DEB789830E9476
:10D1D000C966898180933B14282F40E06FE188E481
:10D1E00091E00F90DF91CF910C94E06B0E94E16889
:10D1F0008091390181FD03C086E00C94CE660895CC
:10D20000FA018093620190936301609360017093CF
:10D2100061013097C1F0808180936B01818180939F
:10D220006A0182818093690183818093680184818E
:10D230008093670185818093660186818093650173
:10D24000878180936401089582EC92E00E94925459
:10D2500081E080930C2980910D2990910E290196EF
:10D2600090930E2980930D2981E090E0089580919C
:10D27000142992E8899FF0011124EB5EF64D10828B
:10D280008F5F833018F48093142902C01092142900
:10D29000E091142982E8E89FF0011124EB5EF64D3D
:10D2A000808181110C94246910920C2908951F9398
:10D2B000CF93DF932091142912E8129F900111243B
:10D2C000D901AB5EB64D4C91411103C00E94376944
:10D2D00093C05091390151FD8FC05091A12A55231F
:10D2E00009F48AC047FF16C00E9437698091D52A89
:10D2F0009091D62AA091D72AB091D82A0196A11D43
:10D30000B11D8093D52A9093D62AA093D72AB093A3
:10D31000D82A72C04330B0F40E9437698091D12A74
:10D320009091D22AA091D32AB091D42A0196A11D1E
:10D33000B11D8093D12A9093D22AA093D32AB0937F
:10D34000D42A5AC050E0EA0122976C177D07B0F446
:10D350000E9437698091CD2A9091CE2AA091CF2A40
:10D36000B091D02A0196A11DB11D8093CD2A909332
:10D37000CE2AA093CF2AB093D02A3EC0B9016A5ECC
:10D38000764D0E94F791E09114291E9FF00111241F
:10D39000EB56F64D8081809305290E943769809174
:10D3A00047018093062990910B29992311F0891741
:10D3B00010F480930B296091062970E084E00E94AC
:10D3C0001C5C6091052970E083E00E941C5C409128
:10D3D000E92A5091EA2A6091EB2A7091EC2A4F5F7A
:10D3E0005F4F6F4F7F4F4093E92A5093EA2A609333
:10D3F000EB2A7093EC2A02C0C0E0D0E0CE01DF91AE
:10D40000CF911F910895CF93DF93EC01888199818B
:10D410000097E9F08730954021F01982188283E067
:10D4200026C06238C1F410920C290E94A35B0E94AE
:10D430000A5B60E870E00E945769181619066CF4E0
:10D440000E94055BE0915503F0915603099587E032
:10D4500095E09983888381E00AC0809109299091A1
:10D460000A29019690930A2980930929F0CFDF9128
:10D47000CF91089591E090933A140E948F660C9496
:10D480002A688091390181FD06C040E06FE085E4A3
:10D4900091E00C94D66B80E108950F931F93CF9386
:10D4A000DF93182F21E020933A140091A12A809154
:10D4B000390181FF16C0809194009091950090935E
:10D4C000362B8093352B2093242B2093A02A8091F8
:10D4D00039018D7F809339018091A02A8111FCCF81
:10D4E00000E00E94C9668091A12A882309F43FC008
:10D4F0008091262B8823D9F18091940090919500FA
:10D50000E091392BF0913A2B8E179F07A0F44091B0
:10D51000092B50910A2B60910B2B70910C2B4C57BF
:10D52000514E6F4F7F4F4093092B50930A2B6093BE
:10D530000B2B70930C2B20919400309195002E1B97
:10D540003F0B4091092B50910A2B60910B2B70914E
:10D550000C2B420F531F611D711D4093092B5093DB
:10D560000A2B60930B2B70930C2B1092262B80911F
:10D57000390181FD03C089E10E94CE6686E00E94E8
:10D58000275C892B51F00E94416AC82F86E00E94D7
:10D59000275C81500E948F6602C0C0E0D0E02091DD
:10D5A0009400309195003093382B2093372B81E0F5
:10D5B0008093252BF8948091390182608093390102
:10D5C000809139018D7F8093390162E0610F87EB93
:10D5D00093E10E94116C789420919B2A30919C2AAF
:10D5E0002F5F3F4F30939C2A20939B2A0E94C9664D
:10D5F00045E060EE82E491E00E94D66B182F86E051
:10D600000E94275C892B19F08C2F0E948F660023C3
:10D6100019F00E94AF6702C00E940E678091252B0F
:10D620008823D9F18091940090919500E091372B57
:10D63000F091382B8E179F07A0F44091052B509145
:10D64000062B6091072B7091082B4C57514E6F4F52
:10D650007F4F4093052B5093062B6093072B7093BD
:10D66000082B20919400309195002E1B3F0B409188
:10D67000052B5091062B6091072B7091082B420FC0
:10D68000531F611D711D4093052B5093062B609312
:10D69000072B7093082B1092252B8091A12A8823A9
:10D6A00061F0209194003091950030933A2B2093B3
:10D6B000392B81E08093262B07C023E040E06FE107
:10D6C00082E491E00E94E06B0E942A681130E9F048
:10D6D0001330A9F48091DD2A9091DE2AA091DF2AEF
:10D6E000B091E02A0196A11DB11D8093DD2A90938F
:10D6F000DE2AA093DF2AB093E02A12E009C0153099
:10D7000031F0173029F411E003C010E001C013E03C
:10D71000812F90E0DF91CF911F910F910895CF93CA
:10D72000DF93EB010E943D68009729F4CE010E942F
:10D730004D6A009751F020919E2A30919F2A2F5FC9
:10D740003F4F30939F2A20939E2ADF91CF910895D7
:10D75000CF93DF938091A12A811104C00E94E067DA
:10D76000D1E001C0D0E00E947366863111F08131B2
:10D7700019F4C091470109C040E06FE186E491E0EF
:10D780000E94D66BC82FCC0FC80FD1110E9498678A
:10D790008C2FDF91CF91089510923E1410923D147A
:10D7A000EFE6F0E08081806280830895FC01808153
:10D7B000862390E002C0959587954A95E2F70895F3
:10D7C000F894FC015081362F30955323042E01C06C
:10D7D000220F0A94EAF72623522B50837894089557
:10D7E00040917B01FC014193A0E8B1E050E8540F67
:10D7F0009D012F5F3F4F6C916193521711F0D9013A
:10D80000F7CF4150E42FF0E0E058FE4F2181FC01BA
:10D81000E058FF4F2083FC01EF57FF4F21E02083AA
:10D82000089560938001E1E8F1E061589F012F5F66
:10D830003F4FDC014D91CD014083621711F0F9019A
:10D84000F5CF08951F920F920FB60F9211240BB6C9
:10D850000F922F933F934F935F936F937F938F9389
:10D860009F93AF93BF93EF93FF9380914701809372
:10D8700006298091132922E8829FC00111248B5E22
:10D88000964D0E94F06B809113298F5F833018F4BE
:10D890008093132902C0109213290E942469FF91DA
:10D8A000EF91BF91AF919F918F917F916F915F9118
:10D8B0004F913F912F910F900BBE0F900FBE0F9085
:10D8C0001F9018951F920F920FB60F9211240F9070
:10D8D0000FBE0F901F9018951F920F920FB60F92C8
:10D8E00011240F900FBE0F901F9018951F920F924A
:10D8F0000FB60F9211240F900FBE0F901F90189526
:10D900001F920F920FB60F9211241092A02A0F901F
:10D910000FBE0F901F9018951F920F920FB60F9287
:10D9200011241092A02A0F900FBE0F901F901895EF
:10D930001F920F920FB60F9211248F9381E0809364
:10D940000C298F910F900FBE0F901F9018951F926A
:10D950000F920FB60F9211241092A02A0F900FBEB3
:10D960000F901F9018951F920F920FB60F921124CF
:10D970008F939F9380913D1490913E1401969093C4
:10D980003E1480933D149F918F910F900FBE0F9086
:10D990001F901895CF92DF92EF92FF920F931F93F3
:10D9A000CF93DF937C018B016A018FE394E10E94A6
:10D9B0003155EC01009751F0EC81FD81309711F069
:10D9C000C8010995CE010E94D955F3CFA601B8012F
:10D9D000C701DF91CF911F910F91FF90EF90DF90E2
:10D9E000CF900C94BB520F931F93CF93DF9300D033
:10D9F000CDB7DEB78091A92A9091AA2AA091AB2A2F
:10DA0000B091AC2A0196A11DB11D8093A92A9093D3
:10DA1000AA2AA093AB2AB093AC2A0E945D6F8C0116
:10DA20008FE394E10E943155009779F0DC01129662
:10DA3000ED91FC911397309729F089839A8309958A
:10DA40009A8189810E94D955EFCF0115110549F0BE
:10DA5000C8010F900F90DF91CF911F910F910C94FF
:10DA6000B2520F900F90DF91CF911F910F910895B7
:10DA70000E9450740E94A35B0E94846D81E493E035
:10DA80009093A42A8093A32A0E945B6F2FEF31E02A
:10DA900040E05EE160E074E082E090E00C94246F8E
:10DAA000BC018FE394E10C949155BC018FE394E1A8
:10DAB0000C947655CF93DF93EC014091A52A5091B9
:10DAC000A62A6091A72A7091A82A4F5F5F4F6F4FD7
:10DAD0007F4F4093A52A5093A62A6093A72A70935C
:10DAE000A82A0E94706F009761F00E94235BE0916A
:10DAF0004503F0914603BE018AEC9CE6099581E05E
:10DB000090E0DF91CF91089585E494E10C942D5538
:10DB10000F93CF93DF93EC017B836A8318865F8337
:10DB20004E83BC0185E494E10E949155E09141143B
:10DB3000F0914214309749F04C815D8101E020E082
:10DB400030E068858A819B810995DF91CF910F91A3
:10DB50000895BC0185E494E10C9476550F93DC01A3
:10DB600018961C921897E0914114F0914214309746
:10DB700059F000E020E030E040E050E060E0129634
:10DB80008D919C91139709950F9108950F93DC0146
:10DB9000AB0114962D913C91159781E018968C93CA
:10DBA000189715967C936E931497E0914114F09119
:10DBB0004214309739F000E061E012968D919C910B
:10DBC000139709950F9108950F93DC01E09141148B
:10DBD000F0914214309771F014964D915C91159725
:10DBE00001E09A0118966C91189712968D919C916C
:10DBF000139709950F910895E0914314F0914414FF
:10DC0000309709F009940895909344148093431435
:10DC100008959093421480934114089585E494E10B
:10DC20000C943155EF92FF920F931F93CF93DF9394
:10DC30008C01EB017A0185E494E10E943155009753
:10DC4000D9F0DC0112962D913C9113972C173D07CA
:10DC500081F41696ED91FC911797309769F0970132
:10DC6000AE01B801DF91CF911F910F91FF90EF901E
:10DC700009940E94D955E3CFDF91CF911F910F9165
:10DC8000FF90EF9008950895CF93DF93C8E7D4E114
:10DC90006881798120E030E043E65EE682E694E147
:10DCA0000E94B1570E944E74688179810E94FE8B58
:10DCB00020E030E047E75EE6BC0182E594E1DF91D9
:10DCC000CF910C94B1578091781490917914209150
:10DCD000761430917714880F991F2817390708F4A4
:10DCE000C90190937914809378140C94446ECF9367
:10DCF000DF930E94A35B0E940A5BEC0119821882E9
:10DD00000E940E6E28813981009719F1FC0140852F
:10DD10004423F9F0FC0142815381F901EE0FFF1F0A
:10DD2000EE0FFF1FEC0FFD1F53834283FC01448164
:10DD300055812F5F3F4FF901EE0FFF1FEE0FFF1FC1
:10DD4000EC0FFD1F51834083398328830E94D955EE
:10DD5000D9CFC901880F991F880F991F02960E9479
:10DD6000055B88819981892B31F087E494E1DF910B
:10DD7000CF910C948952DF91CF910895AF92BF92C9
:10DD8000CF92DF92EF92FF920F931F93CF93DF9387
:10DD900000D0CDB7DEB76B010E940A5BFC010081A9
:10DDA00011811A8309830C30110518F4E12CF12C30
:10DDB0000DC01F930F9380E899E09F938F930E946B
:10DDC000AC920F900F900F900F9021C0E016F106CB
:10DDD000F1F00E940A5BF701EE0FFF1FEE0FFF1F2D
:10DDE000E80FF91FA280B3800E940A5BFFEFEF1AD1
:10DDF000FF0AF701EE0FFF1FEE0FFF1FE80FF91FDD
:10DE000040815181B501C6010E94126EDFCF0F9093
:10DE10000F90DF91CF911F910F91FF90EF90DF90C6
:10DE2000CF90BF90AF9008950F93013059F4809137
:10DE300072149091731490937914809378140F91C5
:10DE40000C94446E0F910895EF92FF920F931F93DD
:10DE5000CF93DF938B01EA0179014EE253E0BC01DD
:10DE600087E494E10E946D5210937314009372142E
:10DE7000D0937514C0937414F0927714E0927614D2
:10DE800084E19FE6DF91CF911F910F91FF90EF907A
:10DE90000C94096E82E694E10E94355882E594E183
:10DEA0000E94355887E494E10C948752809178144D
:10DEB0009091791408950C94C752CF93DF93E09119
:10DEC0003203F09133030995EC01009729F06A8140
:10DED0007B8181E00E941C5CCE01DF91CF9108958F
:10DEE0000F931F93CF93DF93EC01E0913403F091F4
:10DEF000350309958C016A817B8181E00E941C5C5D
:10DF000081E090E0012B11F480E090E0DF91CF916F
:10DF10001F910F910895E0913603F0913703099412
:10DF200020E030E00296FC0132974081442331F03A
:10DF3000FC0131974081240F311DF4CFC9010895B0
:10DF4000FC01208130E0322F22278181282B02C062
:10DF5000220F331F6A95E2F7832F9927FA01E85CB5
:10DF6000FC4F208130E08223932328E030E0241B03
:10DF7000350B02C0969587952A95E2F708956F9222
:10DF80007F928F929F92AF92BF92CF92DF92EF9249
:10DF9000FF920F931F93CF93DF938C01EB016A01E4
:10DFA00079012830310524F4A901B601CE014AC017
:10DFB000590123E0B594A7942A95E1F7411551053D
:10DFC00021F04801612C712C03C0D801FB0120C055
:10DFD00048E050E0B601CE01860D971D0E94A06F6B
:10DFE000F40181934F01FFEF6F1A7F0A6A147B04DB
:10DFF0007CF3C501B7FE02C080E090E0A701477046
:10E0000055274115510511F1080F191FB60118C008
:10E01000CF018C1B9D0B8A159B051CF481918D9360
:10E02000F7CFC501B7FE02C080E090E0A7014770BE
:10E0300055274115510551F0080F191F60E070E098
:10E040008C0F9D1F0E94A06FF8018083DF91CF91FC
:10E050001F910F91FF90EF90DF90CF90BF90AF9006
:10E060009F908F907F906F9008958F929F92AF9224
:10E07000BF92CF92DF92EF92FF920F931F93CF93B5
:10E08000DF9300D0CDB7DEB70E940A5B8C0182E03F
:10E0900090E00E94E85A892B19F480E090E05DC07E
:10E0A000F801818190E0982F88272081820F911DAF
:10E0B0000E94D8527C01009781F30E940A5B4C01B8
:10E0C000F7012681822F86958695869590E0422FCE
:10E0D000477021E030E011F420E030E0820F931F20
:10E0E0000E94E85A892BC9F2F70104811581C12CDD
:10E0F000D12CF8018081882379F1F801A180B12C1D
:10E10000B60133E0759567953A95E1F7A60147703A
:10E110005527680D791D883168F09501CE0101966B
:10E120000E94BF6FBE016F5F7F4FF80180810E9428
:10E13000305C0DC01A8219829501CE0101960E94B1
:10E14000BF6F69817A81F80180810E941C5CCA0CD2
:10E15000DB1C0E5F1F4FCDCFC7010F900F90DF91DB
:10E16000CF911F910F91FF90EF90DF90CF90BF90D4
:10E17000AF909F908F900895DC0150E0E0E1F0E0D7
:10E18000E61BF70BE21BF30B02C0440F551FEA9589
:10E19000E2F78C91852B8C9311968C911197842B9F
:10E1A00011968C9308956F927F928F929F92AF9267
:10E1B000BF92CF92DF92EF92FF920F931F93CF9374
:10E1C000DF938C016B01EA017901283031051CF4E1
:10E1D0004881C8015CC0390153E0759467945A9531
:10E1E000E1F76115710521F04E01A12CB12C03C09E
:10E1F000D801FE0127C0F40141914F0128E030E031
:10E20000B601C8018A0D9B1D0E94BC70FFEFAF1ABA
:10E21000BF0AA614B7047CF3C30177FE02C080E0F6
:10E2200090E09701277033272115310509F43FC08D
:10E23000C80FD91F488150E0B601621B730B685F9D
:10E240007F4F1CC0CF018C1B9D0B861597051CF4BE
:10E2500081918D93F7CFC30177FE02C080E090E0FB
:10E260009701277033272115310509F1C80FD91FF0
:10E27000488150E068E070E0621B730B02C0559566
:10E2800047956A95E2F760E070E0800F911FDF919B
:10E29000CF911F910F91FF90EF90DF90CF90BF90A3
:10E2A000AF909F908F907F906F900C94BC70DF9197
:10E2B000CF911F910F91FF90EF90DF90CF90BF9083
:10E2C000AF909F908F907F906F9008956F927F9204
:10E2D0008F929F92AF92BF92CF92DF92EF92FF9276
:10E2E0000F931F93CF93DF9300D0CDB7DEB78C0190
:10E2F000FC018681E82EE694E694E694F12C282F22
:10E30000277081E090E011F480E090E0E80EF91EC3
:10E31000C70102960E946C5B009709F445C00E94F9
:10E32000115BF8012281FC012083F8012381FC01AB
:10E3300021830E94115B02965C01A70160E070E0FE
:10E340000E940092F80104811581E12CF12CF80162
:10E350008081882339F1F8018180912C670163E085
:10E36000D594C7946A95E1F73701F7E06F227724D7
:10E37000CA0CDB1C883128F00E943A5C9401AC0185
:10E3800008C00E94275C9A8389839401AE014F5F85
:10E390005F4FB301C6010E94D370E80CF91C0E5FF9
:10E3A0001F4FD5CF81E090E00F900F90DF91CF917C
:10E3B0001F910F91FF90EF90DF90CF90BF90AF90A3
:10E3C0009F908F907F906F900895E0915303F0910C
:10E3D00054030994E0912C03F0912D030994E091EA
:10E3E0005703F09158030994E0915903F0915A03AF
:10E3F000099480E090E008950895E0912403F0915D
:10E400002503099480E090E008950F931F93CF9324
:10E41000DF93CDB7DEB7E0970FB6F894DEBF0FBE3F
:10E42000CDBF0E94575B8C010E940A5BAE014F5F1B
:10E430005F4F602F0E94D579882309F446C088A9D0
:10E440009801281B3109C9010E94E85A892BE9F17A
:10E450002E8121110CC0BE016A5E7F4F88E10E94AF
:10E46000305CE0914703F091480309952EC08A85FE
:10E470009B858D3C3BEA930711F0019631F52230E4
:10E4800019F088E090E002C082E090E001979C01E2
:10E490002F5F3F4F12161306F4F6E1E0F0E0EC0FA9
:10E4A000FD1FE80FF91F23852F3F81F3BE01645F35
:10E4B0007F4F89E10E94305C89E10E943A5C62EB07
:10E4C00078E20E942652892B31F6E0960FB6F89436
:10E4D000DEBF0FBECDBFDF91CF911F910F91089589
:10E4E000AF92BF92CF92DF92EF92FF920F931F9362
:10E4F000CF93DF93CDB7DEB7E0970FB6F894DEBFCA
:10E500000FBECDBF8C016B01CE0101967C0180E373
:10E51000F70111928A95E9F781E089838CE00E94E6
:10E52000275C8C831D821F8280917C1491E0980F60
:10E5300090937C14898783E0B82EB8868DEC9BEA93
:10E540009B878A8789E10E943A5C60E073E00E94C1
:10E550002652892B31F082E08E838FEF8C878D8756
:10E5600009C089E10E943A5CBC01CE010C960E9470
:10E570001D52BE828DEC9BEA9D8B8C8B62EB78E208
:10E58000CE0146960E941D520E940A5B9FA78EA74D
:10E590000E94575B88ABC7010E94CE78B82E90E0EE
:10E5A0000E946C5B892B31F10E94115BBC014B2DE9
:10E5B000C7010E94EC78E0901A03F0901B030E94C0
:10E5C000615B5C010E94115BB501F70109950115C2
:10E5D000110581F0009739F0019761F441E050E0B6
:10E5E00064E070E004C041E050E060E070E0C6012B
:10E5F000F8010995E0960FB6F894DEBF0FBECDBFC7
:10E60000DF91CF911F910F91FF90EF90DF90CF900E
:10E61000BF90AF9008950E944E7480937C14E09157
:10E620002403F09125030994892B29F0E091240318
:10E63000F091250304C0E0912603F091270309948B
:10E64000CF93DF93EC0189919991009729F060E0D5
:10E6500070E00E947154F7CFDF91CF910895CF936E
:10E66000DF93EC0189919991009719F00E94C353AF
:10E67000F9CFDF91CF910895CF93DF93EC017B83A6
:10E680006A830E94E56499838883DF91CF9108951E
:10E69000FC018081918122813381820F931F9183BC
:10E6A00080830895CF93DF93EC010E94E564998302
:10E6B0008883DF91CF910895CF93DF93EC010E947F
:10E6C000E56428813981821B930B9C012F5F3F4FAA
:10E6D00081E090E04A815B814217530710F080E0AF
:10E6E00090E0DF91CF910895CF93DF93FC01C28139
:10E6F000D38180819181C80FD91F0E94E5649E015A
:10E70000281B390BC901DF91CF910895CF93DF9377
:10E71000EBE2FBE2CDEEDAE2AFE1BBE21192119265
:10E7200019921992199219921D928BE2E334F8070B
:10E73000A9F7DF91CF910895CF93DF93FC01E15EBC
:10E74000F44D40819C01220F331F220F331F4423BD
:10E7500001F1A0919400B0919500FC01EE0FFF1F14
:10E76000E55DF44D80819181AD01481B590BCA01D3
:10E77000E901C351D54D488159816A817B81480F98
:10E78000591F611D711D488359836A837B83B1833F
:10E79000A083F901E351F54D6081718182819381FC
:10E7A000DF91CF91089560E070E0CB010895FC0106
:10E7B000EE0FFF1FEE0FFF1FE351F54D4083518316
:10E7C000628373830895CF93DF932FE13BE2CDEE15
:10E7D000DAE2EBE2FBE2D9018D919D018823B9F0E9
:10E7E000409194005091950080819181BA01681BFD
:10E7F000790B88819981AA81BB81860F971FA11D02
:10E80000B11D88839983AA83BB8351834083249657
:10E810003296BBE22B323B07F1F6DF91CF910895A0
:10E820000C945D780F931F93FC01CB0140917D14F4
:10E8300050917E1433832283158304837183608314
:10E84000F0937E14E0937D14452B11F40E947778A9
:10E8500080E090E01F910F91089580917D14909138
:10E860007E140097C1F010927E1410927D14DC018A
:10E8700014966D917C9115971296ED91FC911397DA
:10E880000995E0917D14F0917E14309721F08081FC
:10E8900091810C94777808950C948A8E0C94868ECE
:10E8A00084ED92E00E94A8548CEC92E00C94A85461
:10E8B000CF93DF930E94175B892BA9F08CEC92E039
:10E8C0000E94C654EC01009721F10E94575B998386
:10E8D00088830E94525B9B838A83CE0104960E94A8
:10E8E000935A8CAB14C084ED92E00E94C654EC01A4
:10E8F000009779F002960E94A55A99838883BE01F9
:10E900006E547F4FCE018E579F4F0E94FA5BCE010F
:10E9100002C080E090E0DF91CF910895BC016E5479
:10E920007F4F8E579F4F0C94FA5BCF93DF93EC0190
:10E93000BC0184ED92E00E941055BE01892B19F0B4
:10E9400084ED92E009C08CEC92E00E941055892B76
:10E9500039F0BE018CEC92E0DF91CF910C94EB5436
:10E96000DF91CF9108950F931F93CF93DF93EC0125
:10E97000BC0184ED92E00E941055892B91F0FE01BC
:10E9800061917191CF010E94B65BBE016E547F4FC1
:10E99000CE018E579F4FDF91CF911F910F910C9415
:10E9A0000B5CBE018CEC92E00E941055892BD1F0DB
:10E9B0000E94A35B688179818A819B810E94B65BFA
:10E9C0008CA990E00E946C5B0CA910E00E94115B86
:10E9D000BE016C5F7F4FA801DF91CF911F910F9116
:10E9E0000C94F791DF91CF911F910F910895CF93E0
:10E9F000DF93EC01BC0184ED92E00E941055892B5D
:10EA000019F0CE0102960CC0BE018CEC92E00E947F
:10EA10001055892B19F08A819B8102C080E090E01B
:10EA2000DF91CF910895FC01808191810895860F37
:10EA3000911D860F911D8E579F4F0895860F911D32
:10EA4000860F911D8E579F4FFC0180819181089503
:10EA500008958CED9AE10E94EA56892B21F08CED05
:10EA60009AE10C94D7560895E091C81AF091C91A0A
:10EA7000309709F0099480E00895EF92FF920F9388
:10EA80001F93CF93DF937C01EA01FC018081918188
:10EA9000009741F08C30934071F1F70111821082A0
:10EAA00083E0F2C080E024E0829FF0011124E6536D
:10EAB000F54E118210828F5F8430A8F38093C71ABD
:10EAC00080910212909103129093DB1A8093DA1ACC
:10EAD0000E94BC538093432B60E470E08CED9AE17C
:10EAE0000E94C3560E944B7B8CE093E0F701918318
:10EAF000808381E0C9C06230D9F48091442B909129
:10EB0000452B892B89F38091552B863029F48091F0
:10EB10006D2B81FD0E94297581E00E94897C809186
:10EB2000442B9091452B892BF9F20E944D77DCCF35
:10EB3000633060F5611114C02097B1F2D093523068
:10EB4000C093513083E00E94897C8091442B909146
:10EB5000452B892B11F00E9434750E942975C4CF72
:10EB6000613011F6209709F4BFCFD0934E30C09397
:10EB70004D3085E00E94897C8091442B9091452BFB
:10EB8000892B09F4B1CF0E943475AECF6738E9F50F
:10EB90001092C61A0AEC1AE18091C61A8430B8F4B1
:10EBA000F801828193818C179D0749F480819181BE
:10EBB0000E94567CF80111821082138212820C5F2F
:10EBC0001F4F8091C61A8F5F8093C61AE5CFECE67F
:10EBD000F0E3838194818C179D0719F414821382CA
:10EBE0001082B09620E3EC3EF20799F7E9EEF0E3ED
:10EBF000818592858C179D0711F4158214823D96AC
:10EC000081E3EB36F807A1F76FCF683809F06CCFD6
:10EC1000CC5DDA4109F068CF8CED9AE10E94EA56AA
:10EC2000892B09F461CF1092C61AE091C61AE4301C
:10EC300008F05ACF20E2E29FF0011124ED5AFF4C78
:10EC4000818D8823D9F08CED9AE10E94D75680916E
:10EC5000C61AE0E28E9FC00111248D5A9F4C9093FA
:10EC600052308093513082E00E94897C8091442B05
:10EC70009091452B892B11F00E9434758091C61A12
:10EC80008F5F8093C61AD1CFDF91CF911F910F91E3
:10EC9000FF90EF9008959093C91A8093C81A089531
:10ECA000209102123091031260E0EAECFAE1643044
:10ECB00098F4408151814817590759F44281538192
:10ECC0004217530731F46093C51A118210820C94D5
:10ECD000567C34966F5FEBCF6093C51A089540E081
:10ECE000EAECFAE14430A8F451E0540F208131817C
:10ECF000232B61F44093C41A9183808320910212E4
:10ED000030910312338322830C94707C3496452F08
:10ED1000E9CF4093C41A0895209102123091031252
:10ED2000FC01358F248F778F668F08952091021212
:10ED300030910312FC01328721877487638708951D
:10ED4000CF93DF93EA010E94F97B009749F020916D
:10ED5000021230910312FC0132872187D487C387C6
:10ED6000DF91CF9108950F931F93CF93DF9300D03E
:10ED700000D0CDB7DEB78C01AB018FEF89838A83DA
:10ED80008B838C83B801CE0101960E94A0760097F8
:10ED900019F0FC01158304830F900F900F900F90D2
:10EDA000DF91CF911F910F91089540E050E062E014
:10EDB0008CED92E00E9462541092452B1092442BED
:10EDC0000895AC0161E08CED92E00C944454AC01E8
:10EDD00060E08CED92E00C9444540F931F93CF931A
:10EDE000DF938A010E94777BEC01009759F08091B4
:10EDF0000212909103129D8F8C8F1F8F0E8FCE0168
:10EE00000E94E776CE01DF91CF911F910F91089577
:10EE1000CF93DF93A0915130B0915230109719F0F9
:10EE2000ED016C9605C0C0914D30D0914E302996C1
:10EE300080914C3086FF22C01092C31A40E0EAEC69
:10EE4000FAE14430B8F42081318114968D919C917F
:10EE500015972817390759F482819381009739F063
:10EE60004093C31A998388831B821A8205C0349603
:10EE70004F5FE7CF4093C31A0E942975888199811B
:10EE8000009741F04A815B816091432BDF91CF91E4
:10EE90000C946254DF91CF9108950F931F93CF93F9
:10EEA000DF938091552B863009F071C08091442BFF
:10EEB0009091452B8115954009F069C0C4E9D2E0D5
:10EEC000D093452BC093442B02E000934E2B14E9C2
:10EED00010934F2B1092712B1092702B0E94457B38
:10EEE000809590959093712B8093702B1092572B57
:10EEF0001092562B0E94347B809590959093572BBF
:10EF00008093562B0E943475D093452BC093442B8D
:10EF100000934E2B10934F2BA0914F30B091503057
:10EF2000FD01E459FD4F8CE692E001900D920197AE
:10EF3000E1F76CE672E084E69BE20E94F37A80914E
:10EF4000482B8093642B8091492B8093652B809173
:10EF50004A2B8093662B80914B2B8093672B1092CA
:10EF6000712B1092702B0E94457B80959095909309
:10EF7000712B8093702B1092572B1092562B0E945E
:10EF8000347B809590959093572B8093562BDF91EF
:10EF9000CF911F910F910C943475FC01680F791F6C
:10EFA00080E048E1E617F70781F0219198E0322FE1
:10EFB0003827532F517030FD84278695513009F43E
:10EFC00080682695915099F7EDCF08951F920F9282
:10EFD0000FB60F9211240BB60F922F933F934F93BE
:10EFE0005F936F937F938F939F93AF93BF93EF93B1
:10EFF000FF9380919400909195009093302B809393
:10F000002F2B81E08093212B80917100807D809354
:10F0100071000E942D748091212B8823D9F1809159
:10F0200094009091950040912F2B5091302B841794
:10F030009507A0F48091F52A9091F62AA091F72ADD
:10F04000B091F82A8C57914EAF4FBF4F8093F52A5D
:10F050009093F62AA093F72AB093F82A209194006F
:10F0600030919500241B350B8091F52A9091F62A5A
:10F07000A091F72AB091F82A820F931FA11DB11D0C
:10F080008093F52A9093F62AA093F72AB093F82A52
:10F090001092212BFF91EF91BF91AF919F918F9192
:10F0A0007F916F915F914F913F912F910F900BBE88
:10F0B0000F900FBE0F901F9018959FB7F894E1E73F
:10F0C000F0E08081807D808388B38F6288BB10925E
:10F0D0009000E1E9F0E01082109292001092950009
:10F0E000109294008081856080839FBF08952FB720
:10F0F000F894909399008093980088B38F6288BBAE
:10F10000E1E7F0E08081826080832FBF0895CF9394
:10F11000DF93FC01DB0185E0EB0119928A95E9F7A9
:10F120008581837011F082E08C938781837021F058
:10F1300082E012968C9312978581837081F087818B
:10F14000837069F02389348981859285281739076E
:10F1500031F481E0848312961C92129701C01482CC
:10F1600085818370823021F0833021F080E003C0FC
:10F1700082E001C088E011968C931197878183709B
:10F18000823021F0833021F080E003C082E001C0B2
:10F1900088E013968C93DF91CF910895CF93DF93FE
:10F1A00000D000D01F92CDB7DEB7BE016F5F7F4F9A
:10F1B0000E94877889819A81890F8D5F9B81890F51
:10F1C0009C81890F9D81890F0F900F900F900F9058
:10F1D0000F90DF91CF9108954F925F926F927F923F
:10F1E0008F929F92AF92BF92CF92DF92EF92FF9257
:10F1F0000F931F93CF93DF9300D000D000D0CDB7F3
:10F20000DEB78C017B01BE016F5F7F4F4E830E9492
:10F210008778B981AA815B804C808B2F90E0039620
:10F220002A2F30E0820F931F850D911D642D70E011
:10F23000860F971F5D81850F911D4E8150E0481705
:10F2400059070CF49AC0F801818180FB662460F8AC
:10F25000712C43E0660C771C4A95E1F7828180FBB4
:10F26000882480F8912C54E0880C991C5A95E1F779
:10F27000862880818770882A838180FBAA24A0F851
:10F28000B12C85E0AA0CBB1C8A95E1F78A28848101
:10F2900080FBCC24C0F8D12C96E0CC0CDD1C9A95D8
:10F2A000E1F78C28F7018082F80145814370F4E092
:10F2B0004F9FA0011124F80186818370F0E18F9F98
:10F2C000C0011124482BF8018781F0E48F9FC00111
:10F2D0001124482BF7014183F8018085F7018283CF
:10F2E000B23059F4F8018185F7018383F8018285F2
:10F2F000F701848395E0C92E02C083E0C82EB0E0F8
:10F3000080E090E0200F311FDB2EDC0C0197BA1754
:10F3100061F0A901480F591FFA01B384A7014D0DEF
:10F32000511DFA01B082BF5FEFCF9D2DF2E05F1259
:10F330000EC0D701AD0DB11DF80183898C9381E01A
:10F340008D0DD701A80FB11D9E5F84898C9340E07D
:10F3500020E030E0060F171F842F890F215031095C
:10F36000441561F0D801A20FB31F55965C91D701E7
:10F37000A80FB11D5C934F5FEFCF80E026960FB6CC
:10F38000F894DEBF0FBECDBFDF91CF911F910F91DB
:10F39000FF90EF90DF90CF90BF90AF909F908F90B5
:10F3A0007F906F905F904F900895BF92CF92DF92C1
:10F3B000EF92FF920F931F93CF93DF937C01D62E92
:10F3C000EA0182E0861708F0B2C0F701808186FB6F
:10F3D000BB24B0F89181292F269526952370C92E3C
:10F3E000C294C694C69453E0C522382F3770388330
:10F3F00083FB332730F9398384FB332730F93A8391
:10F4000085FB882780F98B83BC822D83892F829589
:10F4100083708E83CF8282818887222391F133810A
:10F42000848190E0982F8827830F911D9A87898780
:10F4300087010B5F1F4F223079F460E073E0CE014B
:10F440000B960E941D52F70186818B8785818C87E0
:10F450008701095F1F4F20C02330F1F4F7013D966B
:10F4600080E090E03E2F2F2F4291DE01A80FB91FC0
:10F470001B964C93019688309105B1F7032F122FFC
:10F480000BC087010D5F1F4F60E073E0CE010B964C
:10F490000E941D521A861986CC20B9F1B1100DC0F8
:10F4A000F8012081818190E0982F8827820F911D9B
:10F4B0009C8B8B8B0E5F1F4F04C089859A859C8B1C
:10F4C0008B8BF2E0CF120EC060E073E0CE01459668
:10F4D0000E941D52F80181818D8B80818E8B0E5F81
:10F4E0001F4F1BC0F3E0CF1218C0085F1F4FF80179
:10F4F00080E090E02291DE01A80FB91F55962C9371
:10F50000019688309105B1F708C060E073E0CE0144
:10F5100045960E941D521C8A1B8AC8018E199F099C
:10F520002D2D281B2FA71EA70DA7D81608F480E0A5
:10F53000DF91CF911F910F91FF90EF90DF90CF90CF
:10F54000BF900895FB0141505109460F571FE41722
:10F55000F50778F4208130E0322F22276181260FD1
:10F56000311D820F931F8217930708F4019632967C
:10F57000EECFE417F50751F4208130E0322F222737
:10F58000820F931F8217930708F401960895CF9373
:10F59000DF93C0914F2BD0E0649720914E2B30E049
:10F5A000322F2227C20FD31F48E050E068E57BE2EC
:10F5B0009E01280F311DC9010E94A27AAE0160E6AA
:10F5C0007BE20E94A27A009721F09827892798274A
:10F5D00002C08FEF9FEFDF91CF9108959093F51ABE
:10F5E0008093F41A0895FC015381560F50934B2BCE
:10F5F000872F99274281480F40934A2BA181A093DE
:10F60000492BE081E093482B242F30E0281739075D
:10F6100048F481E08A0F8093492B811103C0EF5F8A
:10F62000E093482B852F90E077278617970788F47B
:10F630004F5F40934A2B41110CC08091492B8F5F43
:10F640008093492B811105C08091482B8F5F809357
:10F65000482B0895AB01BC0180E090E00E94A27AA3
:10F66000982789279827089544E150E06CE47BE2CD
:10F6700080E090E00E94A27A009721F098278927E5
:10F68000982708958FEF9FEF089586E00C94C77A2E
:10F6900081E10C94C77A80E0E82FF0E0EE0FFF1FC5
:10F6A000ED52FF4C118210828F5F8430A8F380E00E
:10F6B00090E2899FF0011124ED5AFF4C118E8F5F6B
:10F6C0008430B0F380E094E09093EF1A8093EE1AC8
:10F6D00080E09DE0989FF0011124E751FF4C1582D6
:10F6E00014828F5F8A30B0F38093ED1A0895CF9320
:10F6F0002091EE1A3091EF1A2F5F3F4F21154DE701
:10F70000340710F020E030E1522F432FE3E5F0E31F
:10F71000C0E0C43059F0A18DAA2329F0A481B5819D
:10F72000A417B50749F3CF5FB096F3CF3093EF1A24
:10F730002093EE1A1092ED1A20E0E0E0F0E0243081
:10F74000E8F430E2239FD0011124AD5ABF4C599602
:10F750003C915997311104C02093ED1AFD0110C05E
:10F76000373041F4309739F05A964C915A97328D90
:10F77000341708F0DF012F5FFD01E1CF2093ED1A70
:10F780003097A1F122E0218F2091F01A2487209157
:10F79000F11A25872091F21A26872091F31A2787DC
:10F7A00028ED34E0338B228B358B248B21E030E045
:10F7B000318B208B138E21E0228F23E0208F168A3D
:10F7C00020E1278B2091EE1A3091EF1A3227232760
:10F7D00032273583248377836683DC014D915D91E5
:10F7E0006D917C914083518362837383CF01CF916C
:10F7F0000895CF93DF932091EE1A3091EF1A2F5F87
:10F800003F4F21154DE7340710F020E030E1522F33
:10F81000432FEDEEF0E3C0E0CA3041F0A081B181AA
:10F82000CF5F3D96A417B507B9F7E9CF3093EF1A2C
:10F830002093EE1A40E05DE04A30A0F4A1E0A40F6E
:10F84000549FF0011124E751FF4C24813581232B73
:10F8500039F44093ED1A309741F480E090E023C0F2
:10F860004A2FEACF4093ED1AF8CF2091EE1A30914B
:10F87000EF1A322723273227358324837783668341
:10F88000009729F4108211821282138209C0EC01C0
:10F8900088819981AA81BB8180839183A283B3836C
:10F8A00080E48087CF01DF91CF91089540E044301C
:10F8B000A0F4E42FF0E051E0540FEE0FFF1FED52E3
:10F8C000FF4C208131812817390729F44093ED1A24
:10F8D000118210820895452FEACF4093ED1A0895C2
:10F8E00040E0443098F4E42FF0E051E0540FEE0F84
:10F8F000FF1FED52FF4C20813181232B29F44093CF
:10F90000ED1A918380830895452FEBCF4093ED1A34
:10F910000895AF92BF92CF92DF92EF92FF920F9332
:10F920001F93CF93DF93C0915130D09152308430E8
:10F9300009F4DCC124E73BE23093503020934F3090
:10F940003093472B2093462B833059F4898D8F7049
:10F95000833009F06BC088899989892B09F0DFC64B
:10F960007FC0823009F080C08091F31A8F5F80934E
:10F97000F31A811113C08091F21A8F5F8093F21AEB
:10F9800081110CC08091F11A8F5F8093F11A81115F
:10F9900005C08091F01A8F5F8093F01A1092452B6A
:10F9A0001092442B1092E8301092E730298D822F6C
:10F9B0008D7F853041F48A8D8F5F8A8F843109F085
:10F9C000AEC6198EACC6222309F4A9C688899989C6
:10F9D000892B09F441C08A8D9FEF980F9A8F81116E
:10F9E0009EC68B8D883031F09FEF920F923048F495
:10F9F000853039F4198E80E880934C300E94087766
:10FA000047C5853038F493E0082E01C0990F0A9459
:10FA1000EAF701C090E39A8F8F5F8B8F822F8F70F0
:10FA20008330A1F048F4813009F44FC3823009F0EB
:10FA300076C610926D2B4CC3863009F4C8C488304A
:10FA400009F4C5C4843009F06AC6C1C484E0809357
:10FA50004C300E9408774EC52F70233009F05FC6E6
:10FA600088E080934C3009C5853019F5E0914D3020
:10FA7000F0914E3084819581892B09F450C6109203
:10FA800052301092513088E69BE290935030809330
:10FA90004F309093472B8093462B1092E830109272
:10FAA000E7301092452B1092442B88E080934C3025
:10FAB0001BC180914C2B853409F031C600914E2B2F
:10FAC00010E0102F002780914F2B080F111D8091FF
:10FAD000442B9091452B8017910708F420C6109372
:10FAE000452B0093442B8091522B8F7309F017C63E
:10FAF0008091532B811113C68091E3309091E430B3
:10FB0000C0915D03D0915E038C179D0759F440911D
:10FB1000E5305091E63020915F0330916003421749
:10FB20005307A1F020915C2B30915D2B28173907EA
:10FB300009F0F5C520915E2B30915F2B8091E53067
:10FB40009091E6302817390709F0E9C50E94347B07
:10FB5000019609F0E4C58091552B863009F429C13E
:10FB60008131E9F1813009F0DAC58091602B88306C
:10FB700009F0D5C51092602B8091622B9091632B78
:10FB8000873F3FEF930710F0099601C008969093C6
:10FB9000632B8093622B8091582B9091592BA091CD
:10FBA0005A2BB0915B2B80935C2B90935D2BA09391
:10FBB0005E2BB0935F2B8091E3309091E430A09165
:10FBC000E530B091E6308093582B9093592BA09359
:10FBD0005A2BB0935B2B80E48093542B7DC50C5142
:10FBE00011091093452B0093442B88E69BE29093D8
:10FBF000503080934F308091662B9091672B892BEA
:10FC000029F00E94487B019609F089C52091622B5A
:10FC10003091632B2115310509F481C589EE90E3FC
:10FC200090934E3080934D30A090602BB090612B1C
:10FC300040915F0350916003609161037091620392
:10FC4000A0916303B09164030091582B1091592B3C
:10FC5000E0905A2BF0905B2BE0914D30F0914E30BC
:10FC600081E3EB36F80708F05AC584819581009747
:10FC700021F12817390709F586819781009719F036
:10FC8000A816B906D1F4808191818C179D0729F4BB
:10FC9000C280D380C416D506B1F08617970729F421
:10FCA000C280D380CA16DB0671F00817190729F441
:10FCB00082819381E816F90631F03D96F0934E303B
:10FCC000E0934D30C9CF109252301092513082E003
:10FCD00080934C3088E69BE29093472B8093462B91
:10FCE0001092E8301092E7300E9408778091E73058
:10FCF0009091E830009709F412C59C01245E3F4FB3
:10FD00003093452B2093442B30934E2B20934F2B35
:10FD1000E0914D30F0914E3020852093542B21E11D
:10FD20002093552B08969827892798279093652B21
:10FD30008093642B1092672B1092662B848195819F
:10FD40009093612B8093602B868197819093632B96
:10FD50008093622B8091E3309091E430A091E53064
:10FD6000B091E6308093582B9093592BA0935A2B47
:10FD7000B0935B2B80819181A281B38180935C2BB6
:10FD800090935D2BA0935E2BB0935F2B84E79BE257
:10FD90009093503080934F300E94487B809590958F
:10FDA000009711F48FEF9FEF9093672B8093662B52
:10FDB00093C40E94457B019609F0B1C48091622BE7
:10FDC0009091632B009709F4AAC42091602B309185
:10FDD000612B2115310509F4A2C44091582B509193
:10FDE000592B60915A2B70915B2BECE6F0E3C3E545
:10FDF000D0E3F080FF20A9F0AC81BD818A179B077A
:10FE000081F4AE81BF812A173B0759F4A881B981DB
:10FE10004A175B0731F4AA81BB816A177B0709F493
:10FE20006FC1A096B096A0E3C33DDA0711F7209109
:10FE30006D2B2F732230D9F49093EB1A8093EA1A2A
:10FE400040E0443090F4E42FF0E0EE0FFF1FED525D
:10FE5000FF4C208131814F5F8217930791F71092F9
:10FE6000ED1A20E0C0E0D0E07EC04093ED1A809112
:10FE70006D2B82FD54C484E180936D2B88E290E069
:10FE80009093452B8093442B80E580936C2B80913D
:10FE9000672B90916B2B9093672B3091662B9091F1
:10FEA0006A2B9093662B30936A2B2091652B90914F
:10FEB000692B9093652B2093692B9091642B9093E1
:10FEC000ED1A4091682B4093642B9093682B8F5FC1
:10FED00080936B2B81110FC081E0830F80936A2B7D
:10FEE000811109C081E0820F8093692B811103C0C9
:10FEF0009F5F9093682B8091602B9091612B9093E2
:10FF0000EB1A8093EA1A2091622B3091632B309385
:10FF1000612B2093602B9093632B8093622B8091B5
:10FF2000582B9091592BA0915A2BB0915B2B809319
:10FF30005C2B90935D2BA0935E2BB0935F2B8091F5
:10FF4000E3309091E430A091E530B091E6308093B9
:10FF5000582B9093592BA0935A2BB0935B2BA1C392
:10FF6000373089F02F5F2430C0F430E2239FC00186
:10FF70001124FC01ED5AFF4C318D3111F1CF20934A
:10FF8000ED1AEF010CC0209721F0428D3A8D341705
:10FF900048F7EC01CD5ADF4CE5CF2093ED1A2097BE
:10FFA00009F4BDC3D0935230C093513083E08A8F9F
:10FFB000888F1E8A84E08F8B1B8E8091622B90919C
:10FFC000632B9D838C838091602B9091612B9F8309
:10FFD0008E838091582B9091592BA0915A2BB091E0
:10FFE0005B2B88839983AA83BB8381E0898F80916F
:10FFF000F01A8C878091F11A8D878091F21A8E8782
:020000021000EC
:100000008091F31A8F8781E090E0998B888B8091A3
:10001000672B8B878091662B8A878091652B8987D8
:100020008091642B888781E090E00E94F383809127
:100030006C2B282F207F30E0213531050CF445C092
:1000400082958F7090E00597880F991F880F991FF0
:100050003091EC1A20E0E22FF0E0E817F9078CF578
:10006000E45BF44D30A5311105C02093ED1A1092D8
:10007000EC1A2BC0313011F42F5FEDCF3230E1F4A8
:1000800041A54430C9F42093ED1A3093EC1A82A5AF
:1000900090E0982F882723A5822B9093EB1A8093CA
:1000A000EA1A893DA4E09A0710F088ED94E09B8B52
:1000B0008A8B9D8B8C8B09C041A5442311F0240FA2
:1000C000CACF2093ED1A3093EC1A80E180936D2B08
:1000D00080916D2B826080936D2B82E08093742BD6
:1000E00084E08093752B8093762B88ED8093772B1B
:1000F0008CE290E09093452B8093442B80E67EC267
:10010000D0935230C093513010924C3090916D2B5F
:1001100092FF03C0198E80E21AC280916C2B8295E7
:100120008F70880F880F8093ED1A081B11090451F6
:1001300011091093452B0093442B8F2D8F70823023
:1001400029F4892F8F73823139F41FC0813021F453
:10015000892F8F738230C9F0012B19F4892F837096
:10016000A1F02091642B888528133EC22091652B35
:100170008985281339C22091662B8A85281334C2B9
:100180002091672B8B8528132FC294FF4AC0688962
:1001900079896115710509F444C0CE010C960E945D
:1001A000F37A3091682B8091482B38133AC0209114
:1001B000692B8091492B281334C090916A2B809130
:1001C0004A2B98132EC080916B2B40914B2B84139C
:1001D00028C03C872D879E878F878B8D81111AC001
:1001E0002E89888D9A8D891B922F96959695969536
:1001F000891B280F2E8B87FD81959F89392F369576
:100200003695931B980F9F8B822F869586958695A2
:10021000890F888F81E080934C30888D8A8F198A6E
:10022000188A498D842F8F7090E0FC013197E83057
:10023000F10508F074C2E057FF4F0C94C28D809115
:100240004C3080FF14C083E0898F80E480934C3071
:10025000198A188A8091442B9091452B009709F4B4
:1002600008C122E420934C300E94F38302C18091A4
:100270006D2B8F73823009F052C227CF80914C30A2
:1002800080FF70C080916D2B8F73823109F06AC03E
:1002900080916C2B282F207F30E0213531050CF424
:1002A00045C082958F7090E00597880F991F880F41
:1002B000991F3091EC1A20E0E22FF0E0E817F907DF
:1002C0008CF5E45BF44D30A5311105C02093ED1A97
:1002D0001092EC1A2BC0313011F42F5FEDCF323079
:1002E000E1F441A54430C9F42093ED1A3093EC1A9F
:1002F00082A590E0982F882723A5822B9093EB1A54
:100300008093EA1A893D24E0920710F088ED94E08A
:100310009B8B8A8B9D8B8C8B09C041A5442311F04C
:10032000240FCACF2093ED1A3093EC1A83E0898F03
:100330008091642B88878091652B89878091662BBB
:100340008A878091672B8B8781E090E00E94F383FE
:1003500082E480934C30198A188A1092452B1092AF
:10036000442B87C080E280934C300E940877E09154
:100370005130F0915230118E7ACD80916D2B80FFEB
:1003800028C044FD26C088899989892B09F0C7C1F6
:100390008091442B9091452B01960E94F3832091EC
:1003A0004C30822F806180934C308091442B90910F
:1003B000452B892B19F0226120934C300E9408773D
:1003C00081E090E0998B888B88E0898F1B8E81E19A
:1003D0000CC185FF1CC08091722B90E0982F88275C
:1003E0002091732B822B20914F3030915030280F69
:1003F000391F3093503020934F302091442B30914F
:10040000452B281B390B3093452B2093442B80918F
:10041000442B9091452B009749F044FD07C0209153
:100420004C30226020934C300E94F38380916E2BDD
:1004300090E0982F882720916F2B820F911D909329
:10044000EB1A8093EA1A2C893D892817390710F096
:10045000892B21F43093EB1A2093EA1A8091EA1A3F
:100460009091EB1A9B8B8A8B80914C30837009F4AE
:1004700056C11092E8301092E7300E9408778091C0
:100480004C3085FF07C01092E8301092E730198E8B
:1004900084E1ABC084FF0AC01092E8301092E730CC
:1004A00081E090E0998B888B84E08FCF2091E730BA
:1004B0003091E83021153105E1F080FF02C0198A42
:1004C000188A88899989009781F48A899B8982177B
:1004D000930720F49093E8308093E7308091E730E1
:1004E0009091E830998B888B04C09093E83080938A
:1004F000E7301B8E8091462B9091472B9093503084
:1005000080934F308091E7309091E830892B59F0FB
:1005100088899989009739F088969093452B809324
:10052000442B88E10BC080914C3081FFF8C088E2F9
:1005300090E09093452B8093442B80E180936D2B2A
:100540005CC080914C3080FFEAC0198E80E18093BE
:100550004C300E940877E3C08091442B9091452B4A
:10056000009711F00E94F38390916D2B80914C3095
:1005700090FF0BC080FF06C087E0898F1A8E198A12
:10058000188A19C086E0898F16C080FF1EC085E0DA
:10059000898F198A188AC3C08091442B9091452B6A
:1005A000009711F00E94F38380916D2B80FF0DC0A6
:1005B00087E0898F1A8E81E090E00E94F38380E1CA
:1005C00080934C300E9408770FC08091442B90910B
:1005D000452B892B49F4A3C080914C3080FF9FC0EC
:1005E00087E0898F1A8E9BC080E180936D2B88E213
:1005F00090E09093452B8093442B80E580936C2B67
:1006000088858093682B89858093692B8A85809360
:100610006A2B8B8580936B2B8C858093642B8D85C7
:100620008093652B8E858093662B8F858093672BB7
:1006300086E08093552B8C819D819093612B8093D4
:10064000602B8E819F819093632B8093622B80918E
:10065000E3309091E430A091E530B091E6308093A2
:10066000582B9093592BA0935A2BB0935B2B8881D6
:100670009981AA81BB8180935C2B90935D2BA09381
:100680005E2BB0935F2B898D84FF05C010926F2B7A
:1006900010926E2B06C084E080936E2B88ED8093C1
:1006A0006F2B80E48093542B8091442B9091452BA9
:1006B00090934E2B80934F2B1092732B1092722B92
:1006C0001092712B1092702B0E94457B8095909513
:1006D0009093712B8093702B85E480934C2B109218
:1006E0004D2B1092532B1092522B8091F41A909113
:1006F000F51A01969093F51A8093F41A9093502B63
:100700008093512B1092572B1092562B0E94347BC2
:10071000809590959093572B8093562B04C0109200
:10072000452B1092442B10924C30DF91CF911F91AA
:100730000F91FF90EF90DF90CF90BF90AF90089512
:1007400098278927982708950E94C88D0895FC014D
:100750008091462B9091472B2CE430E3281B390BDA
:10076000AB01261737070CF4A9011416150654F42B
:100770005093E8304093E730E817F90719F0BF01CC
:100780000C94F791089580E88093610010926100C5
:100790000E9479620E94D9530E9455668091F32885
:1007A0009091F428009729F001979093F428809372
:1007B000F328C090F528D090F628E090F728F09024
:1007C000F8280E941365C616D706E806F90611F345
:1007D0000E9413656093F5287093F6288093F7289C
:1007E0009093F828D7CF2091513030915230BC01EE
:1007F000C90108960E94F37AE0915130F09152308D
:100800008091482B80878091492B818780914A2B4A
:10081000828780914B2B838708952F923F924F922E
:100820005F926F927F928F929F92AF92BF92CF9280
:10083000DF92EF92FF920F931F93CF93DF93CDB789
:10084000DEB763970FB6F894DEBF0FBECDBF7C0155
:100850001B016A01FC0117821682838181FF66C336
:10086000BE016F5F7F4F4B01F7019381F10193FD53
:10087000859193FF81911F01882309F453C3853229
:1008800039F493FD859193FF81911F01853239F4ED
:10089000B70190E00E947A9256016501E5CF10E021
:1008A000512C20E02032A0F48B3269F030F48032F9
:1008B00059F0833269F420612CC08D3239F08033D5
:1008C00039F4216026C02260246023C0286021C042
:1008D00027FD27C030ED380F3A3078F426FF06C0E8
:1008E000FAE01F9F300D1124132F13C06AE0569EAB
:1008F000300D1124532E20620CC08E3221F426FDBF
:1009000011C3206406C08C3611F4206802C08836FA
:1009100041F4F10193FD859193FF81911F018111B4
:10092000C1CF9BEB980F933018F42061805E06C016
:100930009BE9980F933008F0AAC12F7E26FF16E09E
:100940002F73722E853621F4F22FF0647F2E08C0AB
:10095000863621F4622F6068762E02C01111115084
:1009600077FE07C01C3348F444244394410E27E02B
:100970000BC0183030F4212F06C027E04CE3442E82
:1009800003C027E017E0412C560174E0A70EB11C0C
:10099000F6016081718182819381042DA4010E94FE
:1009A000FF906C01098100FF02C003FF06C071FCCB
:1009B00007C072FC08C0612C08C03DE2632E05C070
:1009C0002BE2622E02C090E2692E802F8C7099F18A
:1009D000662011F084E001C083E0851510F0512CF1
:1009E0000BC0581A73FC08C0B70180E290E00E9467
:1009F0007A925A94C9F7F3CF662029F0B701862D71
:100A000090E00E947A9203FD03C00EE011E102C063
:100A10000AE011E1F72DF0717F2EF801849188230F
:100A200009F476C271108052B70190E00E947A9268
:100A30000F5F1F4FF2CF77FE0FC04C0C04FF04C0B6
:100A40008A81813309F44A94141474F5F8E0F4159A
:100A500078F588E0482E2CC076FC2AC0812F90E0E3
:100A60008C159D059CF06CEFC6166FEFD60674F0E2
:100A7000772D7068772E0AC0E2E0F0E0EC0FFD1FE2
:100A8000E10FF11D8081803319F411501111F4CF61
:100A900077FE0EC044244394410E812F90E0C81687
:100AA000D9062CF41C1904C04424439401C010E05E
:100AB00077FE07C01C141D043CF496012F5F3F4FC6
:100AC00005C025E030E002C021E030E0662011F0F2
:100AD0002F5F3F4F112331F0412F50E04F5F5F4FA9
:100AE000240F351F452D50E02417350714F4521AF2
:100AF00001C0512C872D897049F4552039F0B70178
:100B000080E290E00E947A925A94F7CF662029F012
:100B1000B701862D90E00E947A9273FC09C055209F
:100B200039F0B70180E390E00E947A925A94F7CFAF
:100B300077FE5FC09C2D8D2DD7FE02C090E080E037
:100B4000692E782E40E050E0C601841991099D87F6
:100B50008C87960126193709280D391D812F90E0C1
:100B6000EE27FF27E81BF90BFF87EE87FFEF6F16D5
:100B70007F0669F4B7018EE290E02B8B3A8B488BAD
:100B8000598B0E947A92598948893A892B89C614CF
:100B9000D70454F06C857D85661577052CF4F90132
:100BA000E40FF51F818101C080E371E0671A7108CD
:100BB0004F5F5F4FEE85FF856E167F066CF0B701C5
:100BC00090E02B8B3A8B488B598B0E947A922B8921
:100BD0003A8948895989CACF6C147D0439F49A81BD
:100BE000963318F4953311F404FF81E3B70190E0D4
:100BF0004BC08A81813309F00F7EB70190E00E94DB
:100C00007A92111105C074FE18C085E490E017C0F7
:100C1000B7018EE290E00E947A9282E066246394AB
:100C2000680EF401E80FF11D8081B70190E00E9489
:100C30007A92115041F3862DF1CF85E690E0B7010D
:100C40000E947A92D7FC05C0C114D10439F404FF84
:100C500005C0D194C194D1088DE201C08BE2B701E7
:100C600090E00E947A9280E36AE0C616D1042CF0EC
:100C70008F5FFAE0CF1AD108F7CFB70190E00E945A
:100C80007A92B701C601C0960E947A9241C183361A
:100C900031F0833779F0833509F058C021C056010F
:100CA00072E0A70EB11CF6018081898301E010E09B
:100CB000640114C05601F2E0AF0EB11CF601C08011
:100CC000D18026FF03C0612F70E002C06FEF7FEF7D
:100CD000C6012B8B0E9426928C012B892F7715C081
:100CE0005601F2E0AF0EB11CF601C080D18026FFA4
:100CF00003C0612F70E002C06FEF7FEFC6012B8B46
:100D00000E94E8918C012B892068722E23FD1AC065
:100D1000852D90E008171907A8F4B70180E290E04C
:100D20000E947A925A94F4CFF60177FC859177FE6F
:100D300081916F01B70190E00E947A9251105A940C
:100D4000015011090115110579F7E2C0843611F03F
:100D5000893651F5560127FF09C0F4E0AF0EB11CEA
:100D6000F60160817181828193810AC0F2E0AF0E49
:100D7000B11CF60160817181882777FD8095982FDD
:100D8000022F0F7697FF08C090958095709561951A
:100D90007F4F8F4F9F4F00682AE030E0A4010E94F0
:100DA000B493C82EC8183EC0022F853721F40F7E99
:100DB0002AE030E01DC0097F8F3691F018F48835A5
:100DC00059F0B0C0803719F0883711F0ABC000611E
:100DD00004FF09C0046007C024FF08C0066006C005
:100DE00028E030E005C020E130E002C020E132E040
:100DF000560107FF09C0F4E0AF0EB11CF601608197
:100E000071818281938108C0F2E0AF0EB11CF601BE
:100E10006081718180E090E0A4010E94B493C82EAB
:100E2000C8180F7706FF0BC0202F2E7FC11650F475
:100E300004FF0AC002FD08C0202F2E7E05C0DC2C56
:100E4000202F03C0DC2C01C0D12E24FF0DC0FE01D9
:100E5000EC0DF11D8081803311F4297E09C022FF41
:100E600006C0D394D39404C0822F867809F0D3941B
:100E700023FD13C020FF06C01C2DD51418F4150D3A
:100E80001D19D52CD51468F4B70180E290E02B8BA6
:100E90000E947A92D3942B89F5CFD51410F45D1863
:100EA00001C0512C24FF12C0B70180E390E02B8BCE
:100EB0000E947A922B8922FF17C021FF03C088E588
:100EC00090E002C088E790E0B7010CC0822F8678DE
:100ED00059F021FD02C080E201C08BE227FD8DE2C6
:100EE000B70190E00E947A92C11638F4B70180E30E
:100EF00090E00E947A921150F7CFCA94F401EC0D61
:100F0000F11D8081B70190E00E947A92C110F5CF67
:100F1000552009F4C2CCB70180E290E00E947A9299
:100F20005A94F6CFF7018681978102C08FEF9FEF29
:100F300063960FB6F894DEBF0FBECDBFDF91CF91A1
:100F40001F910F91FF90EF90DF90CF90BF90AF90E7
:100F50009F908F907F906F905F904F903F902F90D9
:100F600008955058BB27AA270ED04EC23FD230F06A
:100F700044D220F031F49F3F11F41EF4FFC10EF46F
:100F8000E095E7FBF5C1E92F50D280F3BA1762076D
:100F900073078407950718F071F49EF568C20EF484
:100FA000E0950B2EBA2FA02D0B01B90190010C0179
:100FB000CA01A0011124FF27591B99F0593F50F491
:100FC000503E68F11A16F040A22F232F342F4427E9
:100FD000585FF3CF469537952795A795F0405395E1
:100FE000C9F77EF41F16BA0B620B730B840BBAF0B1
:100FF0009150A1F0FF0FBB1F661F771F881FC2F71C
:101000000EC0BA0F621F731F841F48F4879577952F
:101010006795B795F7959E3F08F0B3CF9395880FE6
:1010200008F09927EE0F979587950895DFD158F02E
:1010300080E891E009F49EEFE0D128F040E851E02B
:1010400059F45EEF09C09AC112C2E92FE078EDD1E0
:1010500068F3092E052AC1F32617370748075907F1
:1010600038F00E2E07F8E02569F0E025E0640AC0AC
:10107000EF6307F8009407FADB01B9019D01DC0179
:10108000CA01AD01EF9347D0BFD10AD05F9155237C
:1010900031F02BED3FE049E450FD49EC63CF08957A
:1010A000DF93DD27B92FBF7740E85FE316161706F9
:1010B00048075B0710F4D92FE5D19F938F937F9357
:1010C0006F934AD3E0E3F1E06CD19ED12F913F9131
:1010D0004F915F919ED2DD2349F09058A2EA2AED0C
:1010E0003FE049EC5FE3D0785D274DDFDF918CC1B5
:1010F0001BD108F481E008950CD086C17ED140F068
:1011000075D130F021F45F3F19F032C15111B0C1F7
:1011100035C18BD198F39923C9F35523B1F3951BAE
:10112000550BBB27AA2762177307840738F09F5F08
:101130005F4F220F331F441FAA1FA9F333D00E2E77
:101140003AF0E0E830D091505040E695001CCAF7E4
:1011500029D0FE2F27D0660F771F881FBB1F2617A9
:1011600037074807AB07B0E809F0BB0B802DBF017C
:10117000FF2793585F4F2AF09E3F510568F0F8C053
:1011800077C15F3FECF3983EDCF3869577956795E2
:10119000B795F7959F5FC9F7880F911D969587952D
:1011A00097F90895E1E0660F771F881FBB1F62174C
:1011B00073078407BA0720F0621B730B840BBA0B0A
:1011C000EE1F88F7E095089519F40EF0D1C04FC1D5
:1011D000D5C033D1C8F39638C0F707F80F92E8941A
:1011E0002BE33AEA48EB5FE716D20F920F920F9289
:1011F0004DB75EB70F92CED1EDE5F1E0D2D04F9171
:101200005F91EF91FF91E595EE1FFF1F49F0FE57AB
:10121000E0684427EE0F441FFA95E1F74195550B1E
:101220003AD10F9007FE2EC1089597FB0EF4A9D076
:101230003EC0E89409C097FB3EF490958095709568
:1012400061957F4F8F4F9F4F9923A9F0F92F96E912
:10125000BB279395F695879577956795B795F11187
:10126000F8CFFAF4BB0F11F460FF1BC06F5F7F4F24
:101270008F4F9F4F16C0882311F096E911C0772336
:1012800021F09EE8872F762F05C0662371F096E83F
:10129000862F70E060E02AF09A95660F771F881F0E
:1012A000DAF7880F9695879597F90895E894F92FBE
:1012B00096EBFF2381F0121613061406440B939548
:1012C000F69587957795679557954040FF23B9F731
:1012D0001BC099270895882351F49850D2F7872B83
:1012E000762F652F542F432F322F20E0B1F31216A3
:1012F00013061406440B88233AF09A95440F551FA1
:10130000661F771F881FCAF755234AF4440F551FDD
:1013100011F460FF04C06F5F7F4F8F4F9F4F880FA6
:101320009695879597F90895990F0008550FAA0B80
:10133000E0E8FEEF16161706E807F907C0F01216E8
:101340001306E407F50798F0621B730B840B950BEB
:1013500039F40A2661F0232B242B252B21F4089540
:101360000A2609F4A140A6958FEF811D811D0895DD
:1013700097F99F6780E870E060E008959FEF80EC48
:10138000089590958095709560955095409530950D
:1013900021953F4F4F4F5F4F6F4F7F4F8F4F9F4F65
:1013A0000895DF93CF931F930F93FF92EF92DF92F5
:1013B0007B018C01689405C0DA2EEF012AD1FE0171
:1013C000E894A5912591359145915591AEF3EF01A2
:1013D000DADDFE019701A801DA9479F7DF90EF904A
:1013E000FF900F911F91CF91DF91089500240A94EF
:1013F0001616170618060906089500240A941216F0
:101400001306140605060895092E0394000C11F422
:10141000882352F0BB0F40F4BF2B11F460FF04C0CF
:101420006F5F7F4F8F4F9F4F089557FD9058440F28
:10143000551F59F05F3F71F04795880F97FB991F33
:1014400061F09F3F79F087950895121613061406F0
:10145000551FF2CF4695F1DF08C01616170618067D
:10146000991FF1CF86957105610508940895E89458
:10147000BB2766277727CB0197F9089555DF08F436
:101480008FEF08959B01AC0160E070E080E89FE37E
:1014900033CE6ECF64C1D1DFE8F39923D9F3940F33
:1014A000511DBBF39150504094F059F0882332F015
:1014B000660F771F881F91505040C1F79E3F51051E
:1014C00044F7880F911D9695879597F908955F3F8A
:1014D000ACF0983E9CF0BB27869577956795B795BD
:1014E00008F4B1609395C1F7BB0F58F711F460FF92
:1014F000E8CF6F5F7F4F8F4F9F4FE3CFB9CF0AD0B9
:1015000029ED3BE54EED5EE378C00EF028C136CF05
:1015100068942ECF92DFC8F39923D1F3C6F3DF93FB
:10152000CF931F930F93FF92C92FDD2788232AF0B3
:101530002197660F771F881FDAF720E030E040E838
:101540005FEB9FE3883920F0803E30F021968F7763
:1015500009DDE5E8F1E003C005DDE2EBF1E021DFC4
:101560008B01BE01EC01FB2E6F5771097595771F3A
:10157000880B990B60DE28E132E741E35FE349D055
:10158000AF2D9801AE01FF900F911F91CF91DF9188
:10159000FADC3ACFFA01DC01AA0FBB1F9B01AC01B8
:1015A000BF5728F422273327442750781FC0B7514C
:1015B00088F4AB2F0024469537952795011CA395F9
:1015C000D2F3002069F0220F331F441FB395DAF3E2
:1015D0000DD0C7CC61307105A0E88A07B94630F458
:1015E0009B01AC016627772788279078309621F0F9
:1015F000208331834283538308950BD005CFF6DED9
:1016000028F0FBDE18F0952309F0B2CEB7CE1124F6
:101610002FCF0BDFA0F3959FD1F3950F50E0551F0F
:10162000629FF001729FBB27F00DB11D639FAA2737
:10163000F00DB11DAA1F649F6627B00DA11D661F86
:10164000829F2227B00DA11D621F739FB00DA11DA7
:10165000621F839FA00D611D221F749F3327A00D61
:10166000611D231F849F600D211D822F762F6A2FFD
:1016700011249F5750408AF0E1F088234AF0EE0F82
:10168000FF1FBB1F661F771F881F91505040A9F78F
:101690009E3F510570F06CCEEBCE5F3FECF3983E71
:1016A000DCF3869577956795B795F795E7959F5FF6
:1016B000C1F7FE2B880F911D9695879597F9089590
:1016C000FA01EE0FFF1F30962105310599F16115E2
:1016D000710561F48038BFE39B0749F16894903845
:1016E000810561F08038BFEF9B0741F0992342F5F7
:1016F000FF3FE1053105210511F1E8940894E795D4
:10170000D901AA2329F4AB2FBE2FF85FD0F310C064
:10171000FF5F70F4A695E0F7F73950F019F0FF3A43
:1017200038F49F779F930CD00F9007FC9058089542
:101730003EF024CE60E070E080E89FE308954FE73C
:101740009F775F934F933F932F93E4DE2F913F91C9
:101750004F915F9152DF3DCD9B01AC014ECF9F3F3A
:1017600031F0915020F4879577956795B795880F5C
:10177000911D9695879597F908950E94C58B3323FF
:1017800012F48A1B9B0B0C94D68BA29FB001B39FC3
:10179000C001A39F700D811D1124911DB29F700D7A
:1017A000811D1124911D08950E94C58BB7FF0895D6
:1017B000821B930B08950E94C58BA59F900DB49F2B
:1017C000900DA49F800D911D11240895B7FF0C94D6
:1017D000DB8B0E94DB8B821B930B0895DB018F93C5
:1017E0009F930E94DB8BBF91AF91A29F800D911DB3
:1017F000A39F900DB29F900D11240895AA1BBB1BAF
:1018000051E107C0AA1FBB1FA617B70710F0A61B00
:10181000B70B881F991F5A95A9F780959095BC0121
:10182000CD01089597FB072E16F4009407D077FD9D
:1018300009D00E94FE8B07FC05D03EF4909581955F
:101840009F4F0895709561957F4F0895A1E21A2EDC
:10185000AA1BBB1BFD010DC0AA1FBB1FEE1FFF1F54
:10186000A217B307E407F50720F0A21BB30BE40BA4
:10187000F50B661F771F881F991F1A9469F76095EB
:101880007095809590959B01AC01BD01CF010895A5
:10189000052E97FB1EF400940E94738D57FD07D010
:1018A0000E94268C07FC03D04EF40C94738D509547
:1018B0004095309521953F4F4F4F5F4F0895689465
:1018C00001C0E894F92FF12B12F00C94938CA0E056
:1018D000B0E0EDE6FCE80C94918D092E059422F41D
:1018E0000E947B8D112392F4F0E80F26FFEFE09425
:1018F000F09400951095B094C094D094A194BF0A30
:10190000CF0ADF0AEF0AFF0A0F0B1F0B0E94228D7E
:1019100007FC0E947B8DCDB7DEB7ECE00C94AD8D5B
:10192000689401C0E8948F929F92CF93DF930E94B6
:10193000228DDF91CF919F908F900895DF93CF9369
:101940001F930F939A9DF02D219FF00D8B9DF00D0D
:101950008A9DE02DF10D039FF00D029FE00DF11D1A
:101960004E9DE00DF11D5E9DF00D4F9DF00D7F939E
:101970006F93BF92AF925F934F93D5010E94C58B37
:101980008B01AC01D7010E94C58BEB01E80FF91F59
:10199000D6010E94EE8C2F913F91D6010E94C58BFB
:1019A000C60FD71FE81FF91FAF91BF910E94EE8CA1
:1019B0002F913F910E94C58BC60FD71FE81FF91FBB
:1019C000D6010E94C58BE60FF71F9801BE01CF011B
:1019D00011240F911F91CF91DF9108950E94C58B23
:1019E000460F571FC81FD91F08F431960895E89471
:1019F000DF93CF93FC01DB010E94C58B7F936F9334
:101A0000E9019A01AC01BF93AF933F932F93DF019C
:101A10000E94C58B26F46C1B7D0B820B930B9E01E1
:101A2000EB01FC010E94EE8CAF91BF912F913F9191
:101A30000E94EE8CBE01CF01F9012F913F91CF9111
:101A4000DF91089588249924F401E401B0E49F9380
:101A5000AA279A158B049C04ED05FE05CF05D00737
:101A6000A10798F4AD2FDC2FCF2FFE2FE92D982C56
:101A7000892E982F872F762F652F542F432F322FA3
:101A80002227B85031F7BF9127C01B2EBF91BB272B
:101A9000220F331F441F551F661F771F881F991F72
:101AA000881C991CEE1FFF1FCC1FDD1FAA1FBB1F28
:101AB0008A149B04EC05FD05CE05DF05A007B107E0
:101AC00048F08A189B08EC09FD09CE09DF09A00B34
:101AD000B10B21601A94E1F62EF49401AF01BE011E
:101AE000CD01000C089590958095709561957F4F7C
:101AF0008F4F9F4F08956095709580959095309584
:101B00004095509521953F4F4F4F5F4F6F4F7F4FFF
:101B10008F4F9F4F08952F923F924F925F926F92F7
:101B20007F928F929F92AF92BF92CF92DF92EF926D
:101B3000FF920F931F93CF93DF93CDB7DEB7CA1BEE
:101B4000DB0B0FB6F894DEBF0FBECDBF09942A8819
:101B5000398848885F846E847D848C849B84AA84C1
:101B6000B984C884DF80EE80FD800C811B81AA814E
:101B7000B981CE0FD11D0FB6F894DEBF0FBECDBF19
:101B8000ED010895EE0FFF1F0590F491E02D0994EB
:101B900069279627692778278727782708950F933D
:101BA000083090F0982F872F762F652F542F432FD2
:101BB000322F22270850F4CF220F331F441F551F06
:101BC000661F771F881F991F0A95B2F70F91089516
:101BD00097FB10F8169400080F93083098F00850FF
:101BE000232F342F452F562F672F782F892F902D95
:101BF000F4CF059497958795779567955795479571
:101C0000379527950A95AAF70F9108952A0D3B1D40
